:1000000000800020BD01000005FA0000D1F90000C9
:10001000D1F90000D1F90000D1F90000D1F90000B8
:10002000D1F90000D1F90000D1F9000005FA000073
:1000300005FA0000D1F90000CD150100911601006C
:1000400005FA000005FA000005FA000005FA0000B4
:1000500005FA000005FA000005FA000005FA0000A4
:1000600005FA000005FA000005FA000005FA000094
:1000700005FA000005FA000005FA000005FA000084
:1000800005FA000005FA000005FA000005FA000074
:1000900005FA000005FA000005FA000005FA000064
:1000A000E1E10000EDE1000005FA000005FA0000C2
:1000B00005FA000005FA000005FA000005FA000044
:1000C00005FA000005FA000005FA000005FA000034
:1000D00005FA000005FA000005FA000005FA000024
:1000E00005FA000005FA000005FA000005FA000014
:1000F00005FA00003D08010005FA0000551E010048
:1001000005FA0000711F010005FA000005FA000061
:1001100005FA000005FA000005FA000005FA0000E3
:1001200005FA000005FA000005FA000005FA0000D3
:1001300005FA000005FA000005FA000005FA0000C3
:1001400005FA000005FA000005FA000005FA0000B3
:100150005D1801007118010085180100991801004F
:1001600005FA0000D10A010005FA000005FA0000B6
:1001700005FA000005FA000005FA000005FA000083
:1001800005FA000005FA000005FA000005FA000073
:1001900005FA000005FA000005FA000005FA000063
:1001A00005FA000005FA000005FA000005FA000053
:1001B00005FA000005FA000005FA0000564B4CF263
:1001C000205210B51A804DF628121A8000BF00BFC9
:1001D00008F0EEFF514B4FF010621A60504A9A60DF
:1001E000504ADA60504A136813F4807301BF4F49D4
:1001F0000B604FF4A85313604D4B4E491A7810070B
:1002000042BF1A7842F008021A704B4B2A221A7029
:100210004A4A4B4B8B4204D252F8040F43F8040B6A
:10022000F8E7484B484A0021934202D243F8041BA6
:10023000FAE7464A4648002350F8231042F82310B4
:1002400001336F2BF8D1434B434A802103F8011B44
:100250009342FBD1414B3D4A1A60414B8A221A70AE
:10026000A3F5805324225A70A0221A709A7991071C
:10027000FCD59A79D206FCD43A4A937903F00C0360
:10028000082B384BF9D103221A7140225A719A79FE
:100290009406FCD533498A79324B5006FBD5324A55
:1002A000324911600221516020221A709A7902F0BD
:1002B0000C020C2AFAD12E4B2E4A1A602E4B2F4AD2
:1002C0001A6000225A60072243F8042C2C4AC3F813
:1002D0000C2D62B60FF078FF144B1B68DA0705D5BA
:1002E00028480FF071FD284B284A1A60284B1B78CC
:1002F0005B0609D5244C254B22689A4204D121483B
:100300000FF062FD0023236015F088F90FF07DFBEC
:1003100011F028FDFEE700BF0E20054030800440AC
:10032000823F04000100002B10D0034014D0034092
:1003300002D00740D895FF1F00E00740E0B701005A
:100340002089FF1FD895FF1F54A0FF1F0084FF1FA7
:100350000000000000E400E05FE400E008ED00E0E1
:100360000050064000400640448004400000030165
:1003700004800440C010050014E000E0FF76010096
:1003800000002020C3CB375F1CE00340A5C3945A74
:1003900000F00740FFFFFFFFFFFFFFFFFFFFFFFF32
:1003A000FFFFFFFFFFFFFFFFFFFFFFFFFFFFFFFF5D
:1003B000FFFFFFFFFFFFFFFFFFFFFFFFFFFFFFFF4D
:1003C000FFFFFFFFFFFFFFFFFFFFFFFFFFFFFFFF3D
:1003D000FFFFFFFFFFFFFFFFFFFFFFFFFFFFFFFF2D
:1003E000FFFFFFFFFFFFFFFFFFFFFFFFFFFFFFFF1D
:1003F000FFFFFFFFFFFFFFFFFFFFFFFFFFFFFFFF0D
:10040000FFFFFFFFFFFFFFFFFFFFFFFFDEF9FFFF23
:1004100010B5054C237833B9044B13B10448AFF33E
:1004200000800123237010BDD895FF1F000000003D
:10043000DCB70100084B10B51BB108490848AFF301
:1004400000800848036803B910BD074B002BFBD0A0
:10045000BDE81040184700BF00000000DC95FF1FFA
:10046000DCB70100D895FF1F0000000040F6FF72C6
:100470009142044B28BF11468AB2C1B218680CF0F1
:1004800071BD00BFF495FF1F10B4B8B10A2840F643
:10049000FF7328BF0A20994200F1FF300A4628BFA7
:1004A0001A46074B33F91040064B13F81010064B51
:1004B00092B253F8240010BC0CF054BD10BC70472D
:1004C000B4960100C8960100F495FF1F084A012365
:1004D0000221136042F8403C42F8401C2022013ABD
:1004E000FDD1044A136042F8403C42F8401C70477A
:1004F00088F00F4084F00F402DE9F34101210F20D7
:100500000FF0AEFC1F4B204D01241C602146102033
:100510000FF0A6FC2C60214611200FF0A1FC022355
:100520002B601A4D27464FF0000855F8043F3BB9A1
:10053000342011F01FFCE1B206460CF083FC2E6063
:10054000012300971A46194628680CF0A1FC0023E5
:10055000CDF800801A46194628680CF0C1FC002628
:10056000F1B20022286801360CF0FCFC042EF7D111
:100570000134042CD9D1FFF7A9FF002002B0BDE857
:10058000F08100BF84F00F4044F00F40F095FF1F52
:10059000072A2DE9F74F0D469046994600F28D80C7
:1005A000072900F28A80C6B201213046454F464CE9
:1005B0000FF056FC0A200FF0F1FD57F83630617B42
:1005C00020694FF0010A83F880A00CF09FFF3F4A9A
:1005D0003F4920690CF002FEEDB232200FF0DEFD43
:1005E0005FFA88FB45F060012046AD000CF0E3FFA8
:1005F00045F061014FEA8B05EDB201F0FD012046A7
:100600000CF0B8FC45F0620120460CF0B3FC45F05C
:10061000630120460CF0AEFC72B600235246617BAB
:1006200020690CF0D5FF4FF4B353013BFDD157F8CF
:10063000363083F800A162B60022617B20690DF09C
:1006400049FA0546B9F1000F08D0224808F078F8B9
:10065000554514BF2048214808F00CF964200FF0DC
:100660009DFD57F836301848012583F880504BF02F
:1006700060010CF0A0FF0026062113480CF07AFC64
:10068000627B00962B4621690F480DF064FA60B931
:10069000B9F1000F0AD0124808F052F8404608F0AD
:1006A000C5F8104808F0E6F800E0354620690E4A23
:1006B00007490CF093FD284601E04FF0FF3003B0EE
:1006C000BDE8F08F38B00100F49CFF1FA086010048
:1006D000006CDC02DC960100EA960100F296010053
:1006E000F996010097A20100801A060010B5044691
:1006F00008F0CAFA2346012200210F20FFF748FF25
:100700002346022200211020FFF742FF2346032246
:1007100000211120BDE81040FFF73ABF38B50F4C5B
:10072000236843B9102011F025FB0D4A0D490546F9
:100730000BF0A0FD256020684FF07E510BF020FEED
:10074000206809490BF0A6FD206801210BF0C0FDCF
:100750002068BDE838400BF0F1BD00BF0096FF1FD8
:1007600009CE0000F5CE00000000484270B50D46ED
:1007700090B00021064614F0B5FC044620B106F105
:10078000004014F0E3FC2BE00146202268460EF006
:10079000CBFE154B19686B1E2046C3EBC302131822
:1007A000D43301EB43039B889BB24DF820300130DA
:1007B0000728F4D105F2A71508AC31F815300B4D18
:1007C0009BB207930FCD0FC495E80F0084E80F008C
:1007D000304614F0BBFC08236A4608A900F0B4FDBB
:1007E00080B210B070BD00BFBC8CFF1F0497010029
:1007F00038B50D460146044614F092FC00B10024C1
:1008000029462046BDE83840FFF7B0BF2DE9F74F35
:100810009846274B1C689246E26D236E01938B46E7
:100820000146104614F0B6FA019BD4F86490A76E06
:10083000A56D06465946184614F0ACFA01463046F6
:1008400014F0A0F951460646484614F0A3FA0146B2
:10085000304614F097F941460646384614F09AFAA5
:100860000146304614F08EF9294614F08BF94FF00A
:1008700080410546D4F8980014F02AFC28B1D4F839
:1008800098000C4914F038FC30B90021284614F0C7
:100890001FFC40B1002506E02846D4F8981014F05B
:1008A00079FA0546F1E7284603B0BDE8F08F00BFAE
:1008B000BC8CFF1FCDCC4C3E2DE9F047384DDFF806
:1008C000FC80384F384EDFF8F8900446FFF726FFDB
:1008D00032200FF063FC002C286808BF01240BF0C5
:1008E000ABFD14F0FFF9C8F8000028680BF0ABFD71
:1008F00014F0F8F9386028680BF0ACFD14F0F2F948
:10090000306028680BF091FD14F0ECF933683A6818
:10091000D8F80010C9F80000FFF778FF234B002C2F
:100920000546186038DD204614F0E0F9DFF894A0A1
:1009300004460146D8F80000DFF88C8014F0DEFA97
:10094000DAF8001014F01EF92146CAF800003868E1
:10095000174F14F0D3FAD8F8001014F013F9214609
:10096000C8F800003068134E14F0C8FA396814F063
:1009700009F921463860D9F8000014F0BFFA31684F
:1009800014F000F930600C4E2146284614F0B6FAF7
:10099000316814F0F7F830602846BDE8F08700BFF2
:1009A0000096FF1F3896FF1F2C96FF1F3C99FF1FD4
:1009B0005C97FF1F7497FF1F3096FF1F4096FF1F25
:1009C0005096FF1F3099FF1F4899FF1F10B53049FF
:1009D000044615F081F908B92E4B0BE02E4920464C
:1009E00015F07AF90028F7D02C49204615F074F953
:1009F00010B92B4B186810BD2A49204615F06CF928
:100A00000028F6D02849204615F066F90028F0D0D5
:100A10002649204615F060F90028DDD00D22244932
:100A2000204615F073F928B107222249204615F017
:100A30006DF910B904F10D0006E003221E492046AD
:100A400015F064F920B9E01C14F0B5FD1B4B18E05B
:100A50000B221B49204615F059F928B107221949E4
:100A6000204615F053F910B904F10B0006E00322FB
:100A70001549204615F04AF940B9E01C14F09BFDD9
:100A8000124B53F8200014F031F910BD002010BDB6
:100A9000A3A501003C99FF1F2D9701002497010099
:100AA0007C99FF1F3D970100459701004D9701007C
:100AB00055970100639701006B970100C496FF1FD3
:100AC0006F9701007B970100839701001C97FF1F20
:100AD0002DE9F043334C25686E1C26602F78282FB3
:100AE0008FB00AD100F062F823685A1C22601B788C
:100AF000292B05463AD02C4D38E0A7F12B03DBB269
:100B00000E2B0DD847F6ED7222FA03F3DB0707D55B
:100B10002846214615F064FF13F0DEFF054625E068
:100B2000384614F0AAFD08B95F2FE4D12560B0461D
:100B300018F8017B384614F097FD814608B1464607
:100B4000F5E707F0FB035B2BF9D05D2FF7D0771BA0
:100B50003A46294601A815F0EEF80EAB1F4401A84D
:100B600007F8349CFFF732FF2660054623685A1CBD
:100B700022601C782A2C01D02F2C0CD1FFF7A8FF63
:100B80002A2C0146284602D114F004F901E014F0A1
:100B9000B5F9054601E0034A136028460FB0BDE8E9
:100BA000F08300BF0496FF1F0000C07F38B5FFF739
:100BB0008FFF0D4B1A68511C196015782D2D0446B6
:100BC00001D02B2D0CD1FFF7F1FF2B2D0146204634
:100BD00002D113F0D7FF01E013F0D2FF044600E08A
:100BE0001A60204638BD00BF0496FF1F014B1860F5
:100BF000FFF7DCBF0496FF1F10B54FF40234A4F5D5
:100C0000006003469C4205D804F50064B4F5802FCB
:100C1000F5D110BD53F8042B0132F3D000211AF0A6
:100C2000C3FD01460028EFD0014807F0C3FDEBE704
:100C3000C39701002DE9F04300241C601E46037891
:100C400085B03A2B05460F469146DDF8308009D134
:100C500015F054F80A2850D901AA2A49681C15F041
:100C600001F808B9002049E0284615F047F8019B33
:100C70005B000B339842F5D34A462349E81C14F035
:100C8000F1FF0028EED042461E49E81D14F0EAFFAD
:100C90000028E7D09DF8044098F80030D9F800000B
:100CA000234453FA80F3C0F3072009351C18326837
:100CB000019B9A4213D003AA1249284614F0D2FF8E
:100CC0000028CFD03368039AFA543368FA5C0133B2
:100CD000FF2B05F1020514443360E8D9C2E702AAEC
:100CE0000849284614F0BEFF0028BBD002982044D3
:100CF000C0B2B0FA80F0400900E0204605B0BDE87F
:100D0000F08300BFD9970100DE9701002DE9F0477D
:100D100002234FF48072D8B09049914807F04AFD01
:100D2000FFF76AFF8F4B904A9A4205D98F4A9A4241
:100D300002D98F4A9A4201D88E4812E04FF400330C
:100D40001A6801321C46A3F1040302D1002BF7D12B
:100D50001C46211D884807F02DFDB4F5FC3F05DD3C
:100D6000864807F027FD58B0BDE8F0878448854ED7
:100D700007F020FD844807F01DFD0024354607F0EC
:100D8000D5FB0028FBD007F0B5FB58AB0A2823445D
:100D900002D00D2840F0CE80002203F8C82C9DF828
:100DA00098303A2B40F0C4803368002B40F0C0806C
:100DB00005AA7649764F26A814F054FF012827D1BA
:100DC00005993A6891421FD1724B1B68E3B1DFF875
:100DD000E481714CD8F800202168704807F0EAFCE3
:100DE00064200FF0DBF9D8F8001020681AF0E4FC5A
:100DF000011E03DD6A4807F0DDFC99E0D8F8001019
:100E000020681AF0CDFC03E0664807F0D3FC8FE0C1
:100E10003B68DFF8BC91013304AC3B604A46009468
:100E200003AB06A926A8FFF705FF28B926A95E4847
:100E300007F0C0FC012348E05C48D9F80030D0F846
:100E400000A0039A53449918B1F5FC3F04D95848BF
:100E500007F0B0FC022338E02168042930D8DFE82D
:100E600001F03603232F29004FF47A700FF096F922
:100E7000494C39684F4F00913B6822684E4807F053
:100E800099FC3F68246807F5FF3704F5003407F53F
:100E9000FA77A74256D90C223049204614F036FF83
:100EA00000284BD00134F4E7BDF818305BBA9BB290
:100EB0001B0103E0BDF818305BBA1B04036037E088
:100EC00026AA3E4807F076FC03232B6030E003F5AA
:100ED000003818F0030F06D1910704D102F5003451
:100EE00005AF1C4405E0364807F064FC2EE008F12D
:100EF0000408C8EB0403002B0BDD57F8041F404621
:100F00001AF056FC01460028F1D02E4807F052FC9A
:100F10001CE0D9F800302749039A086853441A4462
:100F2000824200D90A601C4A11688B4238BF1360A4
:100F3000002424E703F8C80C013420E7154B0122F4
:100F40001A60F5E7204807F035FCF1E7D9F80020F2
:100F500003991E4807F02EFC0423B6E7E39701002F
:100F6000F0970100FFFF03002189FF1FD589FF1FB4
:100F7000558AFF1F1498010029980100409801002C
:100F8000579801000C96FF1F7B980100989801006C
:100F90001C96FF1F1896FF1FB48CFF1FA29801001C
:100FA000B9980100C5980100EA9801001496FF1F46
:100FB000FB9801000896FF1F0E9901004E99010051
:100FC00068990100819901009D990100BA99010079
:100FD0001096FF1F10B5044610F01EFC204610BDF1
:100FE000114B1A6870B51D46EAB972B60F4B104A1C
:100FF0001C88104B1B78D05C0F4A52F8301001232C
:1010000081F8803020210139FDD10C4940260E6045
:1010100010260E6061010CB10139FDD152F830206B
:1010200082F800312B6070BD3098FF1F1497FF1FAE
:10103000189A01002C98FF1F38B00100C8F00F402B
:10104000074B421E9A4209D8302303FB00F2013AB3
:10105000232A03D90349044810F096BB704700BF08
:1010600057555505E10F00005099FF1F0368C9B29D
:101070001B68184710B504782CB10130FFF7FAFF50
:1010800000FB044010BD44F2AD3010BD70B54FF40C
:101090007A71124807F08AFC064623200EF0CCFB3A
:1010A000054623200EF0C8FB054423200EF0C4FBA8
:1010B00004460B4807F044FB2819032490FBF4F086
:1010C00013F014FE214607F099FB07F0FBFB01200B
:1010D0000FF064F80136DAD170BD00BF42A0010004
:1010E000289A010038B5054635B14FF47A71244885
:1010F00007F05CFC044601E04FF0FF34214807F0A4
:101100001FFB21480AF094FD022107F077FB1F48DE
:1011100007F016FB1C480AF0AFFD022107F06EFB3A
:101120001B4807F00DFB18480AF0E9FD022107F003
:1011300065FB184807F09EFB124807F001FB1648B4
:101140000AF076FD022107F059FB144807F0F8FA7F
:1011500011480AF091FD022107F050FB0C4807F0FE
:10116000EFFA0D480AF0CBFD022107F047FB0948D2
:1011700007F080FB64200FF011F80134B4D138BDC2
:1011800042A001002F9A01005C96FF1F329A0100D5
:10119000369A010097A201009096FF1F339A010032
:1011A0002DE9F74F424C434E8DE80300FFF7B6FAA6
:1011B0002546A246009B33B14FF47A713E4807F0B2
:1011C000F5FB074601E04FF0FF374FF004083220EF
:1011D0000EF0E4FF0420FFF76FFBB8F10108206078
:1011E000F5D1364ADFF8FC90DFF8FC8000234FF49D
:1011F0002F703360C9F80030C8F8003013602B60DE
:101200000EF0CCFF4FF0040B14200EF0C7FF0420AB
:10121000FFF752FBBBF1010BCAF80000F4D1284ADA
:10122000019B1060274A1168274A1160214A116802
:10123000264A1160264AD9F800101160254AD8F8CC
:101240000010DFF878801160234AD8F80010116090
:10125000224AA2F800B023B90137ABD103B0BDE8F0
:10126000F08F1F4807F06CFA3068012107F0C6FACA
:1012700007F028FB1B4B0121186807F0BFFA07F0A5
:1012800021FB194B0121186807F0B8FA07F01AFB87
:10129000D8F80000012107F0B1FA07F013FB286825
:1012A000032107F0ABFA114807F0E4FAD4E700BFD6
:1012B0003096FF1F3099FF1F42A001007497FF1F57
:1012C0004C99FF1F3C99FF1F7C99FF1F7099FF1FCE
:1012D000F096FF1F8897FF1FD497FF1F8097FF1F6F
:1012E000399A01004899FF1F5C97FF1F77A60100FC
:1012F00010B50446FFF7C8F8FFF7E8F8044B1A5D8D
:10130000044B53F83230012283F8802010BD00BF17
:10131000189A010038B0010070B5094D094E01243A
:1013200020460021FFF7B0F8FFF7D0F8A35D0122B7
:1013300055F8333014440B2C83F80021F0D170BDE4
:1013400038B00100189A010070B50C68844201DBC6
:10135000106870BD03F18043013B51F82340A04267
:101360001CDA01231CB2A60051F82440A04202DD81
:101370000133DBB2F6E701D1905970BD03F1804330
:10138000013B51F8235052F8231093595A1A431B2A
:101390005343601B93FBF0F0084470BD52F82300E8
:1013A00070BDFFFF30B5174C85B00546D0212046F3
:1013B0000CF001F9290A2046FFF758FEE9B2204651
:1013C0000025FFF753FE627B21690095012320462B
:1013D0000CF0C1FB01230093617B01950823D0220F
:1013E00020690CF0CDFB20690CF0E2FB02AB20EA97
:1013F000E070E8540135082DF5D1DDE9020105B0B2
:1014000030BD00BFE09CFF1FF0B585B004A961E9C5
:101410000223144E00F1080704460D1AD02111488A
:101420000CF0C9F8210A0F48FFF720FEE1B20D4881
:10143000FFF71CFE295D0B48FFF718FE05200EF094
:10144000ADFE0023727B00933169064801230CF046
:1014500082FB013405200EF0A1FEA742DED105B0CB
:10146000F0BD00BFE09CFF1F2DE9F0411C4CDFF8F0
:101470008C801C4F054620460AF0DAFBC8F80000B5
:1014800020460AF0F9FB386020460AF038FC16497D
:1014900013F034FD154B06461860284613F026FC61
:1014A000134D04460146D8F8000013F027FD2968C3
:1014B00013F068FB28600F4D3868214613F01EFDBD
:1014C000296813F05FFB28600B4D2146304613F06E
:1014D00015FD296813F056FB2860BDE8F08100BFB8
:1014E0005C96FF1F2896FF1F0000C842A897FF1FA9
:1014F0003499FF1F9497FF1FF896FF1F5899FF1FFD
:101500002DE9F0411C4CDFF88C801C4F054620462D
:101510000AF08EFBC8F8000020460AF0ADFB3860E8
:1015200020460AF0ECFB164913F0E8FC154B064682
:101530001860284613F0DAFB134D04460146D8F82C
:10154000000013F0DBFC296813F01CFB28600F4D32
:101550003868214613F0D2FC296813F013FB286089
:101560000B4D2146304613F0C9FC296813F00AFBE5
:101570002860BDE8F08100BF9096FF1F3C96FF1FDA
:101580000000C842F097FF1F1897FF1F3899FF1FF0
:101590007C97FF1FFC96FF1F2DE9F04F1E463C4B2A
:1015A00080460D46101E4FF000018FB0196001DA21
:1015B000414206E0ACB213F099FB2146FFF718F95F
:1015C00001462846FEF760FFFEF780FF701E0021EF
:1015D00009F05CFF0A200EF0E1FD189EDFF8C4A0C0
:1015E0004FF0400976010DF102074FF6FF74CB462C
:1015F0004FF4FA43013BFDD172B6264A264B515DAA
:1016000053F83110012081F8800020210139FDD1EB
:101610001021CAF800B0CAF8001016B131460139DD
:10162000FDD1525D53F83230032C4FF0010283F8A4
:1016300000210AD8132104A809F0C6FF4FF07C52FC
:10164000132104A807F08AFB388062B60134134BDB
:10165000A4B21022042C1A6007F10207C3F800900C
:10166000C6D14FF07C52052101A807F077FB199CE9
:101670000B4D90FBF8F0013C13F038FB55F82410AB
:1016800013F080FA45F824000FB0BDE8F08F00BFDA
:10169000CC97FF1F189A010038B00100C4F00F402A
:1016A0004497FF1FC8F00F4070B5064600200AF0AF
:1016B000F3FC044600200AF0EFFC0146204613F03C
:1016C00061FA044600200AF0E7FC0146204613F0C8
:1016D00059FA0A490A4D13F011FC0A4B04461860E6
:1016E000304613F003FB0146204613F007FC29683F
:1016F00013F048FA2860204670BD00BF000040404B
:101700005896FF1F1899FF1F2DE9F04F9BB00DA9A8
:101710000CA893460EAA0BF0ABF811AA10A90FA8BB
:101720000AF050FD0F9B1293109B139312A8119B6C
:10173000149308F087F914991398AD4CAD4DAE4F42
:10174000DFF818A308F098F9206012A807C823460C
:1017500008F09CFA3B6828600246216815A808F04A
:10176000C5FA3A462946204608F070F9159812F055
:1017700067FECAE900010F9813F0B8FA9F4B186092
:10178000109813F0B3FA9E4B1860119813F0AEFA4C
:101790009C4B18609C4B0C98D3F80080D8F80C90A8
:1017A000D8F8086013F0A2FA494613F0E9F90146A7
:1017B00013F0E8F9314613F0A1FB944AD8F81890D9
:1017C00010600B900D98D8F8146013F08FFA49460A
:1017D00013F0D6F9014613F0D5F9314613F08EFB1C
:1017E0008B4AD8F82490106006460E98D8F82080CE
:1017F00013F07CFA494613F0C3F9014613F0C2F91D
:10180000414613F07BFB83490290086082492068BF
:1018100013F074FB12F014FE8046894610F0EAFDC6
:10182000029ACDE90001104612F00AFECDE902014C
:101830004046494610F02CFECDE90401764928685F
:1018400013F05CFB12F0FCFD8046894610F0D2FDDF
:10185000CDE906014046494610F01AFE0B9BCDE942
:101860000801184612F0ECFDDDE9002312F03CFE01
:10187000DDE9042380468946DDE9020112F034FEE9
:1018800002460B464046494612F07CFCDDE9042343
:1018900080468946DDE9000112F074FC02460B46E1
:1018A0004046494612F04AFF13F016F912F0C8FDFF
:1018B000CDE90001304612F0C3FDDDE9062312F048
:1018C00013FEDDE9082380468946DDE9020112F0B6
:1018D0000BFE02460B464046494612F053FCDDE93A
:1018E000082389468046DDE9060112F04BFC0246DA
:1018F0000B464046494612F021FF13F0EDF812F076
:101900009FFDDDE9002310F02BFE37A3D3E9002370
:1019100012F0EAFD0022414B12F034FC13F0DCF827
:101920000021064613F0F2FBB94608B93E6004E018
:101930003B49304613F024F93860D9F800003849A3
:10194000384EDFF81C81384F13F01CF9374B2268F2
:101950001A602A68C9F800003260C8F80000DAE9A5
:101960000001009313F0B8F831493860314810F0A5
:1019700090F9D9F800403049DFF8B890204613F0CC
:10198000A7FB009B1D4620B92C49204613F0BEFB47
:1019900008B12B4995E02849204613F0B7FB38B130
:1019A0002849204613F09EFB10B12749484689E09C
:1019B0002449204613F0AAFB30B12449204613F0F5
:1019C00091FB08B122497CE02049204613F09EFBA0
:1019D000002847D01F49204613F084FB002841D03F
:1019E0001D496EE0AFF3008000000000DCA54C4014
:1019F000EC96FF1F0497FF1F0897FF1FFC97FF1F20
:101A00006C97FF1F0098FF1FBC8CFF1F8497FF1F60
:101A10000899FF1F0499FF1FE02E65420080564081
:101A20000000B4433496FF1F5496FF1FA497FF1F76
:101A30004D9A01006099FF1F0000B44100C0A84307
:101A4000509A010000008742539A01000000E142D1
:101A5000569A010000801D43599A0100E897FF1F24
:101A60009097FF1F4249204613F050FB30B1414987
:101A7000204613F037FB08B13F4922E03D4920469C
:101A800013F044FB30B13D49204613F02BFB08B165
:101A90003B4916E03949204613F038FB30B139494B
:101AA000204613F01FFB08B137490AE035492046AC
:101AB00013F02CFB40B13549204613F013FB18B14D
:101AC0003349344810F0E5F8BBF1010F49D13248F1
:101AD00006F036FED9F8000006F032FE2F4806F078
:101AE0002FFE2F4806F02CFED8F80010084613F001
:101AF00017FB10B12B4B2C4A1A600221D8F80000BA
:101B000006F07CFE294806F01BFE3968084613F0F3
:101B100007FB10B1264B244A1A600321386806F0EF
:101B20006DFE244806F00CFE3168084613F0F8FA02
:101B300010B1214B1C4A1A600221306806F05EFE8B
:101B40001E4806F0FDFD2968084613F0E9FA10B1B9
:101B50001B4B154A1A600221286806F04FFE06F05A
:101B6000B1FE16A80FF0C0FF1BB0BDE8F08F00BF9C
:101B700000801D4300804A435C9A01000080774347
:101B80005F9A010000409243629A010000C0A8439E
:101B9000659A01006099FF1F689A010096A20100F2
:101BA0007E9A01009097FF1F000080BF899A010074
:101BB0005496FF1F939A01003496FF1F9D9A0100CF
:101BC000A497FF1F2DE9F84307460E464FF47A7598
:101BD000002423200DF030FE013D0444F9D1274BB1
:101BE0004FF47A7094FBF0F01860254B1D6813F0E9
:101BF0007DF8D5F88C80D5F89090D5F894500446AF
:101C00000146404613F0C6F8214613F0C3F81D49BB
:101C100013F074F949468046204613F0BBF801469C
:101C2000404612F0AFFF294612F0ACFF164913F000
:101C300065F9164B0546186067B9304613F056F83B
:101C4000134D0146204613F059F9296812F09AFF06
:101C5000286010E0012F0DD1304613F047F80D4CED
:101C60000146284613F04AF9216812F08BFF2060E4
:101C70002C4600E000242046BDE8F8833498FF1F7E
:101C8000BC8CFF1F286B6E4E00007A448C97FF1FA0
:101C90002C99FF1F0C99FF1FF8B50E464FF47A756B
:101CA0000024C7B238460DF0C7FD013D0444F9D108
:101CB0004FF47A7094FBF0F013F018F8084B094DCC
:101CC00018600446304613F011F80146204613F020
:101CD00015F9296812F056FF28602046F8BD00BFAC
:101CE000DC97FF1F0097FF1F70B5C0B20E460EF0C5
:101CF000A9F812F0F7FF094B094C18600546304669
:101D000012F0F4FF0146284613F0F8F8216812F0AB
:101D100039FF044B2060186870BD00BF8099FF1F19
:101D2000AC97FF1FDC97FF1F30B52B482B4C2C4D79
:101D300085B006F005FD2B4806F002FD022008F0F4
:101D4000D3FB06F073FD204606F0FAFC264806F0A9
:101D5000F7FC012008F0C8FB06F068FD204606F0FD
:101D6000EFFC224806F0ECFC2B680A22D3F898110D
:101D700068464FF47A73B1FBF3F10FF040FF684609
:101D800006F074FD204606F0DBFC68460FF0ACFE62
:101D9000174806F0D5FC002008F0A6FB06F046FD2B
:101DA000204606F0CDFC134806F0CAFC40F2FC6069
:101DB00006F03CFD204606F0C3FC08F079FF0E4813
:101DC00006F0BEFC2B6893F89C0006F02FFD0B4834
:101DD00006F0B6FC05B030BD50A9010097A2010085
:101DE000BC8CFF1FA69A0100B69A0100C59A01009B
:101DF000DA9A0100E49A0100F39A0100C0A0010000
:101E000038B52E4C2E4806F09BFC2368DD6D294624
:101E1000284613F085F900B12A4D0321284606F023
:101E2000EDFC294806F08CFC284806F089FC236864
:101E30001D6E2946284613F073F900B1214D032188
:101E4000284606F0DBFC204806F07AFC204806F025
:101E500077FC23685D6E2946284613F061F900B1CE
:101E6000184D0321284606F0C9FC174806F068FC07
:101E7000184806F065FC23689D6E2946284613F035
:101E80004FF900B10F4D0321284606F0B7FC0E486C
:101E900006F056FC104806F053FC23689C6D214662
:101EA000204613F03DF900B1064C2046032106F010
:101EB000A5FC0548BDE8384006F042BCBC8CFF1FBD
:101EC000FE9A0100000080BF77A60100129B01006E
:101ED000249B0100369B0100489B01001FB5084B65
:101EE0001A68D37891785078127802920190009114
:101EF000044A0549054806F05DFC05B05DF804FBA1
:101F0000BC8CFF1FEE970100579B0100619B0100F5
:101F10002DE9FF41FFF7E2FFAE48AF4C06F010FCA1
:101F2000AE4806F00DFCAE4806F00AFCAD4806F0DF
:101F300007FCAD4806F004FCA94806F001FCAB48DC
:101F400006F0FEFBAA4806F0FBFBAA4806F0F8FBE9
:101F5000A94806F0F5FBA94806F0F2FB08F0A8FE38
:101F6000A74806F0EDFB2368B3F8300380B206F013
:101F70005DFC9B4806F0E4FBA24806F0E1FB236809
:101F800093F82C0006F052FC954806F0D9FB9E48C9
:101F900006F0D6FB23689D682946284613F0C0F852
:101FA00000B19A4D0221284606F028FC8C4806F024
:101FB000C7FB974806F0C4FB23685D69294628469D
:101FC00013F0AEF800B1914D0221284606F016FC40
:101FD000834806F0B5FB8F4806F0B2FB23681D6A04
:101FE0002946284613F09CF800B1884D0221284666
:101FF00006F004FC7A4806F0A3FB874806F0A0FB35
:102000000025236805F5D47233F8120080B206F07B
:102010000DFC092D02D0724806F092FB01350A2D05
:10202000EFD17E4806F08CFBFFF7EAFE7C4806F015
:1020300087FB00257B4806F083FB00264FEAC50896
:1020400008EB0603226803F5907332F8130000B220
:1020500012F04CFE0146074613F062F800B16B4FD8
:102060000321384606F0CAFB01365D4806F068FBDE
:10207000072EE5D1236803EB0513B3F84E0200B237
:1020800012F034FE0146064613F04AF800B15F4EE6
:102090003046032106F0B2FB092D14BF5F486248A9
:1020A000013506F04DFB0A2DC4D1604806F048FB0F
:1020B0002368D3F88C502946284613F031F800B134
:1020C000524D0321284606F099FB454806F038FB9F
:1020D000574806F035FB2368D3F890502946284628
:1020E00013F01EF800B1494D0321284606F086FB87
:1020F0003B4806F025FB4F4806F022FB2368D3F847
:1021000094502946284613F00BF800B13F4D0321A7
:10211000284606F073FB324806F012FB464806F0EC
:102120000FFB236893F86C0112F0DCFD01460546B5
:1021300012F0F6FF00B1354D0121284606F05EFB96
:10214000274806F0FDFA3D4806F0FAFA2368B3F88E
:10215000680180B212F0C6FD0146054612F0E0FFAC
:1021600000B12A4D0321284606F048FB1C4806F022
:10217000E7FA334806F0E4FA2368B3F86A0180B25C
:1021800012F0B0FD0146054612F0CAFF00B11F4D26
:102190000321284606F032FB114806F0D1FA2948FF
:1021A00006F0CEFA2368D3F8A0512946284612F04B
:1021B000B7FF00B1154D0321284606F01FFB084864
:1021C00006F0BEFA204806F0BBFA2368D3F838526E
:1021D0003CE000BFB29B0100BC8CFF1FEE970100EA
:1021E00097A20100C49B0100D09B0100D79B010076
:1021F000E59B01003FA60100F19B010076A60100CE
:10220000FA9B0100089C0100179C0100000080BFA0
:10221000269C0100359C0100449C010077A601002A
:10222000509C010080A101005B9C01005F9C0100AB
:102230006E9C01007D9C01008C9C01009F9C010014
:10224000B09C0100C39C0100D19C01002946284696
:1022500012F066FF00B1764D0321284606F0CEFA53
:10226000744806F06DFA744806F06AFA2368D3F8E9
:102270003C522946284612F053FF00B16C4D6F4F77
:102280000321284606F0BAFA6A4806F059FA6C4863
:1022900006F056FA012008F027F906F0C7FA65485B
:1022A00006F04EFA674806F04BFA012008F01CF9D8
:1022B00006F0BCFA5F4806F043FA634806F040FABD
:1022C000022008F011F906F0B1FA5A4806F038FA7F
:1022D0005E4806F035FA23680A22D3F8981168465A
:1022E0004FF47A73B1FBF3F10FF089FC684606F006
:1022F000BDFA504806F024FA68460FF0F5FB544842
:1023000006F01EFA002008F0EFF806F08FFA4948B0
:1023100006F016FA4F4806F013FA072006F086FA80
:10232000444806F00DFA4C4806F00AFA00254B48DE
:1023300006F006FA0026C5EBC508236808EB06027E
:10234000D43203EB42030136988880B206F06EFA6D
:10235000384806F0F5F9062EEFD13A680E2303FB54
:102360000523B3F8B80180B206F060FA092D14BF56
:102370003B483C48013506F0E3F90A2DD7D13A48ED
:1023800006F0DEF9002523682C4E05F11E0203EB52
:1023900082030421586806F031FA0135254806F019
:1023A000CFF9032DEFD133680421D3F8880006F06C
:1023B00025FA2B4806F0C4F93468D4F8981008467A
:1023C00012F0AEFE30B9D4F89800002112F080FE71
:1023D000E8B10EE04FF07E55D4F89800294612F08F
:1023E0006DFE08B9C4F89850204A1378D907FCD577
:1023F000E9E74FF07E55D4F89800294612F05EFECA
:1024000008B9C4F89850194A1378DB07FCD5184866
:1024100006F096F9094B1B680321D3F8980006F0E3
:10242000EDF9144806F08CF904B0BDE8F08100BF66
:10243000000080BF97A20100E09C0100BC8CFF1F40
:10244000ED9C0100B69A0100FB9C0100C59A0100B9
:10245000DA9A01000B9D0100169D010080A1010088
:1024600077A601005B9C0100229D01000100024053
:10247000379D0100C0A00100012870B5054615D0A8
:10248000002006F06BFD0446FFF728FD1A4A1B48A2
:10249000214606F08FF9012D1CDC194806F050F991
:1024A000184806F04DF9FFF73FFC20E0164E0324D4
:1024B0000021164806F07AFA154B1B681A5DC0B267
:1024C000904218BF18553378DB07FCD514F1FF3460
:1024D000EED2D5E70F4806F033F90F4806F030F991
:1024E00040F2FC6006F0A2F90C4806F029F90B480E
:1024F000BDE8704006F024B9D09B0100449D010066
:102500006D9D010012A001000100024042A00100E7
:10251000BC8CFF1F1FA00100E49A0100C0A00100B5
:102520002DE9F04FA1B0054606F0AEFB2C4628463B
:1025300013F0E4FB631B834208D214F8010B13F081
:10254000A5F80028F3D104F8010CF0E72C78002C52
:1025500001F0DF83204613F087F8002801F0D983CB
:10256000303C092C284602D813F025F801E0FEF78C
:1025700081FDC84B9842044601F0B38300F2058206
:10258000C54B984201F0158000F2A480C34B9842DD
:1025900000F0148440D840F21D43984201F0398382
:1025A00017D8B0F57C7F00F0D1870AD8B0F57A7FD4
:1025B00000F0048440F2EF33984200F0BC8701F051
:1025C000A2BB40F20343984201F0448040F207432B
:1025D000B4E3B34B984200F0F7830CD840F2364393
:1025E000984201F0278340F2D773984241F08B83E1
:1025F000022000F0A8BFAB4B984200F0E88703F53B
:10260000540303F2EF13984201F01483A64B98424F
:1026100041F079830122D8E3A44B984200F09B87D4
:1026200019D8A34B984200F0878609D8A14B98424D
:1026300000F0AD87A04B984200F0428501F063BBEB
:102640009E4B984201F092829D4B984241F05B83F1
:102650009C4801F05CBB9C4B984200F011852FD840
:102660009A4B984201F0D582994B984241F04B83A6
:102670000021984806F082F9804689469548002155
:1026800006F094F900210446924806F08FF90021E3
:102690000546904806F08AF90646284612F026FBC1
:1026A0000546204612F022FB49460446404612F0F9
:1026B000CBF933462A46214608F0B8FC01F029BB85
:1026C000854B984200F0F483844B984201F02183BB
:1026D000834BAAE2834B984200F0B78600F28980D0
:1026E000814B984200F041875BD803F17643A3F514
:1026F0003C23A3F52373984200F0018646D8A3F14A
:10270000A163A3F5E723A3F55E73984201F0C782A6
:1027100003F1507303F5CA3303F25113984241F0A9
:10272000F282724D0FCD07AC0FC42B687048236046
:10273000002106F023F912F0CFF9002182466C48FF
:1027400006F01CF912F0C8F900218146684806F02D
:1027500015F912F0C1F900218046654806F00EF91E
:1027600012F0BAF900210746614806F007F912F0A5
:10277000B3F9002106465E4806F000F912F0ACF904
:10278000002505900DF11C0B01F07EB8594B9842C5
:1027900000F0208403F1D47303F5B73303F5ED7330
:1027A000A9E1554B984200F0BF830BD8534B984298
:1027B00000F0DE86524B984241F0A58206F014FCF0
:1027C00001F0A7BA4F4B984201F0AB8003F55903D3
:1027D00003F6C653984201F08882A3F15E73A3F515
:1027E0001B336FF4F5721344984241F08C8200F071
:1027F000ADBE454B984200F0838435D8434B984298
:1028000000F000830ED8424B984201F0FF8103F1A3
:10281000BC7303F5873303F5FC73984200F02D85F4
:1028200001F071BA3B4B984200F0908703F10573B9
:1028300003F5BE3303F5E173984200F02683A3F15C
:102840000463A3F54E236E3B984241F05C82002165
:10285000274806F093F812F0F7F8C4B2002120469A
:102860000DF0FEFA01F0C1B92B4B984200F0CF8277
:1028700056D8A3F11763A3F57823A3F69D039842D6
:1028800000F03883254B984241F03D82012400F04E
:10289000F1BE00BF94935D73D28D362450662C0533
:1028A0002A671E00C616860034321F009620250DAA
:1028B000D4813D08B43C850570B5A60672C0DC091C
:1028C00057B9A70BBC97010003AF32150973320D3E
:1028D00051DE830E40A0010020439620DEFD7123CF
:1028E000109A841677AA61477098C033E099010066
:1028F00042A00100E0CC872D0063263693E1163517
:1029000040FED93577BE37419AEC14651260955276
:102910007688FE50D294815C60F9E0709223076E55
:10292000D64B984200F03C8303F5FD0303F580434A
:102930004A33984201F0818103F17F4303F5082374
:1029400003F64C63984241F0DE810021CC4806F04A
:102950002DF800210546CA4806F028F80021074650
:10296000C74806F023F800210646C54806F01EF8C1
:10297000012482460090029401943B463246294647
:10298000204607F0CDFC00F04BBEBE4B984200F055
:10299000868500F2FA80BC4B984201F0108100F26B
:1029A0008680BA4B984200F0B78546D803F16A4357
:1029B000A3F51A23A3F66C43984200F01E8219D89F
:1029C000A3F18E63A3F58833393B984200F0DA8493
:1029D00003F1417303F5B5430E33984241F09381FF
:1029E0000021AB4805F0CAFF12F056F8C1B2022030
:1029F00000F0EABDA74B984201F09A8003F14573BD
:102A000003F5AB332A33984241F07D810021A04881
:102A100005F0B4FF12F018F80A28A8BF0A2020EA2F
:102A2000E07400219A4805F0A9FFA5B212F054F80D
:102A30002946FDF7DDFE00F03FBD974B984200F0C0
:102A40007A8512D8A3F1CE63A3F5B8333B3B984205
:102A500000F0028603F54E1303F66173984241F0CD
:102A6000528108F025F901F054B98C4B984200F0DE
:102A70009D858B4B984200F06B858A4B984241F0C4
:102A800042810021824805F079FF06460F468048C2
:102A9000002105F073FF11F0FFFF3946C4B2304644
:102AA00011F0FAFF214608F0A1F800F025BC7E4B9A
:102AB000984200F0488423D803F17C4303F56E0369
:102AC00003F66653984200F084810AD8A3F1237379
:102AD000A3F54F33A3F5F273984200F03785734B9B
:102AE0006CE0734B984200F0838403F1877303F525
:102AF000F83303F586739C4200F05B8501F003B95F
:102B00006C4B984200F0D98310D86B4B984201F07F
:102B1000D08003F1C67303F5E0336D33984241F082
:102B2000F2800020FFF7F4F901F0F3B8634B98420C
:102B300000F03C87624B984200F0BE87A3F1DA7345
:102B4000A3F67863984241F0DE805E4805F0F8FD18
:102B500040F6B830FEF726FC11F076FF05F066FE71
:102B6000594805F0EDFD4FF43C60FEF71BFC11F0F9
:102B70006BFF05F05BFE544805F0E2FD40F6C830FF
:102B8000FEF710FC11F060FFC7E1504B984201F0D6
:102B9000A28000F2B1804E4B984200F0BA8223D856
:102BA0004C4B984200F056810DD84B4B984200F0A8
:102BB000BF8403F5350303F5E14306339C4200F07F
:102BC000EA8201F0A0B8454B984200F0318303F14E
:102BD0009D7303F5823303F5EC73984241F09380C3
:102BE00007F070FF01F095B83D4B984200F07484F7
:102BF00009D83C4B984201F06B803B4B984200F067
:102C0000278601F080B8394B984200F0038503F124
:102C1000CD7303F5CD331A33984200F07583A3F1D9
:102C20005F73A3F50833A3F597739C4241F06B8063
:102C30000BF0A6FD04460BF099FD05460BF08CFD4C
:102C400006460BF06BFD07460BF072FD80460BF05D
:102C500079FD81460BF01CFD334603902A46214640
:102C600023488DE8800305F0A5FD0BF011FD214BF5
:102C7000034442F2107093FBF0F037E12E971D727F
:102C800040A00100F8745ABDC074D6A49107E68F25
:102C900042A00100EE4D4A8158464F99705B8B9ED1
:102CA0005E3A62A1BC7A839CB01A60AB9E4CF3A6DC
:102CB00097E4C7A8B879ECB90357F5B50A7E05BB08
:102CC000EE443FBC5AA0010097A2010019F107DAB7
:102CD0006EB53ECE20E874C298A898C12A5AE8C8BA
:102CE0000625C1D36FFD9AD2D23F64D384AE3BD7C1
:102CF000F7A00100003665C4C94B984200F0AA84D1
:102D000023D8C84B984200F0E9800ED8C64B9842B1
:102D100000F0A38303F1886303F5832303F51E7397
:102D2000984200F05E8200F0EEBFC04B984200F087
:102D30006386BF4B984200F0BB84BE4B9C4240F080
:102D4000E2870025BC4F00F0FFBCBC4B984200F06E
:102D5000D18611D8BA4B984200F0FC80B94B98420A
:102D600040F0D1870021B84805F008FE11F06CFE54
:102D700008F0DCF900F0CDBFB44B984200F0B68308
:102D8000B34B984200F0E382B24B984240F0BB87CD
:102D90000021AD4805F0F2FD04460D46AE4805F0B1
:102DA000CFFC2946204611F077FEFEF7FBFA11F022
:102DB00093FE062105F022FDA848B1E0A84805F0E1
:102DC000BFFCA84800F0A3BF0022A74B1A7000F078
:102DD000A0BF0021A54805F0E9FDA54B1B6893F8AD
:102DE0009C20904218BFC0B2934A18BF83F89C0041
:102DF0001378DB07FCD500F08CBF9D4B1B6893F864
:102E00009C0073E00120FDF771FC00F082BF0021FF
:102E10009648894E05F0CAFD0024054600219348D6
:102E200005F0C4FD924A6B1E1268C3EBC303234432
:102E300002EB430380B2B3F8AC2192B2904218BFC8
:102E4000A3F8AC013378DF07FCD50134072CE5D1BA
:102E500000F05FBF0021854805F0A8FD0021044671
:102E6000824805F0A3FD824B1B6803EB440380B24C
:102E7000B3F84E2392B290426F4A18BFA3F84E03A4
:102E80001378DC07FCD500F044BF4FF47A716E482C
:102E900005F08CFD0121044628200CF0E1FF0C20F8
:102EA0000CF0A2FF214628200DF084F800F031BF7D
:102EB0000021654805F062FD06460F466248002184
:102EC00005F05CFD11F0E8FD3946C4B2304611F062
:102ED000E3FD214607F03AFE00F01BBF00215A48EF
:102EE00005F04CFD11F0D8FD07F04CFE05F09EFCFE
:102EF00000F00FBF0021544805F040FD11F0CCFD5B
:102F000004465C4805F01CFC204605F09FFC534835
:102F100005F016FC204607F085FE05F087FC5648B4
:102F200005F00EFC00F0F5BE0021474805F026FD37
:102F300006460F464448002105F020FD04460520C2
:102F40000D460DF02BF93046394611F0A5FD22460D
:102F50002B4621E00BF000FC06460BF007FC054673
:102F60000BF00EFC0446304611F058FA02460B46B0
:102F700040F6B830FEF748FA284611F04FFA0246FC
:102F80000B464FF43C60FEF73FFA204611F046FA3C
:102F900002460B4640F6C830FEF736FA00F0B9BEDE
:102FA0000021294805F0EAFC11F076FD3B2840F2AB
:102FB000B0864FF47A7358432D4B1B68D3F8982191
:102FC00090421D4A18BFC3F898011378D807FCD562
:102FD00000F09FBE00211C4805F0D0FC11F07CFDE4
:102FE0002649044612F092F8002800F092864FF02D
:102FF0008041204612F06CF8002800F08A861C4BB5
:103000001D682046D5F8981012F058F808B9C5F890
:103010009840094A1378D907FCD500F07ABE00BF62
:1030200090D721F12813DDE3368F4CDAE2D606EC97
:103030009DCD5DEE46B2C0E901000240EE2015F7DD
:103040006A493DF3F8D9E3F542A00100F2D392FDBD
:10305000200902FF68F32FF851A0010097A2010098
:10306000579B010039A001001C99FF1F40A00100DF
:10307000BC8CFF1F49A0010077A60100CDCC4C3EBF
:103080000021B64805F07AFCB54B1C68064694F85A
:103090002C000F4611F0C2F902460B463046394665
:1030A00011F08AFC30B93046394611F0F5FCC0B257
:1030B00084F82C00AB4A1378DB07FCD500F029BE5E
:1030C0000021A64805F05AFC11F006FD0021044637
:1030D00012F012F8002800F01C86204612F05CF86E
:1030E0009F4B1A68B2F830339BB298421CBF80B233
:1030F000A2F830039B4A1378DF07FCD500F009BE25
:103100000021964805F03AFC11F0C6FCC1B200203F
:103110005AE200219148924D05F030FC2C68064699
:10312000B4F8680180B20F4611F078F902460B46F8
:103130003046394611F040FC30B93046394611F07E
:10314000ABFC80B2A4F86801864A1378DFF81482D9
:1031500013F0010FF9D00021804805F00FFC2C6816
:103160000646B4F86A0180B20F4611F057F90246DC
:103170000B463046394611F01FFC30B9304639460F
:1031800011F08AFC80B2A4F86A0198F80030DE07DA
:10319000FBD500F0BEBD744B1B7813B1734805F02E
:1031A00069FB00216D4805F0E9FB01210020FEF7D5
:1031B00009FD11F0F1FF6A4B1A68B2F8683180B26C
:1031C0009BB2984218BFA2F86801664A1378DD07DF
:1031D000FCD507F0B1F96648FDF74CFF844200F0DA
:1031E0009885614B1B7813B1624805F043FB0021C1
:1031F0005A4805F0C3FB01210020FEF7E3FC584BC1
:103200001C680546B4F86A0180B211F06FFD0146F2
:10321000284611F053FF28B9284611F0BDFF80B2AF
:10322000A4F86A014F4A1378DC07FCD500F041BCD2
:1032300000214A484B4E05F0A1FB11F005FC00248B
:1032400005460021454805F099FB11F0FDFB444A75
:10325000126804EBC50302EB430300B2B3F840224B
:1032600012B2904218BFA3F840023378D807FCD5B9
:103270000134082CE5D100F04CBD0021374805F0A1
:103280007DFB374B1C68064694F86C010F4611F025
:10329000C5F802460B463046394611F08DFB30B971
:1032A0003046394611F0F8FBC0B284F86C012D4A63
:1032B0001378D907FCD500F02CBD0021274805F074
:1032C0005DFB11F0C1FB00210546244805F056FBCB
:1032D00011F0BAFB06466421204805F067FB314631
:1032E0000446284607F060FF052105F087FA2248CA
:1032F00005F0C0FA0134EED1204800F008BD1420DA
:1033000007F06EFF00F005BD6421144805F04EFB88
:10331000012104462520FEF7BFFC032105F06EFACB
:10332000174805F0A7FA252005F080FA144805F0A3
:10333000A1FA0134E8D1DFE701210846FEF742FC9B
:10334000032100F0DDBCFDF7A1FE00F0E2BC01218D
:103350000846FDF725FF00F0DCBC00BF42A00100DD
:10336000BC8CFF1F010002401C99FF1F6FA00100D1
:1033700094A001009BA0010097A2010044A00100BD
:1033800065A101000021BF48DFF808A305F0F6FAA7
:1033900011F082FB81464FF47A71BA48BA4F05F0BA
:1033A00005FB00248046012649462046FDF76CF8BF
:1033B000FDF78CF814F80A5057F835300A2083F8D6
:1033C00080600CF0EBFE57F83530204683F8006142
:1033D00000210134FDF758F8FDF778F80B2CE3D104
:1033E000AA4805F047FAB8F1FF3FD4D100F091BCEC
:1033F0000021A44805F0C2FA06460F46A148002164
:1034000005F0BCFA804689469E48002105F0B6FAD0
:1034100004460D469B48002105F0B0FA11F014FB5C
:1034200029460FFA80FA204611F00EFB494605B2F4
:10343000404611F009FB394604B2304611F004FB56
:1034400053462A46214600B203E000231A46194695
:10345000184606F018FD00F05CBC0021894805F014
:103460008DFA11F0F1FAC4B2012120460CF0F8FCFB
:10347000012120460CF0C6FCC8200CF08FFE002174
:1034800020460CF0BFFCC8200CF088FE64217D486B
:1034900005F08CFA0130EBD17D4800F038BC0021FA
:1034A000784805F06BFA11F0CFFA00210446754810
:1034B00005F064FA11F0C8FA01462046FCF7E4FF73
:1034C000FDF704F8734B1A5D6F4B53F8323001224D
:1034D00083F8802000F01DBC00216F4805F066FADB
:1034E00011F004FC07F0F2FE00F013BC00216A4862
:1034F00005F044FA06460F466748002105F056FAE3
:1035000011F0F4FB39460446304611F09DFA0022D2
:10351000214607F07DFCFCE34FF47A71594805F031
:1035200045FA0446012007F04FFB0134F4D1F0E3E3
:10353000FDF7F2FEEDE3594B1B6893F89C300A2B24
:103540000CBF03200020FEF797FFE2E30120FAE71B
:1035500006F014F8DDE300214A4805F00FFA11F0F7
:103560009BFAC0B207F084FBD3E307F0C7FBD0E3BC
:103570004B4D00244FF47A71424805F0FFF911F0E9
:10358000ABFA45F8240001340A2CF3D1C1E3454DD0
:1035900000244FF47A713B4805F0F0F911F09CFAE1
:1035A00045F824000134062CF3D1B2E307F0CAFB3E
:1035B000AFE30021334805F0E1F911F06DFA01287D
:1035C00028BF0120C1B2012006F09CFFA1E3002129
:1035D0002C4805F0D3F906460F462A48002105F08D
:1035E000CDF9314B0446186807901B798DF82030CF
:1035F000204611F051FAC0B2041C3946304618BFBB
:10360000012411F049FA20AB53FA80F0214610F85A
:10361000640CD9E7254805F093F807F0B7FB65E49B
:103620000121184805F0AAF93B46324680468946F2
:103630000120294602940194CDF800A006F070FE06
:1036400064200CF0ABFD4046494611F0FDF9013015
:10365000E6D15EE30DF03AFA00210F4805F0A6F935
:10366000002104460C4805F0A1F90146204607F068
:1036700029FE4EE320460021013407F023FE062CEC
:10368000F8D146E342A0010038B0010065A1010075
:10369000C2A00100189A010040A00100BC8CFF1FCD
:1036A0000498FF1FB497FF1FD8990100C4A0010020
:1036B0000021BA4805F07AF900210446B74805F020
:1036C00075F906464FF47A71B54805F06FF9013483
:1036D000314605462046FCF7C9FEFCF7F7FE0120FF
:1036E0000CF05CFD00212046FCF7C0FEFCF7EEFE6E
:1036F00001200CF053FD0135E4D10AE30021A84874
:1037000005F03CF9A74B04EB44061B682E4403EB81
:1037100086068046B068894610F092FE02460B4647
:103720004046494611F048F920B94046494611F053
:10373000D3F9B0603B78DA07FCD50134032CDDD136
:103740000135032D00F0E5820024D7E700219448DD
:10375000944C05F013F925680646E86D0F4610F005
:103760006FFE02460B463046394611F025F920B966
:103770003046394611F0B0F9E8658B4A13788A4D26
:1037800013F0010FFAD00021854805F0F7F82668FC
:103790008046306E894610F053FE02460B46404686
:1037A000494611F009F920B94046494611F094F90B
:1037B00030662B78DB07FCD50021794805F0DEF870
:1037C00026688046706E894610F03AFE02460B4627
:1037D0004046494611F0F0F820B94046494611F0FC
:1037E0007BF970662B78DF07FCD500216C4805F06B
:1037F000C5F826688046B06E894610F021FE024664
:103800000B464046494611F0D7F820B94046494694
:1038100011F062F9B0662B78DE07FCD50021604814
:1038200005F0ACF824680646A06D0F4610F008FEBF
:1038300002460B463046394611F0BEF820B93046F4
:10384000394611F049F9A0652B78DC07FCD560E218
:103850000021534805F092F8524B1C680646A06DB3
:103860000F4610F0EDFD02460B463046394611F08A
:10387000A3F820B93046394611F02EF9A0654A4A1E
:103880001378D807FCD544E2504610F0D9FD5BF818
:10389000254002460B462046FDF7B6FD03200CF0FE
:1038A0007DFC484610F0CCFD02460B4604F10800B2
:1038B000FDF7AAFD03200CF071FC404610F0C0FD9E
:1038C00002460B4604F11000FDF79EFD03200CF0AC
:1038D00065FC384610F0B4FD02460B4604F11800B2
:1038E000FDF792FD03200CF059FC304610F0A8FDC6
:1038F00002460B4604F12800FDF786FD03200CF07C
:103900004DFC059810F09CFD02460B4604F120008A
:10391000FDF77AFD013503200CF040FC052DB3D1F5
:10392000F7E100211E481F4D05F028F82C680646D7
:10393000D4F8A8010F4610F083FD02460B4630462E
:10394000394611F039F828B93046394611F0C4F833
:10395000C4F8A801144A1378DFF84C8013F0010F63
:10396000F9D000210E4805F009F82C680646D4F875
:10397000A4010F4610F064FD02460B46304639465E
:1039800011F01AF828B93046394611F0A5F8C4F8F4
:10399000A40198F80030D907FBD5BAE140A0010096
:1039A00042A00100BC8CFF1F01000240DFF8108321
:1039B00000240021C04804F0E1FFC04B1D6805EB66
:1039C00084050646D5F834030F4610F027FD02465D
:1039D0000B463046394610F0EFFF28B930463946DD
:1039E00011F032F8C5F8340398F80030DA07FBD547
:1039F0000134072CDDD18CE10021AF48AF4D04F03C
:103A0000BDFF2C680646D4F88C000F4610F018FD58
:103A100002460B463046394610F0CEFF28B93046F4
:103A2000394611F059F8C4F88C00A54A1378A44E11
:103A300013F0010FFAD000219F4804F09FFF2C687B
:103A40008046D4F89000894610F0FAFC02460B46F6
:103A50004046494610F0B0FF28B94046494611F0AB
:103A60003BF8C4F890003378DB07FCD5002192487E
:103A700004F084FF2C688046D4F89400894610F046
:103A8000DFFC02460B464046494610F095FF28B938
:103A90004046494611F020F8C4F894003378DF0717
:103AA000FCD50021844804F069FF0021824804F01D
:103AB00065FF06F041FD2CE100217F4804F05EFF28
:103AC0007E4B1C680646D4F8A0010F4610F0B8FCE7
:103AD00002460B463046394610F06EFF28B9304694
:103AE000394610F0F9FFC4F8A001754A1378DD07D4
:103AF000FCD50EE10021704804F040FF6F4B1C68BC
:103B00000646D4F838020F4610F09AFC02460B46DF
:103B10003046394610F050FF28B93046394610F08B
:103B2000DBFFC4F83802664A1378DC07FCD5F0E006
:103B30000021614804F022FF604B1C680646D4F85F
:103B40003C020F4610F07CFC02460B4630463946DC
:103B500010F032FF28B93046394610F0BDFFC4F8E6
:103B60003C02574A1378D807FCD5D2E000215248CE
:103B700004F004FF10F090FF431E032B044600F2F4
:103B8000C88000214C4804F0F9FE4C4B1B6803EB45
:103B900084040646A06F0F4610F052FC02460B4606
:103BA0003046394610F008FF20B93046394610F04B
:103BB00093FFA067424A1378D907FCD5A9E03F4B91
:103BC000DFF8FC801E680024002706EB8405002136
:103BD000E86F11F073FA00B9EF6798F80030DB076F
:103BE000FBD50134042CF0D193E04FF47A713248C4
:103BF00004F0DCFE054620460CF024F904F044FEF7
:103C0000C8200CF0CBFA0135EFD182E009F0B0F812
:103C10007FE04FF47A71284804F0C8FE0122044680
:103C200011461046FDF770FD264804F023FE0134CE
:103C3000EFD16EE0FDF76AF86BE0234804F01AFE5E
:103C400000211D4804F0B2FE002104461A4804F089
:103C5000ADFE00210546184804F0A8FE00210646E6
:103C6000154804F0A3FE00210746134804F09EFE09
:103C700000218046104804F099FE3B463246294612
:103C80000190CDF8008020460AF082FD0AF000FD88
:103C90000CF09AF84FF4FA600CF080FA39E00B4817
:103CA00004F04EFD012005F059F904F0BFFD054870
:103CB0002DE005F093FB2CE042A00100BC8CFF1F1F
:103CC0000100024065A10100D3A0010049A101004B
:103CD00005F046FB1DE0104A1049114804F06AFD4A
:103CE00017E00120FDF7FEF913E00E4963234FF4BE
:103CF0007A7207A804F0FCFD07A8FCF777FF002103
:103D000004F07CFD05E0084804F01AFD284604F0A4
:103D1000B1FD21B0BDE8F08FF19B0100E59B0100F2
:103D200052A1010063A1010066A101002DE9F04F3D
:103D300089B006AB83E80300079B002B66D0DF68E1
:103D4000002F63DD334804F0FBFC0026B5B2AF4220
:103D500059DD294606A808F0EAF8DFF8CC80DFF83C
:103D6000CCA0D8F80010840021448146D1F8A030BE
:103D700002930023D1F8C820CAF80030D1F8F0B07F
:103D8000D1F81801039211F0E1F9039A0590104659
:103D900011F0DCF90490584611F0D8F94FF0010BFE
:103DA00003900298CDF804B011F0D0F903A9009067
:103DB0000EC95846FDF7F0FBDAF800A0164804F0EB
:103DC000BFFC484604F032FD04F07CFD0321504660
:103DD00004F014FD5D44114804F0B2FCAF4201DD73
:103DE00004F070FDD8F800301C445046D4F870112F
:103DF00011F064F908B9C4F870A1094B1B78DB070E
:103E0000FBD50136A2E7074804F09AFC09B0BDE8EB
:103E1000F08F00BF73A1010080A101007CB70100F9
:103E20000100024077A60100BC8CFF1F4497FF1FD2
:103E30002DE9F04F8BB000270890642003910CF01F
:103E4000ADF99A4804F07CFC00260497089BDFF843
:103E500074A233F91650DAF80030DFF8789203EBE9
:103E60008505D5F8A030D5F8C8B0D5F84081D5F88B
:103E7000F000099311F06AF90446D5F8180111F021
:103E800065F90023C9F800300590584611F05EF935
:103E9000099B06904FF0010B1846D5F87051CDF8EC
:103EA00004B011F053F921460090059B069A58463C
:103EB000FDF772FB7E490398D9F800900DF006FFDC
:103EC00030B1022C06BFDAF80030D3F838520025A2
:103ED0002946404610F054FE0021834611F016F9A1
:103EE000F0B12946484610F04BFE0021824611F001
:103EF0000DF9A8B1584610F0A3FA0EF033FBCDE946
:103F00000601504610F09CFA0EF02CFB02460B46C0
:103F1000DDE9060110F034F910F0DEFD824601E023
:103F2000DFF8B4A1624903980DF0D0FE38B1022C3D
:103F300003D0062C03D1574601E0CDF810A05D4810
:103F400004F0FEFB4946484611F0EAF820B14FF074
:103F5000FF3004F06BFC03E00221484604F04EFC05
:103F600004F0B0FC4146404611F0DAF820B14FF0C1
:103F7000FF3004F05BFC03E00221404604F03EFC0D
:103F800004F0A0FC2946284611F0CAF820B14FF0F1
:103F9000FF3004F04BFC03E00221284604F02EFC25
:103FA00004F090FC5146504611F0BAF820B14FF0A1
:103FB000FF3004F03BFC03E00621504604F01EFCF9
:103FC00004F080FC204604F031FC04F07BFC0598F2
:103FD00004F02CFC013C04F075FC374B53F8240032
:103FE00004F024FC354804F0ABFB0EB904F06AFC85
:103FF0000136022E7FF42AAF314804F0A1FB2C4990
:1040000003980DF063FE00284DD02E4C04982368D1
:10401000D3F8A061D3F83C52394610F0B1FD3146D7
:1040200010F0B8FE294610F0ADFD0546264804F014
:1040300087FB0321284604F0E1FB244804F080FBC1
:104040002368D3F8A0512946284611F069F800B139
:104050001F4D0321284604F0D1FB1C4804F070FBDF
:104060002368D3F838522946284611F059F800B190
:10407000174D0321284604F0C1FB144804F060FBEF
:104080002368D3F83C422146204611F049F800B19C
:104090000F4C2046032104F0B1FB09480BB0BDE8EA
:1040A000F04F04F04DBB0BB0BDE8F08F82A10100D2
:1040B00091A1010080A10100A4A901007CB7010029
:1040C00077A60100BC8CFF1F96A1010097A20100FA
:1040D000000080BF4497FF1F003C1CC624200BF04B
:1040E000ABBBFFFF38B5434B00241C60424B1C6048
:1040F000424B1C60424B1C60424B1C60424B1C609C
:10410000424B1C60424B1C60424B1C60424B1C608B
:10411000424B1C60424B1C60424B1C60424B0025D2
:104120001D60424B1C60424B1C60424B1C60424B6A
:104130001C60424B1D60424B1D60424B1D60424B58
:104140001C60424B1C60424B1C60424B0020002113
:10415000C3E90001404B414941481C600DF099FD05
:10416000404B414A1C60414B14601C60404B414A2B
:104170001C60414B14601C60404B1D60404B1D6037
:10418000404B1D60404B1C60404B1C60404B1C6012
:10419000404B1C60404B1C60404B1C60404B1C6003
:1041A000404B1C60404B1C60404B1C60404B1C60F3
:1041B000404B1C60404B1C60404B1C60404B1C60E3
:1041C000404B1C605C609C603F4B1C603F4B1C6024
:1041D0003F4B1C603F4B1C603F4B1C603F4B1C60C7
:1041E0003F4B1C603F4B1C603F4B1C605C609C6005
:1041F00038BD00BF3096FF1F3C99FF1F5096FF1F30
:104200007497FF1F4096FF1F3099FF1F3896FF1FBE
:104210004899FF1F2C96FF1F5C97FF1F0C99FF1FEB
:104220008C97FF1F2C99FF1F3498FF1F5896FF1F74
:104230001899FF1F9097FF1F0897FF1F7899FF1F7E
:104240000C97FF1F8499FF1F8497FF1F0899FF1F7A
:104250000499FF1FE897FF1F5496FF1F4D9A010016
:104260006099FF1FA497FF1F2099FF1FEC96FF1F67
:104270003496FF1F2499FF1F0497FF1F5897FF1FB5
:104280002496FF1F4499FF1FFC97FF1F6C97FF1F89
:104290000098FF1FA897FF1F2896FF1F5899FF1F20
:1042A000F896FF1F9497FF1F3499FF1FF097FF1F89
:1042B0003C96FF1FFC96FF1F7C97FF1F3899FF1F3E
:1042C0001897FF1F4497FF1F2899FF1FA097FF1FF4
:1042D0009C97FF1F6097FF1F8099FF1FDC97FF1FB0
:1042E0000097FF1FAC97FF1F4496FF1F2DE9F04377
:1042F0000F4685B000219946054690460DF0F8FC22
:104300000378303B092B40F29F80002128460DF0B6
:10431000EFFC03782D2B00F09780002128460DF04C
:10432000E7FC0378402B6AD1012128460DF0E0FC20
:104330000378732B6C460FD10222294668460DF094
:1043400005FD68460DF009FD064668460DF0CCFBFC
:10435000404A33B2157815E0012128460DF0C8FC1B
:104360000378702B15D10222294668460DF0EEFC29
:1043700068460DF0F2FC064668460DF0B5FB354A7E
:10438000957833B239F9132095FBF2F302FB1355FC
:1043900021E0012128460DF0ABFC03786E2B18D1EB
:1043A0002946022268460DF0D1FC68460DF0D5FC86
:1043B000064668460DF098FB2946042268460DF033
:1043C000C5FC68460DF0C9FC054668460DF08CFB3F
:1043D00001E00026354638F916302B440C2505FB44
:1043E000037595E8070084E80700009B0BB9019866
:1043F0002DE0012B01D1019821E001A81DE0002151
:1044000028460DF075FC0378232B15D10121284691
:104410000DF06EFC03786C2B14D1022229466846FD
:104420000DF094FC68460DF098FC044668460DF0CB
:104430005BFB39F914000AE02868FCF7D7FB10F0A1
:1044400085FE04E0002002E0286811F0B4F805B011
:10445000BDE8F0835097FF1F2DE9F04F91B008ACF5
:1044600084E803000393099B0692002B00F0478227
:10447000DB68002B40F34382934B00221A60069BBB
:104480000BB1924800E09248924F04F059F9002392
:104490000593BDF814300293099B002B00F02C8289
:1044A000DB68029A9A4280F2278208A90AA807F0DC
:1044B00018FD00210AA807F044FD01460CA80DF0E4
:1044C00053FB1A9A03991B9B834D844C7E4E0CA878
:1044D000FFF70CFF824B18600CA80DF005FB029A49
:1044E00008A90AA807F0FDFC01210AA807F029FD88
:1044F00001460CA80DF038FB1B9B1A9A03990CA8D7
:10450000FFF7F4FE28600CA80DF0EEFA029A08A955
:104510000AA807F0E6FC02210AA807F012FD0146EE
:104520000CA80DF021FB1B9B1A9A03990CA8FFF70E
:10453000DDFE20600CA80DF0D7FA029A08A90AA89F
:1045400007F0CFFC03210AA807F0FBFC01460CA8EA
:104550000DF00AFB1B9B1A9A03990CA8FFF7C6FEE5
:1045600030600CA80DF0C0FA029A08A90AA807F05A
:10457000B8FC04210AA807F0E4FC01460CA80DF0E1
:10458000F3FA1A9A03991B9B0CA8FFF7AFFE10F0E1
:10459000ADFB544B18600CA80DF0A6FA0120019059
:1045A00033680093236829680022FCF7F5FF0A208E
:1045B0000BF0F4FD4FF03C084FF07E59B246AB468D
:1045C00003200BF0EBFD4946384610F0E3FB4FF0BB
:1045D00080410446484610F0D5FA0146204610F0C6
:1045E00081FD20B12046404910F0CCFA04463F49F5
:1045F000204610F08BFD18BBDFF8F8900023C9F8B7
:10460000003004F1004010F0A1FD4FF0010ECDF894
:1046100004E0DAF800300093304BDBF800101B6840
:1046200002467046FCF7B8FF2E4BD9F80000196817
:1046300010F06CFD28B9B8F1010802D0A146BFE71F
:104640002A4C3946204610F059FC052780460320A5
:104650000BF0A4FD2649274C404610F09BFB00239D
:1046600000F1004923608046484610F06FFD4FF08E
:10467000010ECDF804E0DAF800300093174BDBF8B8
:1046800000101B6802467046FCF786FF154B206839
:10469000196810F03BFDA0B11549484610F02EFCFA
:1046A00010F054FD002382460120236001903368FE
:1046B00000930A4B29681B685246FCF76DFF0B25D7
:1046C00053E0013FC3D1E7E7F496FF1F9FA101002C
:1046D000AEA101000000A03F6897FF1F1099FF1FC7
:1046E0007097FF1F6497FF1F0000404000F07F4558
:1046F000C3F5883F4497FF1F01240023DFF8189279
:10470000CBF800300194D9F800300093DFF8108224
:104710007C4BD8F800101B687B4F52462046FCF7B4
:104720003BFF20460BF03AFD013EE5D100233B6004
:104730000194D9F800300093724BD8F800101B6830
:1047400020465246FCF728FF7049386810F0DEFC1E
:1047500088B1504610F0CAFA6D4910F01BFB10F0FA
:10476000F5FC82460A200BF019FD013D03D0052619
:10477000DFF894B1C0E7DFF8C491664BD9F80020A8
:10478000654D43F822A065492B6841F82230012489
:104790008DE818005B4E624F33683968DFF8688136
:1047A00000222046FCF7F8FE0A200BF0F7FC00235D
:1047B000C8F8003001942B6800933368396852467A
:1047C0002046FCF7E9FED8F800300493069B2BBB8B
:1047D000544803F0B5FFD9F8000004F027F804F0BE
:1047E00071F8386804F022F804F06CF8306804F0CE
:1047F0001DF804F067F8286804F018F804F062F86F
:10480000504604F013F804F05DF80021049803F01A
:10481000F5FF099B002B62D0DB6860E0424BD9F8C2
:1048200000401B68386803EB840410F05FFAD4F88A
:10483000F0B080460146584610F040FC08B9C4F874
:10484000F0803A4A1378DFF8E48013F0010FF9D0D2
:10485000D4F818313068079310F048FA079B834664
:104860000146184610F02AFC08B9C4F818B198F8A7
:104870000030D807FBD5D4F8A0302868079310F093
:1048800035FA079B83460146184610F017FC08B915
:10489000C4F8A0B098F80030D907FBD5D4F8C830D8
:1048A0000793504610F022FA079B834601461846AC
:1048B00010F004FC08B9C4F8C8B098F80030DA0762
:1048C000FBD5D4F84011049810F0F8FB10B9049B04
:1048D000C4F8403198F80030DB07FBD578E7029A3E
:1048E000134F013B9A42B4BF1248134803F028FF0C
:1048F000059B01330593CCE50E4803F021FF11B071
:10490000BDE8F08F1099FF1F4497FF1F00606A47B2
:104910006666663F1C97FF1FF496FF1FC496FF1F35
:104920006897FF1F80A10100BC8CFF1F010002409F
:10493000C3F5883F77A601007CB701007097FF1F81
:104940002DE9F0478CB00D4607464A49DDF850A0E6
:1049500004A8994690460DF007F9002128460DF06D
:10496000C7F90378402B7AD1012128460DF0C0F910
:104970000378732B0FD10222294608A80DF0E6F91F
:1049800008A80DF0EAF9064608A80DF0ADF83A4A75
:1049900033B2147815E0012128460DF0A9F9037807
:1049A000702B15D10222294608A80DF0CFF908A8CE
:1049B0000DF0D3F9064608A80DF096F82E4A947823
:1049C00033B23AF9132094FBF2F302FB134421E0D3
:1049D000012128460DF08CF903786E2B18D1294659
:1049E000022208A80DF0B2F908A80DF0B6F90646A3
:1049F00008A80DF079F80422294608A80DF0A6F9B8
:104A000008A80DF0AAF9044608A80DF06DF801E019
:104A10000026344639F9163023440C2404FB038461
:104A200094E8070001AB83E8070028B90A2202993D
:104A300008A80DF0D1F806E001280CD10222029955
:104A400008A80DF02FF908A904A80DF01AF908A874
:104A50000DF04AF803E002A904A80DF01AF904A920
:104A600038460DF031F804A80DF03EF838460CB089
:104A7000BDE8F08765A101005097FF1F036810B5DE
:104A8000044623B94068BDE8104003F0CFBE012BB7
:104A900005D103214068BDE8104003F0AFBE0548D2
:104AA00003F04EFE201D03F04BFE0248BDE810400F
:104AB00003F046BEF7AA010030B585B004460D46A6
:104AC00001A807F06FFE40F2DC532246294601A8F8
:104AD00007F03CFD00280CBF2046002005B030BD8B
:104AE0002DE9F04FB74BB84EADF5C24D9BB001224A
:104AF0001A70B64B00251D60B54B02AF1A68C7F897
:104B0000B020B44AD7F8B01011601A68C7F8AC20CA
:104B1000D7F8AC10B04A1B68C7F8A83007F1C80432
:104B2000AE4B11606560D7F8A820AD491A6007F553
:104B3000DC70C7F8C050C7F8C450C7F8C8500DF0B3
:104B400013F803F04FFE42F210731A46A54930687D
:104B500003F0CEFEA449306811F013F9C7F88C6059
:104B600050B300F10C0207F542711630AE4612F850
:104B7000013F222B0ED03A2B0CD003F0DF065B2E28
:104B800008D02C2B01D05D2E02D101F805E000E009
:104B90004B5501358242EAD107F5427107F568703D
:104BA0000CF0E2FF07F5687107F5DC700DF069F8AD
:104BB00007F568700CF098FFD7F88C30DFF80882A2
:104BC000186807F1A40104F0E1F808B987485EE32A
:104BD000002004F025F90546FDF780F9284610F07D
:104BE00085F88349834E0FF0CBFF834910F086F997
:104BF000824910F0CFF810F0CFFA814A014681487F
:104C000003F0D8FDD8F800907F49484611F0B9F874
:104C10000546B8B97D4907F5687011F067F807F5E2
:104C20006871484606F0BDF87949356007F542706D
:104C300011F05CF807F54271D8F8000006F0CFF8E3
:104C40003D6601E001233B6601233360D7F88C30D9
:104C50006D491D68284611F094F807F1A401C7F8C2
:104C60009000284604F092F8B8676A4803F068FD9F
:104C7000D7F8903013F8023C2C2B4FF000031AD1D8
:104C8000D7F890107D2201F8013C4F4B01F8022C1F
:104C90001D680135294607F56870FFF70DFF07F518
:104CA000C87602462946304607F055F996E80300D3
:104CB00084E8030002E0C7F8C8306360564803F098
:104CC0003FFDD7F88C305549186811F05AF810B1EB
:104CD000534803F035FD5349204607F072F970B38D
:104CE000504A214607F5427007F072F9D7F80C6375
:104CF00006B1F6684FF000084546B045494A2146DE
:104D000014DA07F51C7007F063F9424607F51C71C9
:104D100007F5427007F0E5F8D7F80C3303B1DB680C
:104D2000002BA8BFED1808F10108E6E707F542706F
:104D300007F04EF9D7F80C631EB1F66801E005469E
:104D400006460C204543731EFB660A35730025F0AA
:104D50000705083323F00703ADEB050D0DF1080B34
:104D6000ADEB030D0DF1080AADEB030D02AB2D49C0
:104D7000C7F89430204607F024F97867002800F03F
:104D80008381284A214607F5427007F021F9D7F8B8
:104D90000C33002B00F07881DB68002B40F374812A
:104DA000214803F0CDFC4FF0FF330025C7F88830D1
:104DB00007F50873C7F880503B67AE4236DC002524
:104DC0005AE100BF1499FF1FE097FF1FD897FF1FFC
:104DD000889DFF1F5C99FF1F4099FF1F7499FF1F5B
:104DE00065A1010063A10100BBA10100C7A10100F1
:104DF00000C05A45E497FF1F00002F440000C8423E
:104E0000D09B0100D6A1010000A201000FA2010069
:104E100060A6010023A2010050A901002EA20100FA
:104E200037A2010099A20100A2A20100CD4A2146A9
:104E300007F51C7007F0CCF82A4607F51C7107F53A
:104E4000427007F04EF8D7F80C3303B1DB68D7F89F
:104E5000942022F81530D7F88830FB674FF00C0803
:104E600008FB03B84FF00009FB6FBE4A4B442146D4
:104E700007F51C70C7F8883007F0AAF82A4607F52E
:104E80001C7107F5427007F02CF8D7F80C3303B10A
:104E9000DB68994580F29880B24A386F214607F066
:104EA00097F82A46396F07F5127007F01AF8494645
:104EB00007F5127007F045F80378303B092B19D934
:104EC000A84A214607F51C7007F082F82A4607F524
:104ED0001C7107F5427007F004F8494607F5427067
:104EE00007F02FF80378A3F12D0EDEF1000343EB5A
:104EF0000E0300E07B6F002B46D09A4A214607F54F
:104F00001C7007F065F82A4607F51C7107F542701A
:104F100006F0E7FF494607F5427007F012F82E2128
:104F200010F0CCFEC8B10123C8F80C308D4A2146E0
:104F300007F51C7007F04CF82A4607F51C7107F5B9
:104F4000427006F0CEFF494607F5427006F0D7FFE3
:104F50000FF0C2FDC8F8100031E0C8F80C00814A1B
:104F6000214607F51C7007F033F82A4607F51C7137
:104F700007F5427006F0B5FF494607F5427006F0A6
:104F8000D6FFC8F810001AE00223C8F80C30754AA2
:104F9000214607F51C7007F01BF82A4607F51C711F
:104FA00007F5427006F09DFF494607F5427006F08E
:104FB000C8FF0822014608F1100010F0BCFE09F1FC
:104FC000010908F10C084FE7B7F880302AF81530CE
:104FD000644A214607F51C7006F0FAFF2A4607F5D9
:104FE0001C7107F5427006F07CFFD7F80C3303B153
:104FF000DB68D7F880201A44C7F880200135DCE64A
:105000003AF915300C20434400FB03B0FFF736FD9E
:10501000544A214607F51C7006F0DAFF2A4607F5C8
:105020001C7107F5427006F05CFFD7F80C3303B132
:10503000DB68013B984502DA4B4803F081FB08F13D
:105040000108484A214607F51C7006F0C1FF2A46B0
:1050500007F51C7107F5427006F043FFD7F80C33D3
:1050600003B1DB689845CBDBFB6E9D42B4BF3F4884
:105070003F4803F065FB0135AE4205DD3D4803F0D6
:105080005FFB4FF00008DCE73B49204606F099FF44
:1050900098B3394A214607F5427006F099FF00217E
:1050A00007F5427006F043FF334A0646214607F5EE
:1050B000427006F08DFF012107F5427006F037FFC0
:1050C00036B205462D4803F03BFB304603F0AEFBFD
:1050D0002DB2254803F034FB284603F0A7FB2248F5
:1050E00003F02EFB3AF9160005440C2000FB05B036
:1050F000FFF7C4FC1D4803F023FB2149204606F0BE
:1051000060FF002842D01E4A214607F5427006F093
:105110005FFF002107F5427006F009FF184A0546B7
:10512000214607F5427006F053FF012107F5427052
:1051300006F0FDFE0FF0DAFD064628460FF0D6FD1C
:1051400010490FF0D9FF20B90E4930460FF0CAFFC1
:10515000E0B10D4803F0F4FA03F0A6FB03F042FBC4
:1051600002F01ABD99A2010097A2010077A60100E2
:105170005B9C010080A10100AFA20100B7A2010069
:10518000C7A20100FDF61540D8A2010076492046CD
:1051900006F017FFF0B17449204606F03BFF0146C8
:1051A00007F542700CF0E0FCD7F8943052465946AF
:1051B00007F54270FFF79AF8786507F542700CF032
:1051C00093FC6A4803F0BCFA786D03F02FFB03F000
:1051D00079FB01E001237B653B6E012B0ED1D7F8F3
:1051E0008C306349186810F0CCFD18B9BB6F03F818
:1051F000020C07E0002300F8023C03E0BA6F002332
:1052000002F8023CD7F890501035294607F568702F
:10521000FFF752FC07F5CC7402462946204606F0FB
:1052200039FE94E8030007F1C00383E80300002877
:1052300002F0BC84002902F0B984D7F8C43003B16D
:10524000DB68FB6603F020FD03F0CCFA2822002186
:1052500007F5FC700AF068F92822002107F50870AC
:105260000AF062F92822002107F512700AF05CF9B1
:10527000404B002201201A7103F05AFE58B13E48FB
:1052800003F05EFA03F010FB03F0ACFA3B4803F0C6
:1052900057FA02F081BC3A4803F052FAD7F8B80145
:1052A00003F04EFA03F01EFB3B6E012B02D1354892
:1052B00003F046FA344B10221A6040221A600A208A
:1052C0000AF06CFF7B6D012BB8BF0123FB67002345
:1052D000C7F88C307B66FB63BB62FB62254B97F89B
:1052E0008C201A700023C7F88830D7F88830FA6EFF
:1052F000934282F22B841F4B97F88820DA7007F1D3
:10530000D0090023C7F8D030C9F8043007F1980459
:1053100007F1E003A3F120012046D7F8882006F02A
:10532000F8FD94E8030089E803001849484606F0B0
:1053300048FE38B91649484606F043FE50BB0123E3
:10534000BB673DE01149484606F05AFE0028BEBF43
:105350007B6DC01801300028ECD0D7F88C300138B4
:10536000834242F0C783E5E7FBA2010007A30100E7
:10537000BBA101005097FF1F16A301002EA301003F
:1053800049A3010059A30100C4F00F4062A301002A
:105390006AA301005949484606F03CFE014607F55C
:1053A00042700CF0E1FBD7F894305246594607F5AD
:1053B0004270FEF79BFFB86707F542700CF094FB54
:1053C0004F49484606F0FDFDA8B14D49484606F054
:1053D00021FE014607F542700CF0C6FBD7F8943069
:1053E0005246594607F54270FEF780FFB86707F549
:1053F00042700CF079FB4349484606F0E2FDB0B13B
:105400004049484606F006FE014607F542700CF09A
:10541000ABFBD7F894305246594607F54270FEF779
:1054200065FF394B186007F542700CF05DFBBB6FF0
:10543000002B08BF0123BB6700233B673A6FBB6F9C
:10544000934242F37E83314B97F870209A702E4B33
:10545000C7F830D01A685AB12D4B2E491B68C7F8CF
:10546000B430D7F8B43009685B1A9A42C2F0A98305
:10547000294A07F1D00107F1D80006F0A9FD274A13
:1054800007F1D00107F1E00006F0A2FD244A07F180
:10549000D00107F1E80006F09BFD224A07F1D00198
:1054A00007F1F00006F094FD1F4A07F1D00107F163
:1054B000F80006F08DFD1D4B1B684BB91C4907F128
:1054C000D00006F0A7FD014607F5DC700CF0E1FB0B
:1054D0001849484606F075FD18B11649484606F0C9
:1054E0008FFD1549484606F06CFD38B31249484611
:1054F00006F086FDC7F8900023E000BF6AA3010014
:1055000074A3010085A30100B097FF1F5097FF1FF0
:10551000889DFF1FF897FF1F94A3010099A3010026
:10552000A0A30100AFA30100B9A30100E497FF1FEE
:10553000BBA10100C0A30100C7A301000123C7F85C
:105540009030B249484606F03CFD28B1AF49484684
:1055500006F056FDC7F89000D7F89030AC49002B04
:1055600008BF01234846C7F8903006F049FDA94915
:10557000F861484606F025FD20B1A649484606F0E8
:105580003FFDF867FB6FA449002B08BF0123484685
:10559000FB6706F035FDA149F863484606F030FD8B
:1055A0009F497864484606F00CFD48B19C4948463E
:1055B00006F026FD9B4B0028CCBF012200221A706A
:1055C000994A494607F5807006F002FD974A494618
:1055D00007F5847006F0FCFC954A494607F588708B
:1055E00006F0F6FC934A494607F58C7006F0F0FC8D
:1055F000914A494607F5907006F0EAFC8F4A494601
:1056000007F5947006F0E4FC8D4A494607F598705A
:1056100006F0DEFC8B4A494607F59C7006F0D8FC84
:10562000894A494607F5A07006F0D2FC874A4946E8
:1056300007F5A47006F0CCFC8549484606F0EAFC64
:10564000014607F5E4700CF08FFA824A494607F5E7
:10565000A87006F0BDFC804A494607F5AC7006F01C
:10566000B7FC7E4A494607F5B07006F0B1FC7C4AAB
:10567000494607F5B47006F0ABFC7A4A494607F58F
:10568000B87006F0A5FC784A494607F5BC7006F0EC
:105690009FFC0024754A494607F5C07006F098FC47
:1056A000FC64FC65D7F8FC3003B1DB689C4280F2F7
:1056B0009480214607F1F80006F043FC014607F507
:1056C000F4700CF051FA6A4B07F5F471E6B207F585
:1056D00042701E710CF0CAFAD7F8943052465946FF
:1056E00007F54270FEF702FE054607F542700CF022
:1056F000FBF9224607F59C7107F5427006F0F1FBB5
:10570000D7F80C3303B1DB68FA6C03FB05230025E3
:10571000FB64A846224607F59C7107F5427006F027
:10572000E0FBD7F80C3303B1DB689D4226DA224652
:1057300007F59C7107F51C7006F0D3FB294607F5A9
:105740001C7006F0FEFB014607F542700CF00CFAE7
:10575000D7F894305246594607F54270FEF7C6FD19
:10576000C7F8800007F542700CF0BEF9D7F880301A
:10577000002BC8BF08F101080135CBE7214607F12E
:10578000F80006F0DEFB014607F51C700CF0ECF9A2
:10579000374B07F51C7107F542701E710CF066FA65
:1057A00052465946D7F8943007F54270FEF79EFDF1
:1057B000054607F542700CF097F9FB6D05FB0833C1
:1057C000FB652B4B07F51C701E710CF08DF907F56E
:1057D000F4700CF089F9013464E73B6E012B02D1BF
:1057E000244802F0ADFFFB6D9B000A3323F0070352
:1057F000ADEB030D02AB3B6400231A46F96D9942F1
:105800003ADD396C41F823200133F7E7D0A30100DA
:10581000E2A30100F1A30100FEA3010011A4010015
:1058200021A401007897FF1F2DA401003AA40100D4
:1058300049A4010056A4010067A401006AA4010064
:1058400083A4010059A401008DA401009EA40100BD
:10585000A6A40100ACA40100BAA40100C3A40100E5
:10586000CEA40100D8A4010091A10100E3A401008D
:105870005097FF1F50A90100FEF734FC31494846FC
:1058800006F09FFB00286ED02E4ADFF8D0804946F4
:1058900007F51C7006F09CFB2B4802F051FF00241A
:1058A000D7F8743203B1DB689C4259DA224607F517
:1058B0001C7107F5427006F014FB002107F54270D9
:1058C00006F01DFB0FF0C0F82246064607F51C71D6
:1058D00007F5427006F005FB012107F5427006F05E
:1058E0000EFB0FF0F9F8D8F8003003EB86030546FD
:1058F000996FC7F880300FF0E1FB10B9D7F880300E
:105900009D67124B1B78D807FBD5114802F018FF92
:10591000304602F08BFF0F4802F012FF00212846AC
:1059200002F06CFF0C4802F00BFFD7F8743203B1A1
:10593000DB68013B9C4202DA064802F001FF0134B9
:10594000AEE700BFEBA4010000A50100010002408A
:1059500080A1010097A201007CB70100BC8CFF1F51
:10596000D94802F0EDFED94907F1D00006F029FB35
:1059700038B1D74B1B68C7F8B830D64BD7F8B8202A
:105980001A60D54907F1D00006F01BFB80B1D3485F
:1059900002F0D6FECE4B1B68C7F8BC30CD4BD7F813
:1059A000BC001B68C01A02F041FFCD4802F0C8FEDF
:1059B000CC49484606F005FB00287AD0C94A49463A
:1059C00007F51C7006F004FB002107F51C7006F0BB
:1059D000B8FA014607F542700CF0C6F8D7F89430D3
:1059E0005246594607F54270FEF780FC044607F51B
:1059F00042700CF079F8BB4A494607F51C7006F076
:105A0000E7FA012107F51C7006F09BFA014607F53D
:105A100042700CF0A9F8D7F894305246594607F571
:105A20004270FEF763FC054607F542700CF05CF827
:105A3000AC4A494607F51C7006F0CAFA022107F580
:105A40001C7006F07EFA014607F542700CF08CF8E7
:105A5000D7F894305246594607F54270FEF746FC97
:105A6000064607F542700CF03FF89E4A494607F596
:105A70001C7006F0ADFA032107F51C7006F061FA00
:105A8000014607F542700CF06FF8D7F89430524693
:105A9000594607F54270FEF729FC804607F542702B
:105AA0000CF022F80FFA88F332B229B220B204F0D7
:105AB000EAF98D49484606F084FA88B18B4802F02D
:105AC0003FFE8949484606F0A5FA02F039FE8848AB
:105AD00002F036FE8449484606F09CFAFCF720FDA9
:105AE0008449484606F06DFA28B100231A46194643
:105AF000184604F0C8F98049484606F062FA48B1F1
:105B00007E4802F01DFE05F041F902F08FFE744858
:105B100002F016FE7A49484606F053FAC0B17849B9
:105B2000484606F077FA014607F542700CF01CF87B
:105B3000D7F894305246594607F54270FEF7D6FB27
:105B4000044607F542700BF0CFFF204605F0EEFA51
:105B50006C49484606F035FA002847D0694A49465C
:105B600007F51C7006F034FA002107F51C7006F0EA
:105B7000E8F9014607F542700BF0F6FFD7F89430CC
:105B80005246594607F54270FEF7B0FB054607F549
:105B900042700BF0A9FF5B4A494607F51C7006F0FE
:105BA00017FA012107F51C7006F0CBF9014607F53D
:105BB00042700BF0D9FFD7F894305246594607F59A
:105BC0004270FEF793FB044607F542700BF08CFF22
:105BD0004D4802F0B5FD204602F028FE02F072FEAC
:105BE00021462846FAF742FCFAF770FC474907F1CC
:105BF000D00006F0E6F940B3444A07F1D00107F5BA
:105C00001C7006F0E5F9002107F51C7006F099F903
:105C1000014607F542700BF0A7FFD7F894305246C3
:105C2000594607F54270FEF761FB044607F54270DE
:105C30000BF05AFF012120200AF012F90C200AF083
:105C4000D3F8214620200AF0B5F9314907F1D000F8
:105C500006F0B7F900285FD02D4A07F1D00107F50B
:105C6000427006F0B5F9002107F5427006F05FF9C1
:105C7000274A054607F1D00107F5427006F0A8F95A
:105C8000012107F5427006F052F92DB20446214871
:105C900002F056FD284602F0C9FD24B2104802F079
:105CA0004FFD204602F0C2FD0D4802F049FD3AF9D1
:105CB000150004440C2000FB04B0FEF7DFFE024890
:105CC00002F03EFD28E000BF77A6010019A5010003
:105CD000889DFF1FF897FF1F20A5010027A5010041
:105CE00097A2010031A501003BA5010043A50100D9
:105CF00096A201004FA5010057A501005BA5010078
:105D000062A5010069A5010071A501007CA5010043
:105D1000AFA20100B7A20100E94907F1D00006F0E7
:105D200050F9002843D0E64A07F1D00107F51C706E
:105D300006F04EF9002107F51C7006F002F9014645
:105D400007F542700BF010FFD7F8943052465946D1
:105D500007F54270FEF7CAFA044607F542700BF0E9
:105D6000C3FED74A07F1D00107F51C7006F030F9E1
:105D7000012107F51C7006F0E4F8014607F54270B2
:105D80000BF0F2FE52465946D7F8943007F54270B0
:105D9000FEF7ACFA054607F542700BF0A5FE284663
:105DA0000EF0A4FF00220146204605F031F8C54957
:105DB00007F1D00006F005F9002800F08580C14AFF
:105DC00007F1D00107F51C7006F002F9002107F574
:105DD0001C7006F0B6F8014607F542700BF0C4FEE1
:105DE000D7F894305246594607F54270FEF77EFACE
:105DF000044607F542700BF077FEB24A07F1D00176
:105E000007F51C7006F0E4F8012107F51C7006F098
:105E100098F8014607F542700BF0A6FED7F89430CB
:105E20005246594607F54270FEF760FA054607F5F7
:105E300042700BF059FEA34A07F1D00107F51C7020
:105E400006F0C6F8022107F51C7006F07AF8014644
:105E500007F542700BF088FED7F894305246594649
:105E600007F54270FEF742FA064607F542700BF05E
:105E70003BFE944A07F1D00107F51C7006F0A8F824
:105E8000032107F51C7006F05CF8014607F5427027
:105E90000BF06AFED7F894305246594607F5427027
:105EA000FEF724FA804607F542700BF01DFE3046DF
:105EB0000EF01CFF064628460EF018FF434601462A
:105EC0003246204605F0B2F87F4907F1D00006F0CF
:105ED00078F8D8B17C4907F1D00006F09BF801466C
:105EE00007F542700BF040FED7F894305246594601
:105EF00007F54270FEF7FAF9044607F542700BF019
:105F0000F3FD20460EF0F2FE05F0E0F96F4907F1CF
:105F1000D00006F056F800283FD06C4A07F1D001B7
:105F200007F51C7006F054F8002107F51C7006F008
:105F300008F8014607F542700BF016FED7F89430CA
:105F40005246594607F54270FEF7D0F9044607F568
:105F500042700BF0C9FD5D4A07F1D00107F51C70D6
:105F600006F036F8012107F51C7005F0EAFF01463E
:105F700007F542700BF0F8FD5946D7F894305246B9
:105F800007F54270FEF7B2F9054607F542700BF0CF
:105F9000ABFD2946204605F095F94D4907F1D000A3
:105FA00006F00FF8C8B14A4907F1D00006F032F800
:105FB000014607F542700BF0D7FDD7F894305246F2
:105FC000594607F54270FEF791F9044607F542700D
:105FD0000BF08AFD204605F003F93E4907F1D00099
:105FE00005F0EFFF002857D03A4A07F1D00107F536
:105FF0001C7005F0EDFF002107F51C7005F0A1FFF6
:10600000014607F542700BF0AFFDD7F894305246C9
:10601000594607F54270FEF769F9044607F54270E4
:106020000BF062FD2B4A07F1D00107F51C7005F05B
:10603000CFFF012107F51C7005F083FF014607F52E
:1060400042700BF091FDD7F894305246594607F54F
:106050004270FEF74BF9054607F542700BF044FD20
:106060001D4802F06DFB204602F0E0FB02F02AFC26
:10607000284602F0DBFB194802F062FB2946204665
:10608000FBF736F964200AF089F820462946FBF729
:106090002FF964200AF082F8114907F1D00005F0C9
:1060A00090FF00287CD00E4A07F1D00107F51C7044
:1060B00005F08EFF002107F51C7005F042FF11E08E
:1060C000A5AC010084A5010091A50100A7A50100D0
:1060D000AEA50100B6A50100BEA5010077A601008E
:1060E000CAA50100014607F542700BF03DFDD7F847
:1060F00094305246594607F54270FEF7F7F80446C9
:1061000007F542700BF0F0FCBA4A07F1D00107F531
:106110001C7005F05DFF012107F51C7005F011FFF3
:10612000014607F542700BF01FFDD7F89430524638
:10613000594607F54270FEF7D9F80EF0D7FD06462E
:1061400007F542700BF0D0FC0A2CA8BF0A2424EA01
:10615000E474A1B23046FAF74BFB0546A64802F0BC
:10616000EFFA204602F062FB02F0ACFB022130465F
:1061700002F044FB02F0A6FB284602F057FB9F48C2
:1061800002F0DEFA29462046FAF77EF9FAF79EF980
:106190009B4B1A5D9B4B53F83230012283F88020D1
:1061A000994907F1D00005F00CFF68B1964A07F154
:1061B000D00107F5427005F00BFF002107F5427092
:1061C00005F0B5FE04F000FD904907F1D00005F0A0
:1061D000F8FE40B98E4907F1D00005F0F2FE002824
:1061E00000F0CE80A9E0894A8A4C07F1D00107F57A
:1061F000427005F0EDFE002107F5427005F07FFECC
:106200002568C7E92001E86D0EF01AF902460B4631
:10621000D7E920010EF0D0FB20B9D7E920010EF01C
:106220005BFCE8657C4A13787B4D13F0010FFAD0D4
:10623000764A07F1D00107F5427005F0C9FE012149
:1062400007F5427005F05BFE2668C7E92001306E55
:106250000EF0F6F802460B46D7E920010EF0ACFB33
:1062600020B9D7E920010EF037FC30662B78D9072A
:10627000FCD5664A07F1D00107F5427005F0A8FE8B
:10628000022107F5427005F03AFE2668C7E92001B1
:10629000706E0EF0D5F802460B46D7E920010EF0DD
:1062A0008BFB20B9D7E920010EF016FC70662B7825
:1062B000DA07FCD5554A07F1D00107F5427005F021
:1062C00087FE032107F5427005F019FE2668C7E92D
:1062D0002001B06E0EF0B4F802460B46D7E920015B
:1062E0000EF06AFB20B9D7E920010EF0F5FBB0668D
:1062F0002B78DB07FCD5454A07F1D00107F5427042
:1063000005F066FE042107F5427005F0F8FD2468EB
:10631000C7E92001A06D0EF093F802460B46D7E9BD
:1063200020010EF049FB20B9D7E920010EF0D4FB83
:10633000A0652B78DE07FCD54CE7354A07F1D00184
:1063400007F5427005F044FE002107F5427005F0A4
:10635000D6FD304B1E680446B06D0D460EF070F849
:1063600002460B46204629460EF026FB20B9204661
:1063700029460EF0B1FBB065274A1378DC07FCD53F
:10638000264907F1D00005F01CFE18B101210020BC
:10639000FAF706FF224907F1D00005F012FE0028A7
:1063A00048D1204907F1D00005F00BFE002857D056
:1063B0001C491D4C07F1D00005F02CFE014607F5E5
:1063C00042700BF0D1FBD7F894305246594607F58E
:1063D0004270FDF78BFF207007F542700BF084FBD5
:1063E000124802F0ADF9207802F020FA104802F0CD
:1063F000A7F935E0CAA50100D7A5010077A60100DD
:10640000189A010038B00100ACAC0100CFA5010022
:10641000E4A50100BC8CFF1F01000240F1A50100B2
:10642000F6A5010000A601001499FF1F11A60100A6
:1064300097A20100CC4907F1D00005F0D7FD0EF07E
:106440004BFBCA4B1C68D4F8981005460EF036FE7C
:1064500008B9C4F89850C64A1378D807FCD5A0E705
:10646000C44907F1D00005F0ACFD002800F0C18060
:10647000C148C7F880D002F063F9C04802F060F963
:10648000BC4907F1D00005F0C5FD014607F5EC70E9
:106490000BF06AFBD7F8E031D7F8D811083323F0B6
:1064A0000703ADEB030D0DF1080840460FF01EFC8D
:1064B000402140460FF002FC0646002856D007F562
:1064C0004274C8EB00052A464146013520460FF0CC
:1064D00032FC4FF00008214607F51C7004F80580D7
:1064E0000BF042FB07F51C7002F0C0F907F51C70B9
:1064F0000BF0FAFA0422314607F5C4700FF01BFCCA
:1065000007F5C47107F5F47087F88C810BF02CFB4C
:10651000D7F8943000935A46534607F5F47107F5BF
:106520001C70FEF70DFA07F51C7002F09FF907F5D5
:106530001C700BF0D9FA07F5F4700BF0D5FA9048FF
:1065400002F0FEF8311D20460FF0D0FB214607F582
:106550001C7004F805800BF007FB07F51C7002F0B7
:1065600085F907F51C700BF0BFFA06E0814907F1C9
:10657000D00005F04FFD02F0E3F802F0B3F98149D5
:106580009623002207F51C7002F0B2F97E4802F053
:10659000D7F807F51C7002F0D3F87C4802F0D0F869
:1065A0007B4907F51C700FF097FBE0B9794B1B682E
:1065B000012B0CBF7848794802F0C2F8FB6F07F551
:1065C000EC70013BC7F88C300BF08EFA07F5E470E5
:1065D000D7F880D00BF088FAFB6ED7F830D0C7F828
:1065E000883001F0AEBA07F5EC700BF07DFAD7F801
:1065F00080D06B4907F1D00005F0E3FC002800F0E3
:1066000098805D48C7F874D002F09AF8654802F0A7
:1066100097F8634907F1D00005F0FCFC014607F547
:10662000EC700BF0A1FAD7F8E031D7F8D8110833A5
:1066300023F00703ADEB030D0DF1080840460FF002
:1066400055FB402140460FF039FB064600285AD042
:1066500007F54274C8EB00052A464146013520463D
:106660000FF069FB4FF00008214607F51C7004F895
:1066700005800BF079FA07F51C7002F0F7F807F5C2
:106680001C700BF031FA07F5C4730422314618462A
:10669000C7F880300FF04FFBD7F8803007F5F47063
:1066A000194683F804800BF05FFAD7F89430009312
:1066B0005A46534607F5F47107F51C70FEF740F98A
:1066C00007F51C7002F0D2F807F51C700BF00CFAFD
:1066D00007F5F4700BF008FA294802F031F8311D83
:1066E00020460FF003FB214607F51C7004F80580D7
:1066F0000BF03AFA07F51C7002F0B8F807F51C70B9
:106700000BF0F2F906E0264907F1D00005F082FC13
:1067100002F016F802F0E6F800211A4802F046F9F5
:10672000214802F00DF807F5EC700BF0DDF9D7F811
:1067300074D01E4907F1D00005F043FCD0B301200E
:1067400002F00CFC092835DC194801F0F9FF02F0D1
:10675000ABF802F047F807F5E4700BF0C5F9D7F88D
:1067600030D001F019BA00BFF6A50100BC8CFF1FA4
:106770000100024025A601002CA6010038A6010058
:10678000BC97010042A00100F7AA010076A6010013
:1067900043A60100E497FF1F47A6010056A601008B
:1067A00063A6010069A6010073A601007AA6010094
:1067B0002EA30100A34907F1D00005F002FC002838
:1067C00000F0B1809F4A07F1D00107F5427005F053
:1067D000FFFB002107F5427005F091FB0B460246D6
:1067E0000020FAF711FE142009F0D8FC954A07F1B1
:1067F000D00107F5427005F0EBFB012107F542706F
:1068000005F07DFB0B4602460820FAF7FDFD14203B
:1068100009F0C4FC8B4A07F1D00107F5427005F07E
:10682000D7FB022107F5427005F069FB0B460246D3
:106830001020FAF7E9FD142009F0B0FC814A07F1B5
:10684000D00107F5427005F0C3FB032107F5427044
:1068500005F055FB0B4602461820FAF7D5FD14202B
:1068600009F09CFC774A07F1D00107F5427005F06A
:10687000AFFB042107F5427005F041FB0B460246D1
:106880002820FAF7C1FD142009F088FC00226E4B85
:106890002020FAF7B9FDC82009F080FC6B4801F010
:1068A0004FFF0020FAF77EFD0EF016F9062101F0E9
:1068B000A5FF674801F044FF0820FAF773FD0EF0CA
:1068C0000BF9062101F09AFF614801F039FF102011
:1068D000FAF768FD0EF000F9062101F08FFF5C4821
:1068E00001F02EFF1820FAF75DFD0EF0F5F80621F5
:1068F00001F084FF564801F023FF2820FAF752FDEB
:106900000EF0EAF8062101F079FF514801F018FF76
:106910002020FAF747FD0EF0DFF8062101F06EFFA8
:106920004C4801F00DFF4C4907F1D00005F049FB40
:10693000002852D0484A07F1D00107F5427005F00F
:1069400047FB002107F5427005F0F1FA424AC7F80B
:10695000800007F1D00107F5427005F039FB0121F5
:1069600007F5427005F0E3FA3B4A07F1D00106460D
:1069700007F5427005F02CFB022107F5427005F087
:10698000D6FA354A044607F1D00107F5427005F002
:106990001FFB032107F5427005F0C9FA80462F4816
:1069A00001F0CEFE631E00257B67A54212DA314658
:1069B000D7F8800004F0F8FB022101F01FFF4046E9
:1069C00009F0ECFB7B6F9D4202DA214801F0B8FE32
:1069D0000135EAE71F4801F0B3FE214907F1D00075
:1069E00005F0EFFA002846D01E4801F0A9FE1C4928
:1069F00007F1D00005F00EFB03781949402B07F191
:106A0000D00031D105F006FB014607F51C700BF0F4
:106A1000ABF8D7F8943000935A46534607F51C71EB
:106A200007F54270FDF78CFF07F5427001F01EFF7D
:106A300007F542700BF058F807F51C700BF054F88E
:106A400016E000BF88A601000000F03F8DA60100FF
:106A500097A2010077A601009BA60100A2A6010053
:106A6000A6A40100ADA6010005F0D4FA01F068FE6D
:106A7000AF4801F065FEAF4907F1D00005F0A1FA7B
:106A800008B104F03BF9AC4907F1D00005F099FAE0
:106A900008B104F057F9A94907F1D00005F091FABF
:106AA00008B104F00FF8A64907F1D00005F089FA03
:106AB00010B10020FBF72CFAA24907F1D00005F035
:106AC00080FA08B1FAF728FC9F4907F1D00005F0D9
:106AD00097FA30B19D4C206803F0F4FB206803F076
:106AE000C3FB9B4907F1D00005F06BFA28B3984926
:106AF000984D994C07F1D00005F08CFA014607F546
:106B000042700BF031F852465946D7F8943007F5E9
:106B10004270FDF7EBFB0EF0E9F8286007F54270D4
:106B20000AF0E2FF2B688D48236001F009FE012185
:106B3000206801F063FE01F0C5FE894907F1D0002D
:106B400005F05EFA78B1864907F1D00005F058FAF1
:106B5000002808DD824907F1D00005F051FA814B89
:106B6000984241F33380804907F1D00005F048FA9C
:106B700018B1764B186803F0A5FB7C4907F1D000EB
:106B800005F03EFA18B1714B186803F06DFB7849B7
:106B900007F1D00005F034FA30B16C4C206803F0F6
:106BA00091FB206803F060FB724907F1D00005F00B
:106BB00027FA40B16F4907F1D00005F021FA634B85
:106BC000196803F0DDF96C4907F1D00005F018FAF7
:106BD00068B169495D4C07F1D00005F011FA2168F0
:106BE000054603F0CDF92168284603F087FA63498A
:106BF00007F1D00005F004FA40B1604907F1D00078
:106C000005F0FEF9514B196803F078FA5C4907F179
:106C1000D00005F0FFF9C8B1594907F1D00005F0DF
:106C2000F9F9014607F542700AF09EFFD7F8943053
:106C30005246594607F54270FDF758FB044607F5E2
:106C400042700AF051FF204609F0A8FA07F5B07427
:106C500054F8043CA4F1080163B1DB68002B09DDA2
:106C6000D7F894300193CDF800A05B46002203C909
:106C7000FDF7F2FB63686BB1DB68002B0ADDD7F828
:106C800094300193CDF800A05B46012294E8030004
:106C9000FDF7E2FBD7F86C2107F5B47332B1D26887
:106CA000002A03DD93E80300FDF740F807F5B87309
:106CB000C7F880305B68002B7DD0DB68002B7ADD65
:106CC000304907F51C700AF04FFF0022D7F88010FA
:106CD00007F5427005F005F9D7F80C436E4604B18C
:106CE000E46824B2630003F1080222F00702ADEB6E
:106CF000020D02AD2B442A4600219A4202D14FF0E8
:106D0000000802E022F8021BF7E7A0453CDA002267
:106D1000D7F8801007F5427005F0E3F8414607F513
:106D2000427005F004F925F8180008F10108ECE7B5
:106D300096A20100B7A60100C6A60100E0A60100C8
:106D4000EAA60100F9A6010002A70100B88CFF1F06
:106D500013A701007C99FF1F3C99FF1F27A7010083
:106D60003EA701003F420F0054A7010086A7010083
:106D70006AA701004CA7010062A701007EA70100DD
:106D800095A70100D8A4010007F51C7107F5427012
:106D90000AF06CFF00234FF07E5207F5427128463F
:106DA000FDF746F807F542700AF09EFE07F51C70E5
:106DB0000AF09AFEB546D7F87C310BB3DB68002B9E
:106DC0001EDDBF4907F51C700AF0CEFEBD4B1868EA
:106DD000C7F8E80107F51C7107F542700AF046FF95
:106DE0000023B94A07F5427107F5F470FDF720F862
:106DF00007F542700AF078FE07F51C700AF074FE81
:106E0000B24907F1D00005F0FBF830B1AF4907F106
:106E1000D00005F0F5F803F025F8FDF763F9D7F891
:106E2000903003EB8303BB600023C7F88030D7F8B2
:106E30009030D7F88020934240F3E38301F076FB53
:106E400030B10121A24801F0B1FD013000F0C78648
:106E500007F5A87393E8030007F5D07484E80300EE
:106E60000025636803B1DB689D4221DA2A4621468A
:106E700007F51C7005F035F8002107F51C7005F0CA
:106E800060F8014607F542700AF06EFE914907F579
:106E900042700AF01BFF002840F0B1868E4907F5CA
:106EA00042700AF013FF002840F0A98600F0C9BE26
:106EB0008A4907F1D00005F084F800286CD0874A91
:106EC00007F1D00107F51C7005F082F8002107F5E5
:106ED0001C7005F036F8014607F542700AF044FED2
:106EE000D7F894305246594607F54270FDF7FEF93F
:106EF000044607F542700AF0F7FD784A07F1D00121
:106F000007F51C7005F064F8012107F51C7005F009
:106F100018F8014607F542700AF026FED7F89430BB
:106F20005246594607F54270FDF7E0F9054607F568
:106F300042700AF0D9FD694A07F1D00107F51C70CB
:106F400005F046F8022107F51C7004F0FAFF01462F
:106F500007F542700AF008FE52465946D7F89430B9
:106F600007F54270FDF7C2F9064607F542700AF0D0
:106F7000BBFD5B4801F0E4FB204601F057FC01F04B
:106F8000A1FC284601F052FC564801F0D9FB2A46E4
:106F90003146204602F0BAFF534907F1D00005F010
:106FA00039F8C8B1504907F1D00005F033F801466F
:106FB00007F542700AF0D8FDD7F89430524659468A
:106FC00007F54270FDF792F9044607F542700AF0A2
:106FD0008BFD204609F0E2F800237B6700233B622B
:106FE000BB6300237B621E46BB64BB661C463B65DD
:106FF000FB6C7A6F934240F3EC82BB6EC7F80CD007
:10700000002B40F0E280224607F59C7107F54270A4
:1070100004F067FFD7F80C331BB1DB687B66002BED
:1070200001DC01237B66002307F5FC7107F5127272
:1070300051F8231042F8231001330A2BF4D1002514
:10704000224607F58C7107F51C7004F04AFF2946AB
:1070500007F51C7004F075FF014607F542700AF051
:1070600083FD52465946D7F8943007F54270FDF734
:107070003DF907F5FC7343F8250007F542700AF067
:1070800033FD002107F51C700AF06EFDD7F824319E
:1070900063B3DB689C4229DA224607F5907107F555
:1070A000427004F01EFF294607F5427004F049FFC4
:1070B000014607F51C700AF0ECFDFC6227E000BFFA
:1070C00091A10100F499010000000C42A9A7010060
:1070D00042A00100B8A70100D6A7010022A9010023
:1070E00033A9010077A60100E2A30100FA6A07F5BF
:1070F000907107F5427004F0F4FE294607F54270DE
:1071000004F01FFF014607F51C700AF0C2FD07F5E9
:107110001C7107F542700AF0A9FDD7F89430524669
:10712000594607F54270FDF7E1F8064607F542704B
:107130000AF0DAFC07F5087307F51C7043F82560C0
:1071400001350AF0D1FC0A2D7FF47AAFBC4907F56E
:107150001C700AF009FDD7F8243173B1DB689C423A
:107160000BDA214607F5847004F0EBFE014607F5C3
:107170001C700AF08EFDBC6209E0B96A07F58470E4
:1071800004F0DFFE014607F51C700AF082FDAD4BEE
:10719000D7F870121C7107F542700AF0E5FCD7F8B9
:1071A00094305246594607F54270FDF79FF806465F
:1071B00007F542700AF098FC002E07F51C7008BF16
:1071C00001260AF091FC012300E00023214607F18B
:1071D000E8007B6304F0ABFE224607F59C7185B2A4
:1071E00007F51C7004F07DFE7A6E396D3B6DB3FBC4
:1071F000F2F302FB1313194607F51C70BB6504F08C
:10720000A0FE014607F542700AF0AEFCD7F89430B4
:10721000DFF844825246594607F54270FDF766F89A
:1072200088F8000007F542700AF05EFC224607F578
:10723000947107F5427004F054FEB96D07F5427081
:1072400004F07FFE014607F5EC700AF08DFCD7F8DC
:10725000D81107F542700AF087FCD7F894305246EF
:10726000594607F54270FDF741F80DF03FFDB86152
:1072700007F542700AF038FCBB69002118460DF092
:1072800027FF98F80080BB6920B103F100400DF0A2
:1072900083FF03E041461846F9F7AAFA0146404643
:1072A000F9F7F2F8224607F5987107F51C7004F01B
:1072B00018FEB96D07F51C7004F043FE014607F592
:1072C00042700AF051FC52465946D7F8943007F5FF
:1072D0004270FDF70BF803B207F54270BB610AF08C
:1072E00003FC224607F1F00107F5427004F0F9FDB6
:1072F000B96D07F5427004F01AFE2246786107F571
:10730000887107F54270B7F8148004F0EAFDB96D92
:1073100007F5427004F015FE014607F5F4700AF017
:1073200023FCD7F8E81107F542700AF01DFCD7F8E6
:1073300094305246594607F54270FCF7D7FF424B4E
:10734000188007F542700AF0CFFB002D08BF132507
:10735000B8F1000F00F0DA86C5F34F05BB6E7A6E08
:10736000934228DA002207F5FC7353F82230E3B188
:1073700007F5087151F82200002807DA414289B266
:107380001846BA65F9F780F8BA6D0EE099B27A60DE
:107390003B61B9650DF0AAFCB96DF9F729FA3B69B3
:1073A00001461846F9F770F87A6801320A2ADAD1EC
:1073B000F9F78CF805E0B6F5E17F02D9A6F5E170A2
:1073C00000E03046F9F73CFE01F0B0F830B10121A1
:1073D0001E4801F0EBFA013000F0A286D7F8043124
:1073E0005BB1DB68002B08DD214607F5807004F0F7
:1073F0009EFD002801DD08F0D1FE6B00083323F06C
:107400000703ADEB030D02AAADEB030D02AB3B612D
:107410000F4BBA6500221A601A68002AFCD00D4B87
:1074200000221A60B8F1000F18D0BA8A0095B86926
:107430003B69B96D013A013804F0FAF812E000BF77
:1074400065A101005097FF1F1497FF1F42A0010084
:107450003098FF1FCC97FF1F2C98FF1F2946B86D4F
:1074600004F0B2F862B6B54AB86D10231360402339
:10747000136029464FF07C5201F070FC0DF032FC95
:10748000B865B8F1000F1CD04FF07C52294638691E
:1074900001F064FC0DF026FC7B6A13B9BB6D3B6206
:1074A000B863B96B0DF06CFB396A0DF073FCB96B06
:1074B0000DF024FD0146B86D0DF062FB0123B865A7
:1074C0007B627B6BB3B99E4B1B78002B37D0BA6CB9
:1074D0003B6C53F822000DF005FCB96D0DF052FB2A
:1074E0000DF05AFEBA6C3B6C43F822001346013390
:1074F000BB6424E0934994487D6B002307F5127226
:1075000052F8232022B1825C51F8322082F80051D7
:1075100001330A2BF2D1F8F7D9FF8A498A480023B0
:10752000012507F5FC7252F8232022B1825C51F844
:10753000322082F8805001330A2BF2D1C3E7BB6EB0
:107540000133BB663B6D2146013307F1F8003B6513
:1075500004F0F7FC014607F51C700AF005FB7B4BB5
:1075600007F51C7107F542701C710AF07FFBD7F814
:1075700094305246594607F54270FCF7B7FE05466F
:1075800007F542700AF0B0FA224607F59C7107F53C
:10759000427004F0A6FCD7F80C3303B1DB68BA6E76
:1075A0006B439A4208BF002307F51C7004BFBB66FB
:1075B00001340AF099FA07F5F4700AF095FA07F524
:1075C000EC700AF091FA7B6FD7F80CD001337B672F
:1075D0000EE55F480AF020F9D7F880300133C7F88C
:1075E0008030D7F88020D7F8903093427FF71FACD7
:1075F000FB69002B7FF71BAC1946564801F0D6F902
:1076000015E407F1E00393E8030007F5D47888E870
:10761000030013E9030007F5D87585E8030019B1E5
:10762000CB68C7F8903001E0C7F89010D8F8046034
:1076300006B1F668002307F54274D7F8902093420C
:1076400022DA1A4629462046C7F8803004F049FC61
:107650000021204604F06BFCD7F8803029461A46FA
:1076600007F51C7004F03DFC012107F51C7004F0C7
:1076700068FC014620460AF077FA20460AF034FA00
:10768000D7F880300133D8E7002E13DC324E334870
:1076900001F056F80FCE07F51C750FC596E80F00E0
:1076A00085E80F00202200212046002507F03CFF3E
:1076B0007D676AE02A4801F043F8002529464046E4
:1076C00004F03FFC014620460AF04EFA25492046C8
:1076D0000AF0FCFA30B1244801F032F80020FAF741
:1076E00017FC1BE0214920460AF0F0FA38B1204B84
:1076F0001B68B3F8300380B201F0A8F80EE01D4813
:1077000001F01EF8206801F01BF81B4801F018F882
:107710002068F9F76BFA032101F070F8731EAB4291
:1077200002D001F0CFF802E0144801F009F8204639
:1077300001350AF0D9F9AE42C0D1A7E7C4F00F4035
:107740002C98FF1F38B00100189A01005097FF1FB6
:107750005099FF1F42A00100F89901003AA90100C9
:1077600047A90100F0A6010013A0010052A90100E1
:10777000BC8CFF1FF7AA0100D79A01005DA9010088
:1077800007F5EC700AF0B0F90135D7F8FC3003B119
:10779000DB689D4280F26581294607F1F80004F01C
:1077A000D0FB014607F5EC700AF0DEF907F5EC7145
:1077B00007F5F4700AF05AFAD7F894305246594651
:1077C00007F5F470FCF792FDF86407F5F4700AF021
:1077D0008BF90023BB65BB6DFA6C9342D0DA0023B2
:1077E000C7F8803007F59873BB632A4607F59C718C
:1077F00007F5F47004F075FBD7F8EC3103B1DB68E2
:10780000D7F880209A4280F229812A4607F59C7198
:1078100007F5C47004F065FBD7F8801007F5C47055
:1078200004F08FFB014607F5F4700AF09DF9D7F8D4
:1078300094305246594607F5F470FCF757FD8046E0
:1078400007F5F4700AF050F9B8F1000F40F3008129
:107850002A46B96B07F5F47004F043FBD7F88010A3
:1078600007F5F47004F063FB0023C7F89030BB66A3
:1078700007F590730646BB642A4607F58C7107F539
:10788000F47004F02EFBD7F8EC3103B1DB68D7F8C5
:1078900090209A4280F2AB802A4607F58C7107F55A
:1078A000C47004F01EFBD7F8901007F5C47004F004
:1078B00048FB014607F5F4700AF056F9D7F8943002
:1078C0005246594607F5F470FCF710FD386507F588
:1078D000F4700AF009F92A46B96C07F5C47004F08F
:1078E00000FBD7F8901007F5C47004F02AFB01469E
:1078F00007F5F4700AF038F95246D7F89430594633
:1079000007F5F470FCF7F2FC786207F5F4700AF002
:10791000EBF87B6AB7F85010796318460DF0E6F97A
:10792000796BF8F765FF3B6D022B1ED1B8F1010FA3
:1079300003D1F11E4A424A413BE0B8F1030F04D1A2
:10794000012E14BF0022022233E0B8F1060F04D149
:10795000012E14BF002203222BE0B8F10A0F27D119
:10796000012E14BF0022072223E03B6D092B1FD1FB
:10797000B8F1010F04D1032E14BF00220E2218E02B
:10798000B8F1030F04D1012E14BF0022082210E029
:10799000B8F1060F04D1012E14BF00220A2208E01C
:1079A000B8F10A0F04D1012E14BF00220D2200E00D
:1079B0000022BD4BD200D3F800E00023D11801F51E
:1079C00090713EF8111009B244F823100133082BCE
:1079D000F4D1224607F51C71F9F7B6FCBB6E0344DF
:1079E000BB66D7F890300133C7F8903044E7AE4B10
:1079F0001B681D3603EB860670680DF0A7FBAB4BCA
:107A00001B78012B064608D1B86E0DF06FF9A84916
:107A10000DF074FA0DF09AFB00E000207A6F3B6CD9
:107A200053F8223082199342A3EB0000A0EB06002A
:107A300002D200F0FBFE01E000F008FF7B6F013393
:107A40007B677A6FFB6D934202D09A4800F078FE14
:107A5000D7F880300133C7F88030C6E6BB6D0133FC
:107A6000B8E6954800F06CFEFB6E5A1ED7F88830D9
:107A700093420ADBBB6F396F013B994205DBF96F1B
:107A8000D7F88C000139884212DA00F01BFF7B6CBA
:107A9000002B03DD184608F081FB06E07B6C5A1CC6
:107AA00003DA1946854800F081FF0023194610E0EB
:107AB000D7F888109142F8D13A6F9A42F5D13B6ECF
:107AC0001BB97F4800F03CFEEFE77E4800F072FEF5
:107AD000EBE707F5FC7242F8231001330A2BF8D1CB
:107AE00007F5E4700AF000F83B6FD7F830D00133A7
:107AF000FDF7A3BC744800F023FED7F88C0000F01B
:107B000095FE724800F01CFEFB6ED7F88820013B02
:107B10009A4205DBFA6FD7F88C10013A914202DAEB
:107B200000F0D0FE0DE0D7F888209A4209D1684BCA
:107B30001B681BB9624800F003FE02E0614800F0D8
:107B400039FED7F888300133FDF7CDBBFB6B13B19D
:107B5000184608F023FBD7F88C300133C7F88C3077
:107B6000D7F88C20FB6F93423DF7B8AB574800F035
:107B7000E7FD00F099FE00F035FE564B1B785BB92F
:107B800001235548554C19461A5D013350F83220EF
:107B90000B2B82F80011F7D107F5DC7009F0A4FF78
:107BA00007F5C2476437BD46BDE8F08F4C4800F08A
:107BB00061FE284600F0C4FD414800F05BFEFDF781
:107BC0003CBBBB6F013B3B67FDF752BC454907F12E
:107BD000D00004F015FA444B1860FEF7C4BFFB6EEA
:107BE000013BC7F88830FB6F013BC7F88C30D7F8F2
:107BF0009030C7F88030BB6F3B67FFF729B9D7F8E3
:107C00009000F9F731FCD7F89030D7F88020013B8D
:107C10009A4240F09E80354800F092FD344B052199
:107C2000186800F0EBFD334800F08AFD324B052167
:107C3000186800F0E3FD314800F082FD0521304B6B
:107C40002CE0304907F542700AF040F830B92E496F
:107C500007F542700AF03AF8002863D0D7F8900090
:107C6000F9F74EFCD7F89030D7F88020013B9A42C4
:107C70006FD1264800F064FD254B0521186800F0FF
:107C8000BDFD244800F05CFD234B0521186800F081
:107C9000B5FD224800F054FD214B0521186800F085
:107CA000ADFD00F00FFE54E0BC8CFF1F1499FF1FC8
:107CB0000000204197A20100F8A2010042A00100AB
:107CC0007CB7010052A6010060A90100C0A001001C
:107CD000E497FF1F7897FF1F38B00100189A010042
:107CE00066A901003EA70100B88CFF1FDAA70100BA
:107CF0003499FF1FE9A701009497FF1FF6A7010021
:107D0000F896FF1F74A9010003A8010008A801004C
:107D10001897FF1F18A801003899FF1F26A8010017
:107D20007C97FF1FB14907F5427009F0CFFF00288B
:107D300061D00526322008F031FAB868F8F7BCFDAA
:107D4000013EF7D1D7F89030D7F88020013B9A4216
:107D500006D007F5427009F0C7FE0135FFF781B87C
:107D6000A34BA44A19681160A34A7B671168A34A10
:107D7000A34B1160A34A1968A34B1160A34A196869
:107D8000A34B1160A34A1968DFF8B4821160A24ABC
:107D9000D8F800101160A14AA148168000F0D0FC6C
:107DA0007B6F1E68314630460DF0BAF900B19D4E2A
:107DB0000321304600F022FD9B4800F0C1FC904BAF
:107DC0000121186800F01AFD984800F0B9FC8E4BAC
:107DD0000121186800F012FD954800F0B1FC8C4BB1
:107DE0000121186800F00AFD924800F0A9FC012169
:107DF000D8F8000053E7904907F5427009F066FF94
:107E000028B98E4907F5427009F060FFD8B17B4B65
:107E10001A68794B1A60774B1A68754B1A60794B60
:107E20001A68774B1A60794B1A68774B1A60794B4E
:107E30001A68774B1A60784B1A68814B1A60774B37
:107E400001221A8085E77F4907F5427009F03EFF5D
:107E500088B1D7F89000F9F727FCD7F89030D7F819
:107E60008020013B9A427FF474AF774800F068FCB1
:107E70000221764B12E7764907F5427009F026FF9A
:107E800090B1D7F890100120F9F79CFED7F8903008
:107E9000D7F88020013B9A427FF45BAF6D4800F039
:107EA0004FFC02216C4BF9E66C4907F5427009F072
:107EB0000DFF98B1D7F890100020F9F783FED7F89E
:107EC0009030D7F88020013B9A427FF442AF64485B
:107ED00000F036FC634B0021186880E0624907F52A
:107EE000427009F0F3FE064660B1604B00221A6052
:107EF0005F4B1A605F4B1A605F4B1A60012211469C
:107F0000104608E05D4907F5427009F0DFFE28B130
:107F1000012132460846F9F7F7FB1AE7584907F5F9
:107F2000427009F0D3FEE0B12A46214607F51C70E5
:107F300003F0D7FF012107F51C7003F0F8FFD7F815
:107F40009010F9F7A9FED7F89030D7F88020013BC0
:107F50009A427FF4FEAE4B4800F0F2FB03214A4BFD
:107F60009CE64A4907F5427009F0B0FEE0B12A46A6
:107F7000214607F51C7003F0B4FF012107F51C70C2
:107F800003F0D5FFD7F89010F9F7AEFED7F8903090
:107F9000D7F88020013B9A427FF4DBAE3C4800F0EA
:107FA000CFFB03213B4B79E63B4907F5427009F0D3
:107FB0008DFE002876D02A46214607F51C7003F076
:107FC00090FF012107F51C7003F0B1FF012103F0C0
:107FD000EBF80646314800F0B3FB0521304600F0CF
:107FE0000DFC2F4800F0ACFBB3E600BF2D9701005D
:107FF0003096FF1F4C99FF1F3C99FF1F7C99FF1F74
:108000003099FF1F7099FF1F4899FF1FF096FF1FBF
:108010005C97FF1F8897FF1FD497FF1F8097FF1F54
:1080200034A80100000080BF47A801004DA801004E
:1080300053A8010059A801002497010045970100A9
:108040007497FF1F93A901005FA801005896FF1FB6
:1080500073A801007DA801000C99FF1F8AA80100E8
:1080600098A801002C99FF1FA9A801009097FF1F55
:108070005496FF1F3496FF1FA497FF1FBBA8010053
:10808000D1A80100DDA801000097FF1FECA80100A6
:10809000F9A80100AC97FF1F9BA6010009A90100E8
:1080A00097A20100274907F5427009F00FFE00284A
:1080B0003FF44FAE2A46214607F51C7003F011FF2E
:1080C000012107F51C7003F032FF2A4606462146BF
:1080D00007F51C7003F005FF022107F51C7003F083
:1080E00026FFF6B2804600F02CFA0121304607F058
:1080F000B7FE154A52F8362018F0FF0F4FF0010373
:1081000014BF82F8803082F8003122E60F4BC3F8AA
:108110000080BB694146581E03F0B8F9FFF71EB94D
:10812000FB6F013BC7F88C30BB6F013B3B67FB6CBF
:108130007B67D7F89030C7F88030FB6EC7F888307F
:10814000FFF74CB914A9010038B00100CC97FF1F0C
:10815000F0B5314A314D136893B017460393304B55
:1081600003991960136802932E4B029919601368E2
:108170000193019B2B602C4B197801291E4617D1C6
:108180000524642008F00AF80023642219461046EA
:1081900001F079FE642008F001F800231A46194620
:1081A0001846013C01F06FFE14F0FF04E9D1347071
:1081B00000F00CFF41F2883600F0CBF9431C044676
:1081C0000DD13B680493049B2A689B1AB34203D9E0
:1081D00000F012FF01F0D0F800F0AEFFECE704F081
:1081E00069F95B2C06D100F0F1FE00F0FBFAFCF718
:1081F00077FC0DE000F0EAFE31234FF4FA720B49F0
:1082000005A800F075FB05A8FAF78AF900F0EAFA6C
:1082100000F0DCFE13B0F0BD889DFF1F4099FF1FEA
:108220007499FF1F5C99FF1FF497FF1F42A0010084
:1082300038B50E4D0E4C0021284609F095FC22461B
:108240000C4928460DF0B2F90B4803F0A7FA0B4889
:1082500003F0A4FA0A480B4900230360802303714A
:108260002246BDE838400DF0A1B900BF6099FF1F5C
:10827000B08CFF1FE91A01005C96FF1F9096FF1F4C
:108280005099FF1FD50F000038B50B4D0124285D14
:108290000121013407F0E4FD0B2CF8D10121062067
:1082A000064C07F0DDFD102323600121152007F0A7
:1082B000D7FD4023236038BDCCA90100C4F00F4096
:1082C00070B5404B404E00241C60404B8AB00125E5
:1082D0001D7000F07BFE3E4B3E481C801223417B0C
:1082E0000293132301930595049603950094234666
:1082F0002246006905F038F837481E23417B029377
:108300001D23019305950496039500942346224668
:10831000006905F029F800F0FFFC042000F0D8F80F
:108320004FF4E13000F0CAF82C4B4FF0FF321A60E6
:1083300000F082FCFFF7A8FF294805F0C9FF07F00D
:1083400003FB42F2117009F017FD264B186020461E
:1083500007F0F0F9102007F011FA042007F03AFABC
:10836000022007F0E7F907F029FD06F071F9642013
:1083700007F014FF23462A4621460F20F8F708F994
:108380002346214602220F20F8F702F92346214610
:1083900003220F20F8F7FCF8134B1A680992134ACE
:1083A000099911601A6808920899114A1B68079385
:1083B000104B1160079A1A600F4B1D700F4B1D7008
:1083C0000AB070BDD897FF1F00350C001499FF1F2D
:1083D0008097FF1FF49CFF1FE09CFF1FD097FF1F9B
:1083E0000C92FF1FE097FF1F889DFF1F4099FF1F02
:1083F0007499FF1F5C99FF1F1C99FF1FF497FF1FC3
:10840000094B1B7803F0FF006BB1084B187810F094
:10841000010008D0064B074A1B681068181A0E287E
:1084200094BF002001207047FF9EFF1F109FFF1F79
:10843000889DFF1F4CA0FF1F70B5044608460D46DF
:108440000DF05CFC23680246294620465B68BDE8C7
:108450007040184738B5084D2B685BB1074908488C
:108460000024CC54FFF7E8FF08F056F9204607F047
:1084700095FE2C6038BD00BFAC9AFF1F9C99FF1F72
:108480003893FF1FF8B50A4D0A4E0B4F441E14F8DF
:10849000012F62B12B68F2540133142B2B6002D1EF
:1084A000FFF7D8FFF3E73B68002BF0D1F8E7F8BD02
:1084B000AC9AFF1F9C99FF1F8899FF1F430803F187
:1084C000376303F5D833B3FBF0F007F0CFBEFFFFFF
:1084D0000428064A064B05BF012111600021032232
:1084E0000EBF1A6011601860704700BFB499FF1F7B
:1084F000C08CFF1F10B508F02BF9044630B10A4BB1
:108500000122BDE810401A6008F032B9FFF778FF89
:108510000028F0D008F0ACFE0028ECD0024B1C6024
:10852000BDE8104008F062BE9499FF1F10B5FFF738
:1085300067FF08B108F09CFE044608F009F92044E2
:1085400010BD08B5FFF7F2FF10B1FFF7D3FFF9E751
:1085500008BD08B508F0FCF818B1BDE8084008F0FF
:1085600031B9FFF74DFF30B108F082FE18B1BDE818
:10857000084008F061BE4FF0FF3008BD10B504465A
:108580004FF6FF700139C9B2FF290ED014F8012B44
:1085900082EA102383EA13139AB243EA002383EAA0
:1085A000023383EA421398B2ECE710BD2DE9F04F95
:1085B000474B1E688BB09846002E00F08580454FD3
:1085C000454C3B6806F1010941335FFA89F12046C9
:1085D000A355FFF7D3FF414A034605AD02F1100C46
:1085E00010685168AE46AEE8030008326245754631
:1085F000F6D112788EF800200AA9C3F30F320A448C
:108600000AA8C3F3032112F8142C04F8092001442A
:10861000A21911F8141C9170C3F3031103F00F0396
:108620000344014413F8143C11F8141C1371B31DD6
:10863000D17000250421DFF8AC905171DFF8A8A0BB
:10864000E554C8F80030CB4608F082F810B108F0C5
:108650008FF8F9E7DAF8003013B10DB9A01900E08E
:108660001D48FFF70FFFFFF7F5FED9F80030039321
:10867000039ADBF800300493049B9B1A632B07D901
:10868000174A1368013501333C2D1360DCD110E02B
:10869000019208F097F80130019AEAD008F068F8E2
:1086A000019008F08FF80130019BF7D1DBB2062B67
:1086B000E6D10023C8F800303B681A21013393FB50
:1086C000F1F201FB12333B600BB0BDE8F08F00BF4D
:1086D0008C99FF1F9099FF1FB899FF1FD7A9010020
:1086E0009899FF1F889DFF1FC48CFF1FF7B5114D80
:1086F000114E04462F4614F8012BC2B1042AFAD0B9
:108700002B68F25401332B600C4B1B684BB10023D8
:1087100002A8ADF8043014F8013C00F8043DFFF75E
:10872000B1FE3B68EA2BE6D1FFF740FFE3E703B079
:10873000F0BD00BF8C99FF1FB899FF1FC48CFF1FAD
:1087400038B5174B1B68044653B1164B1B6873B9F9
:10875000FFF756FEC8B121461348FFF76DFE14E03F
:10876000FFF74EFE114D60B92B689B070DD5104BDE
:108770001B68204613B1FFF7B9FF06E0FFF782FE42
:1087800003E02B68DA0705D4EEE72046BDE8384061
:1087900003F0BEBE21460448FFF74EFEE4E700BFEB
:1087A000B499FF1F9499FF1F5893FF1FC08CFF1FA0
:1087B0008899FF1F0FB413B5094C04ABC82153F8B7
:1087C000042B019320460EF035FA0023204684F84E
:1087D000C830FFF7B5FF02B0BDE8104004B07047E5
:1087E0003898FF1F08B5044B1B680BB1FFF7DEFE7E
:1087F000BDE80840FFF72EBE8899FF1F70B58EB008
:1088000006460D464C1C0CF0A1FC0A2318B190FB47
:10881000F3F00134FAE701AB2A462146304607F06F
:1088200049F901A8FFF78CFF0EB070BD00B58FB0FD
:108830000346054A322101A80DF0E2F901A8FFF72D
:108840007FFF0FB05DF804FB9F98010000B58FB06B
:108850000346054A322101A80DF0D2F901A8FFF71D
:108860006FFF0FB05DF804FBEDA901000068FFF792
:1088700067BFFFFF08B5FFF763FF0248BDE8084088
:10888000FFF75EBF64A1010000B58FB00346054A43
:10889000322101A80DF0B4F901A8FFF7EBFF0FB0EA
:1088A0005DF804FB9F98010008B503F00BFE03F090
:1088B000D9FDFFF7DFFFFFF795FFBDE8084003F0A4
:1088C000F9BDFFFF1FB50649684609F06DF9684616
:1088D000FFF7CCFF684609F007F905B05DF804FB27
:1088E00097A201000148FFF72BBF00BF96A201002D
:1088F0002DE9F04F1F4E85B01C4633680293DDF81A
:1089000008A00091054690464FF0000B3268039294
:10891000039FB8F1000F03D0CAEB0702904521D3A3
:10892000FFF717FE0130F1D0FFF7E4FDC2B2814638
:108930001146009801920DF0C1F998B9019A0E48BC
:1089400011460DF0BBF90028E0D105F80B900BF1B2
:10895000010B0CB9BA46D9E7A345FBD32C4404F864
:10896000010C02E0002205F80B20284605B0BDE806
:10897000F08F00BF889DFF1F63A1010000B589B083
:1089800018230A46014601A8FFF7B2FF9DF80430FC
:1089900023B101A800210EF023F801E002490020D4
:1089A00009B05DF804FB00BF0000F87F00B589B096
:1089B0000A461823014601A8FFF79AFF01A80CF008
:1089C000FEFD09B05DF804FB02880B889A4203D0D3
:1089D00004D84FF0FF3070470020704701207047E7
:1089E00070B54D4C4D4E4E4D31782B782278120497
:1089F000FF2042EA03234B4A30700B43287020705B
:108A000080206070A070D360474B9A7912F00C0FF1
:108A100005D19A79D50602D59A7994060BD59B791A
:108A2000414AC3F38103032B16D19379D80613D49B
:108A30009379990610D53D4B3D4A197852F821405B
:108A40001D46002C67D0236820469B6898472B78EA
:108A500004EB83046468F4E7334B9A79C2F3810230
:108A6000022A0CD19A79D20609D49A79960606D5AB
:108A70005A7802F0020202F0FF01002A42D02A4B8B
:108A80009A79C2F38102022A08D19A79D50605D4CF
:108A90009A79940602D45B789807CCD5224B9A79C0
:108AA000C2F38102022A05D19A79D10602D45A78FA
:108AB0009207C0D49B791C4AC3F38103012B08D1D0
:108AC0009379DB0605D593799E0602D453789D07EA
:108AD000B1D4154B9A79C2F38102012A08D19A794F
:108AE000D40605D59A79900602D45B789907A2D569
:108AF0000D4B9A7912F00C0F9DD19A79D2069AD427
:108B00009B7998E7202219701A709A7902F00C026A
:108B10000C2AFAD18FE770BD07C0074005C0074097
:108B200006C007402CA0FF1F004006406C9DFF1FA1
:108B30002C9DFF1F0F4B036090F924305A1CF0B599
:108B400017D00D4A52F823108842114611D10B4C10
:108B500054F823209F0000261AB1D5196A686E6068
:108B6000FAE744F8232041F82320054A1378013B13
:108B70001370F0BDFCA901004C9DFF1F2C9DFF1F31
:108B80006D9DFF1F7047FFFF10B5034B0360044648
:108B9000FFF7D0FF204610BDC8AF010010B5034B52
:108BA00003600446FFF7C6FF204610BDF0AF01008A
:108BB00010B5034B03600446FFF7BCFF204610BD11
:108BC000DCAF010038B590F92420531C15D00B49B7
:108BD000D3B20B700A494FF0FF300860094951F8D1
:108BE00022409D004CB194F825301BB123682046EB
:108BF0001B6898472C446468F4E738BD6C9DFF1FE0
:108C00000082FF1F2C9DFF1F08B5FFF715FC08BD54
:108C100038B50546FFF710FC0446284608F046FE26
:108C2000204438BD38B5054608F08BFE044628467A
:108C300008F03CFE204438BD38B501210220104D1B
:108C4000104C07F00DF9002201214FF4A0702960AB
:108C50000023934202D000BF0133FAE721600246AD
:108C6000013AFDD19A1C282AF1D1054B01221A6044
:108C70004FF47A7007F092FABDE83840F7F73CBC41
:108C8000C4F00F40C8F00F402DE9F041174E184DC9
:108C900033680124002B2C6026DC164F214602206D
:108CA00007F0DEF864203C6007F078FA14236FF0D8
:108CB000010000FB03F12C60283100228A4202D01F
:108CC00000BF0132FAE74FF001083C605A01013A57
:108CD000FDD1013BEDD16420C5F8008007F05EFABC
:108CE000F7F70AFCC6F80080BDE8F081D097FF1FB7
:108CF000C4F00F40C8F00F4008B5054B01221A60C0
:108D00000021022007F0ACF8024B00221A6008BDD7
:108D1000C8F00F40D097FF1F08B501211F2007F0B2
:108D20009FF80B4B01221A604FF47A7007F036FA65
:108D3000F7F7F4FC03F06EFD03F030FA77210548F5
:108D400002F0D6FE76210448BDE8084002F0D0BE0D
:108D5000C8F00F405C96FF1F9096FF1F70B50A4B3E
:108D60000E461546022204460CF0FAFD30460BF082
:108D7000BDFF29460CF00EF809F0CEFB0CF0E6F929
:108D800034F8100070BD00BFC9890000F8B5002498
:108D90000E460C600746411E234611F8012F82B192
:108DA0005D2A0AD003D85B2AF7D10133F5E77B2A85
:108DB00005D07D2AF1D1013CEFE7013BEDE701341D
:108DC000EBE703B924B1134B1B68336000251EE0A9
:108DD0005D2138460CF0C2FF08B90F4BF4E7451C83
:108DE00040780CF05CFC90B103F064FBE91B384662
:108DF00003F06EFB03F066FB03F034FB0822294608
:108E00000CF084FF18B1054B1B68336025462846DB
:108E1000F8BD00BFC88CFF1FCC8CFF1FD08CFF1F7C
:108E2000F8B5012107463C4D212007F019F8102321
:108E30002B604FF41653013BFDD164240026222001
:108E400006F0FAFC013C0644F9D11FB96423B6FBD5
:108E5000F3F449E04FF480610520F7F715FB4FF478
:108E600080610620F7F710FB40F2CA410820F7F7AF
:108E70000BFB40F2CA410920F7F706FB40F2CA415A
:108E80000A20F7F701FBF7F721FB012007F086F92D
:108E9000224B4FF400521A6020221A600222C3F8BB
:108EA00000214FF400221A640422C3F880204FF4FA
:108EB0007A53013BFDD16426222006F0BDFC013E21
:108EC0000444F9D16423B4FBF3F44FF400532B6052
:108ED00020232B60124B02221A604FF4002243F829
:108EE000C02C042243F8802C0021212006F0B8FF7A
:108EF00020460BF0F7FE4FF05E510BF04BFF094997
:108F00000BF048FF08490BF045FF08490BF0F6FF4E
:108F10000CF01CF9F8BD00BF08F00F4004F00F4042
:108F200008F10F40C3F5983F00007A4413E9813EF1
:108F300010B50446FFF774FF1CB10BF0D7FE0549CE
:108F400002E00BF0D3FE04490CF0C2F8003018BF69
:108F5000012010BD9A9959400000604038B5044680
:108F6000FFF75EFF0CB9154C00E0154C0BF0BEFE90
:108F700021460BF005FE2146054612480BF000FE87
:108F8000014628460BF0BAFF0F490BF003FF002102
:108F900004460CF0B1F84FF07C5118B120460BF0AC
:108FA000F1FD02E020460BF0EBFD0CF0CFF8642859
:108FB000D4BF20EAE070642038BD00BF00C05A452D
:108FC00000805445004083450000C842044B82B0F5
:108FD0001B680193019A034B1A6002B0704700BFEF
:108FE000889DFF1F1097FF1F014B024A1A607047B0
:108FF0000CED00E00400FA05164B1B68002B73B55E
:1090000026DD012001F070FA10B3134D134C2B68CC
:1090100000932268009B9B1A41F28832934217D931
:109020000020FFF79BFF0023C0F164061A4601B23F
:1090300030B200F028FF0A2007F0B0F800231A46EB
:109040001946184600F01FFF2B680193019B23600F
:1090500002B070BDD897FF1F889DFF1F5C99FF1F4E
:109060002DE9F041FFF7B2FF0020FFF777FFDFF8AF
:10907000C4802D4D6421044680260120F7F704FAB0
:109080000627F7F723FA94FBF7F0C8F8006007F01B
:1090900085F800210120F7F7F7F9F7F717FAC8214B
:1090A00002202E602026F7F7EFF9F7F70FFAC8F83D
:1090B0000060C4F1640090FBF7F007F06FF8002146
:1090C0000220F7F7E1F9F7F701FA002101202E60FD
:1090D000F7F7DAF9F7F7FAF900210220F7F7D4F9F0
:1090E000F7F7F4F92E60FAF7F9FF47F23053984298
:1090F00018DDC82007F052F84FF4FA710420F7F792
:10910000C3F9F7F7E3F9094B4FF480741C600A20A8
:1091100007F044F800210420F7F7B6F9F7F7D6F97D
:10912000034B1C60BDE8F081C8F00F4084F00F4095
:1091300088F00F40C4F00F40194B1B68002B37B567
:109140002CDD022001F0D0F940B31649164A0B6815
:1091500000931068009B1B1A40F6B83083421DD95B
:109160000B680193019B136000F08EFE054600F032
:10917000F9FE0E4B1B680446B3F8680180B20BF091
:10918000B5FD014628460BF0FBFC21460BF002FE24
:1091900000210BF09DFF08B1FFF762FF03B030BD67
:1091A000D897FF1F889DFF1F7499FF1FBC8CFF1F5E
:1091B00070B53C4B1021198003F1021303F53043C5
:1091C0001B781E076DD53848384D394C2B782678DA
:1091D00002788A4042EA06221A43FF232B7012F0DB
:1091E000010F237003704FF0800343708370314B85
:1091F00001D01A2246E0150701D5212242E0D4060B
:1092000001D504223EE0900601D599603BE0560668
:1092100001D5162236E0150601D5092232E0D40523
:1092200001D50A222EE0900501D50D222AE0510534
:1092300001D50B2226E0160501D51E2222E0D50419
:1092400001D502221EE0940401D507221AE0500441
:1092500001D5062216E0110401D5152212E0D6032D
:1092600001D524220EE0950301D522220AE0D40282
:1092700001D5252206E01003F7D45103F5D492025C
:1092800001D523229A600C4900220A704A708A7024
:10929000CA7018791A705A709A70DA7008711A7157
:1092A000DA6070BD0020054007C0074005C00740D8
:1092B00006C007402CA0FF1F00C0074010B50C4699
:1092C00069B101EB82035968FFF7F8FF94F8253084
:1092D0002BB1236820465B68BDE81040184710BDDD
:1092E00008B590F924305A1C05D00349DAB251F878
:1092F0002310FFF7E3FF08BD2C9DFF1F10B5124898
:10930000124CFFF7B7FA124B012264201A7006F0D4
:1093100045FF40F6B8310F4805F0F0FF0423002266
:1093200012210D4805F09CFC642006F037FF062151
:109330000A4805F0E1FA2428206003D1FFF709F973
:109340000130F4D010BD00BF08AA01009897FF1F9C
:10935000F497FF1F289BFF1F689BFF1FB09AFF1FFA
:1093600008B5FFF7C9FCFFF7D7FC0A2006F016FF87
:10937000BDE80840FFF7C2BF07B5144B14491A688F
:109380000092009A09681B680193521A41F28830D2
:10939000824288BF0F4A019B84BF012010600E4AA1
:1093A0001268D2F898215B1A93420BD9FAF796FE0D
:1093B00047F23053984203DD002001F095F808B9D8
:1093C000FFF7CEFF03B05DF804FB00BF889DFF1FD1
:1093D0001097FF1FD897FF1FBC8CFF1F2DE9F3418B
:1093E00036493748374FDFF8FC80FFF711FC01247E
:1093F0000025E6B23146334804F0DDF800237A7BDD
:10940000009339692F48012304F0A5FB002833D1CC
:109410002D492B48FFF7F8FB0F2C03D82B49284880
:10942000FFF7F2FB002310222146254808F04EFAF0
:1094300027492348FFF7ECFB0E2C05F101050CD161
:10944000244B1B6893F82C200E2A18BF83F82C405D
:1094500098F80030DA07FBD523E00F2E21D11D4B01
:109460001B6893F82C200F2A18BF83F82C6098F8FB
:109470000030DB07FBD514E0042812D11649104850
:10948000FFF7C2FB0F2C03D810490D48FFF7BCFBB8
:109490000023102221460A4808F018FA084808F06C
:1094A00005FA01347F2CA4D10DB90C4900E00C4918
:1094B0000348FFF7ADFB02B0BDE8F08114AA01003C
:1094C0005893FF1FF49CFF1F20AA010047AB010027
:1094D0002FAA0100BC8CFF1F33AA01003EAA010085
:1094E000E49801000100024070B58EB007F040F929
:1094F000061E2BDD642006F051FE002401AD6655EA
:1095000007F036F90134262C0646F7D11548002419
:109510008DF82A40FFF7AEF91348FFF7ABF928465C
:10952000FFF7A8F90F48FFF7A5F925220E492846AD
:109530000CF0ECFB90B10D48FFF79CF90A48FFF7DF
:1095400099F90B48FFF7FCF8284603E00948FFF7B4
:1095500091F90948FFF78EF9002000E001200EB0D4
:1095600070BD00BF4CAA010066AA01008DAA0100CF
:1095700098AA0100A4AA0100C2AA010000B53B48B4
:109580009BB0FFF7DDF84EF660220023384901A8B2
:10959000FFF7AEF94EF660213548FFF707FA4308AA
:1095A00003F1376303F5D833B3FBF0F006F05EFE4A
:1095B0004FF4FA6006F0F2FD2E492F48FFF724FB26
:1095C0004FF4FA6006F0EAFD2C492B48FFF71CFB2C
:1095D0004FF4FA6006F0E2FD29492A48FFF714FB30
:1095E00040F2D2412748FFF71DFB27492248FFF7E9
:1095F0000BFB40F2D2412048FFF714FB4FF4FA6016
:1096000006F0CCFD21491F48FFF7FEFA01A91D48CD
:10961000FFF7FEFA4FF4FA6006F0C0FD1C49164849
:10962000FFF7F2FA01A91448FFF7EEFA4FF4FA60D7
:1096300006F0B4FD17491348FFF7EAFA16490E4839
:10964000FFF7E6FA4FF4FA6006F0A8FDFFF74CFFCB
:1096500010B11248FFF70EF91148FFF70BF9114846
:10966000FFF708F91BB05DF804FB00BFEAAA010090
:1096700042A00100F9AA01003893FF1FFCAA0100D3
:1096800007AB01005893FF1F16AB01001DAB010093
:109690002CAB010034AB010049AB010052AB01001F
:1096A000BFA0010065A10100F8B5264A264B036062
:1096B0000F461178254D264EFF2380F824300629C9
:1096C0004FF0000380F8253080F8263098BF1370E3
:1096D0002B7856F8232004461146980021B1B94250
:1096E0002BD001444968F9E7D2B993B9194A1A490C
:1096F000136843F08063136052F8043C23F0804306
:1097000042F8043C152006F00FFB144B4FF40012F6
:109710001A602B78124A46F8237042F8234005E07D
:109720009B00D1184A68002AFBD14F602B7804EBCC
:1097300083020021516084F8243001332B702046CD
:10974000F8BD00BF0482FF1FFCA901006D9DFF1F33
:109750002C9DFF1F04700440E189000000E100E03F
:109760004C9DFF1F2DE9F04117462A4A2A4B036002
:109770000E461178294DFF2380F8243006294FF03A
:10978000000398BF13702978254A80F8253080F8A7
:10979000263052F82130044690468AB018468A0096
:1097A00020B1B0422BD010444068F9E7D3B991B949
:1097B0001C4A1D49136843F08063136052F8043C4F
:1097C00023F0804342F8043C152006F0ADFA174B15
:1097D0004FF400121A602B78154A48F8236042F8BB
:1097E000234005E089005A185368002BFBD15660CE
:1097F0002B7804EB83020021516084F82430394631
:109800006846FFF751FF6846FFF794F920460AB013
:10981000BDE8F0810482FF1FFCA901006D9DFF1FC0
:109820002C9DFF1F04700440E189000000E100E06E
:109830004C9DFF1F2DE9F04717462D4A0E469946CD
:1098400011782C4B0360FF2380F8243006294FF059
:10985000000398BF1370284A80F8253080F826301E
:109860000446264B107853F820109A468AB00D46CD
:109870009046830025B1B5422DD01D446D68F9E7AF
:10988000D9B990B91E4A1F49136843F08063136029
:1098900052F8043C23F0804342F8043C152006F0C3
:1098A00043FA194B4FF400121A6098F80030174A27
:1098B0004AF8236042F8234005E080000B185968FD
:1098C0000029FBD15E6098F8003004EB8302002190
:1098D000516084F824304A4639466846FFF742FF13
:1098E0006846FFF727F920460AB0BDE8F08700BFB9
:1098F0000482FF1FFCA901006D9DFF1F2C9DFF1F0F
:1099000004700440E189000000E100E04C9DFF1F6D
:109910002DE9F84FDFF8E480DFF8E4A02A4F2B4868
:109920002B4E2C4B036000254FF0FF094246514659
:109930004FF0010B80F8249080F8255080F82650D5
:109940000BF034FE87F82550234B87F824904246CD
:109950002249234C3B60384687F826B00BF026FEA0
:10996000204B214986F8255042463046336086F820
:10997000249086F826B086F825B00BF017FE1B4B16
:1099800023601B4B84F82550E5622563656384F8EA
:10999000385084F839501D806585164D164984F875
:1099A00024904246204684F826B00BF0FFFD224664
:1099B00031463B462846FFF73DFF42465146284682
:1099C000BDE8F84F0BF0F2BD689BFF1FD89AFF1F50
:1099D000009BFF1FFCA90100C8AF0100898B00009C
:1099E000289BFF1FF0AF01009D8B0000DCAF010042
:1099F000789DFF1FB09AFF1FB18B0000B08CFF1F36
:109A0000358B000037B5457B00920B462A4601692D
:109A100004F0A1F803B030BD13B501234FF0000EE0
:109A2000447B8DE8084013460069CAB2214604F021
:109A3000A7F802B010BD0368C9B21B6818470069D7
:109A400004F0B6B883685B428360704770B50D461A
:109A500006460849006814460BF09CF930602868F7
:109A600004490BF097F92860206802490BF092F93D
:109A7000206070BDE02E654270B5064608460AF0CB
:109A8000CDFC04460D4630460AF0C8FC22462B4663
:109A900008F066FD0BF020F870BDFFFF70B50728D9
:109AA00088B006460DD8084D0FCD6C460FC495E81A
:109AB0000F0084E80F0008AB03EB860656F8200C75
:109AC00000E0024808B070BD88AB0100DFAB0100C8
:109AD000F8B52B4904460BF019FB20B12146294863
:109AE0000BF04EF80446284920460BF0F1FA20B15D
:109AF000204624490BF046F80446214620460BF048
:109B000049F921460BF046F90746014620460BF07D
:109B100041F921460BF03EF90646014620460BF07E
:109B200039F921460BF036F91849054638460BF04D
:109B3000E5F9014620460BF023F815490746304663
:109B40000BF0DCF9014638460BF01CF811490646CB
:109B500028460BF0D3F9014630460BF011F82946A0
:109B6000064620460BF016F921460BF013F90A4978
:109B70000BF0C4F9014630460BF004F8F8BD00BF05
:109B8000DB0F4940DB0FC940DB0F49C00000C0407C
:109B90000000F04200809D450030B1482DE9F041C1
:109BA000334904460BF0B2FA20B1214631480AF09D
:109BB000E7FF0446304920460BF08AFA20B12046E0
:109BC0002C490AF0DFFF0446214620460BF0E2F85C
:109BD0008046014620460BF0DDF821460BF0DAF80E
:109BE0000746014620460BF0D5F821460BF0D2F887
:109BF0000646014620460BF0CDF821460BF0CAF888
:109C00004FF07C51054640460BF0C4F801464FF03A
:109C10007E500AF0B5FF1949804638460BF06EF9C0
:109C2000014640460AF0AEFF1549074630460BF0A4
:109C300065F9014638460AF0A3FF12490646284650
:109C40000BF05CF9014630460AF09CFF29460646B7
:109C500020460BF09FF821460BF09CF80A490BF0C8
:109C60004DF9014630460AF08BFFBDE8F08100BF98
:109C7000DB0F4940DB0FC940DB0F49C00000C0418A
:109C80000000344400801D47007C5D4A2DE9F0410E
:109C90001C688046204617460E46FFF719FF05460A
:109CA00030460BF023F829460BF074F805462046A1
:109CB000FFF774FF0646C8F100000BF017F80446E2
:109CC00038460BF013F831460BF064F829460AF0D9
:109CD00059FF014620460BF011F90AF0B1FB08F0DC
:109CE000EBF90AF0F9FEBDE8F081FFFF2DE9F74F2F
:109CF000061D0C4605460021304690461F4607F0DB
:109D000033FF2046FFF74AFF82464046FFF746FFF3
:109D1000014650460BF03EF801902046FFF7D8FE72
:109D2000014604460BF036F881464046FFF7D0FE68
:109D3000014683460BF02EF851460BF02BF85146A6
:109D40000BF028F849460AF01DFF0AF079FB08F0ED
:109D500089FC0AF0C1FE0AF073FB019B804689462C
:109D600018460AF06DFB42464B4608F0F9FB0AF034
:109D7000B3FE36490BF00EF8014635480AF000FFF5
:109D80003249286038460BF005F8002107460BF0F1
:109D9000A9F920B92F4938460BF0AEF918B12E4970
:109DA000304607F076FF594650460AF0F3FF0AF0B6
:109DB00047FB8046894604F100400AF041FB4246D9
:109DC0004B4608F0CDFB0AF087FE20490AF0E2FF7F
:109DD000002104460BF07CF920B120461D490AF011
:109DE000D1FE04461D4920460BF088F80BF0AEF971
:109DF0001B4C1A490440002CBCBF04F1FF3464F032
:109E000007043846B8BF01340BF078F80BF09EF920
:109E1000134B0340002BBEBF03F1FF3363F0070376
:109E2000013323440E48023318400028BEBF00F11E
:109E3000FF3060F007000130FFF730FE014630468A
:109E400007F027FF284603B0BDE8F08FE02E6542FB
:109E50000000B4420000B443F9AB010000003442FA
:109E60000700008038B5C4B20021204605F0F8FF95
:109E70004FF44865204605F0E5FF2B46013BFDD138
:109E80000028F7D038BD7047F8B54FF47A75002434
:109E9000232005F0D1FC013D0444F9D1164B4FF4C9
:109EA0007A7094FBF0F01860144B1D680AF01EFFE6
:109EB000D5F88C60D5F89070D5F8945004460146DA
:109EC00030460AF067FF21460AF064FF0C490BF0A8
:109ED00015F83946064620460AF05CFF0146304632
:109EE0000AF050FE29460AF04DFE06490BF006F82E
:109EF000054B18602046F8BD3498FF1FBC8CFF1F2F
:109F0000286B6E4E00007A448C97FF1F38B50446CC
:109F1000101E0D4607DD0AF0E9FE0F4BA1B21860D6
:109F2000F6F766FC05E0404240F6FF739842A8BF92
:109F3000184601462046F6F7A7FAF6F7C7FA074B88
:109F40001A5D074B53F83230012283F880202846EF
:109F5000BDE8384006F022B93C99FF1FD4AB0100A0
:109F600038B00100044B1B6893F86C31012B14BF0F
:109F70004FF07E5001487047BC8CFF1F000080BF2F
:109F80002DE9F04F89B04D4D1423834691FBF3F337
:109F90004FF0000A00930024009A1FFA8AF39A42B5
:109FA00040F38880464BB3F90030012B02D1454B7A
:109FB00018684DE0444BDFF83C911A68DFF83881AF
:109FC000424F0192D9F80020414E0292D8F8002069
:109FD00003923A6829680492012032680791059239
:109FE0001C6006932C60C9F80040C8F800403C6033
:109FF0003460F6F761FC069B364AD3F800C0C2F81D
:10A0000000C0304AD5F800C0C2F800C0324AD9F8C2
:10A0100000C0C2F800C0314AD8F800C0C2F800C081
:10A020002F4AD7F800C0C2F800C02E4AD6F800C0A8
:10A03000C2F800C0019A1A60029BC9F80030039B65
:10A04000C8F80030049B07993B60059B296033608A
:10A050001FFA8BF1F6F7CCFB01465846F6F714FAD7
:10A06000F6F734FA204B13F80B20204B53F832301C
:10A07000012283F88020142006F090F8FFF704FFF7
:10A080000746FFF76FFF1A4B1B680646B3F86801D7
:10A0900080B20AF02BFE014638460AF071FD3146C7
:10A0A0000AF078FE00210AF1010A0BF011F80028ED
:10A0B0003FF472AF09B0BDE8F08F00BF3C99FF1FBD
:10A0C0008097FF1F7C99FF1F3096FF1F5C97FF1F33
:10A0D0007497FF1F4C99FF1F7099FF1FF096FF1F89
:10A0E0008897FF1FD497FF1FD4AB010038B0010041
:10A0F000BC8CFF1F3099FF1F4899FF1F2DE9F04FBF
:10A10000494D89B082468B464FF0000900241FFA62
:10A1100089F39B4540F38580444BB3F90030012B14
:10A1200002D1434B18684BE0424A2B6800931368F6
:10A130000193414BDFF82C811968404F404E02914A
:10A14000D8F8001003913968049101203168059115
:10A15000146007921C6006932C60C8F800403C60B5
:10A160003460F6F7A9FB079A3649D2F800C0C1F867
:10A1700000C02F49D5F800C0069BC1F800C0324985
:10A18000D3F800C0C1F800C03049D8F800C0C1F809
:10A1900000C02F49D7F800C0C1F800C02D49D6F83B
:10A1A00000C0C1F800C00099296001991160029AAD
:10A1B0001A60039BC8F80030049B3B60059B33602A
:10A1C0001FFA8AF1F6F714FB01465046F6F75CF9E0
:10A1D000F6F77CF9204B13F80A20204B53F8323065
:10A1E000012083F8800005F0D9FFFFF74DFE0746F8
:10A1F000FFF7B8FE1A4B1B680646B3F86A0180B237
:10A200000AF074FD014638460AF0BAFC31460AF0FD
:10A21000C1FD002109F101090AF078FF00283FF48F
:10A2200076AF09B0BDE8F08F3C99FF1F8097FF1F04
:10A230007C99FF1F3096FF1F3099FF1F5C97FF1F0F
:10A240007497FF1F4C99FF1F7099FF1FF096FF1F17
:10A250008897FF1FD497FF1FD4AB010038B00100CF
:10A26000BC8CFF1F4899FF1F2DE9F0410446144E96
:10A27000642005F093FF0A2594FBF5F50024A3B2B2
:10A280009D421BDDFFF76EFE0746FFF7FDFD3368BD
:10A290008046B3F86A0180B20AF028FD01464046C4
:10A2A0000AF06EFC39460AF075FD002101340AF00F
:10A2B0000FFF18B90A2005F071FFE0E7BDE8F08153
:10A2C000BC8CFF1F2DE9F0410446144E642005F0BC
:10A2D00065FF0A2594FBF5F50024A3B29D421BDD22
:10A2E000FFF7D2FD8046FFF73DFE33680746B3F81F
:10A2F000680180B20AF0FAFC014640460AF040FCD0
:10A3000039460AF047FD002101340AF0FFFE18B972
:10A310000A2005F043FFE0E7BDE8F081BC8CFF1F99
:10A320002DE9F04F91B00746101E0D461E46DDF890
:10A330006C8001DA414206E08CB20AF0D7FC21467B
:10A34000F6F756FA01462846F6F79EF8F6F7BEF8F5
:10A35000701E002101F09AF80A2005F01FFF1A9ED6
:10A36000DFF880B14FF0400A76010DF10A094FF68F
:10A37000FF7453464FF4FA42013AFDD172B6504988
:10A38000504A485D52F830004FF0010E80F880E0EE
:10A3900020200138FDD11020CBF80030CBF8000090
:10A3A00016B130460138FDD1495D52F83120032CF9
:10A3B0004FF0010182F800110DD8132106A8019376
:10A3C00001F002F94FF07C52132106A8FEF7C6FCFB
:10A3D000019BA9F8000062B601343B4AA4B21021E7
:10A3E000042C116009F10209C2F800A0C2D1214673
:10A3F0004FF07C5203A8FEF7B1FC0AF073FC1C9BE3
:10A40000324C002B206009DD3148FEF799F92068B5
:10A410000221FEF7F3F92F48FEF72CFAB8F1010FED
:10A4200016D14FF07C52042103A8FEF797FC0AF0E6
:10A4300059FC2060054638460AF058FC264C014677
:10A4400028460AF05BFD21680AF09CFB206034E09E
:10A45000B8F1020F17D14FF07C52042103A8FEF788
:10A460007DFC0AF03FFC1D4B1B4C1860054638462E
:10A470000AF03CFC014628460AF040FD61680AF0FB
:10A4800081FB606019E0B8F1030F16D14FF07C52E8
:10A49000042103A8FEF762FC0AF024FC104B0E4CCA
:10A4A0001860054638460AF021FC014628460AF0A5
:10A4B00025FDA1680AF066FBA06011B0BDE8F08F31
:10A4C000D4AB010038B00100C4F00F402099FF1F49
:10A4D00013AC010097A201004497FF1F2499FF1FAE
:10A4E0002899FF1FC8F00F40054B1B685A680123CD
:10A4F00003FA00F0104214BF18460020704700BF56
:10A50000BC8CFF1F072810B510D8094B1B6801220F
:10A510005C68824024EA0202814011435A689142F9
:10A52000044A18BF59601378DB07FCD510BD00BF83
:10A53000BC8CFF1F01000240124B1B68B3F868116E
:10A54000B3F86A2189B292B2914293F86C210DD985
:10A55000012A16D093F86C21012A1CBF012283F82E
:10A560006C21094A1378D907FCD570474AB193F892
:10A570006C2112B1002283F86C21034A1378DB07A7
:10A58000FCD57047BC8CFF1F010002402DE9F04F45
:10A5900089B000210590072005F062FC0021082009
:10A5A00005F05EFC00240026A346A246254629218C
:10A5B000A74803F000F88321A548FFF73CFAFF21E4
:10A5C000A348FFF738FA00220121A148FFF71AFA41
:10A5D00029219F4802F0EFFF81219D48FFF72BFAC8
:10A5E00070219B48FFF727FA002201219848FFF7C6
:10A5F00009FA2921964802F0DEFF8F219448FFF7DF
:10A600001AFA01219248FFF716FA00220121904818
:10A61000FFF7F8F9052005F0C1FD29218C4802F06B
:10A62000CAFF80218A48FFF706FA03218848FFF70E
:10A6300002FA002201218648FFF7E4F92921844823
:10A6400002F0B9FF052005F0A9FD94218048FFF72D
:10A65000F2F9002201217E48FFF7D4F901222921D5
:10A660007B48FFF7D9F97A48FFF7E9F929218146B4
:10A67000774802F0A0FF95217548FFF7DCF900222A
:10A6800001217348FFF7BEF9012229217048FFF725
:10A69000C3F96F48FFF7D3F9292106906C4802F0FF
:10A6A0008AFF96216A48FFF7C6F90022012168480F
:10A6B000FFF7A8F9012229216548FFF7ADF96448A1
:10A6C000FFF7BDF929210090614802F074FF97213E
:10A6D0005F48FFF7B0F9002201215D48FFF792F9CA
:10A6E000012229215A48FFF797F95948FFF7A7F99E
:10A6F00029210390564802F05EFF98215448FFF745
:10A700009AF9002201215248FFF77CF90122292100
:10A710004F48FFF781F94E48FFF791F9292104903E
:10A720004B4802F048FF99214948FFF784F900227D
:10A7300001214748FFF766F9012229214448FFF724
:10A740006BF94348FFF77BF929218046404802F026
:10A7500032FF9A213E48FFF76EF9002201213C4862
:10A76000FFF750F9012229213948FFF755F93848F8
:10A77000FFF765F929210746354802F01CFF9B21A8
:10A780003348FFF758F9002201213148FFF73AF921
:10A79000012229212E48FFF73FF92D48FFF74FF9F5
:10A7A000012E079056DD069B18460AF09BFA4FF0E3
:10A7B00087410AF0EFFA069048460AF093FA069BA2
:10A7C000014618460AF0DEF9014620460AF0DAF999
:10A7D000044603980AF086FA4FF087410AF0DAFA45
:10A7E000814600980AF07EFA014648460AF0CAF906
:10A7F000014628460AF0C6F9054640460AF072FAB4
:10A800004FF087410AF0C6FA804604980AF06AFAC7
:10A81000014640460AF0B6F9014650460AF0B2F940
:10A82000079A824610460AF05DFA4FF087410AF017
:10A83000B1FA804638460AF055FA014640460AF019
:10A84000A1F9014658460AF09DF9834602E000BF8F
:10A85000E09CFF1F01360C2E7FF4A9AE2020F6F7F6
:10A86000A1FDCDE900010020F6F79CFD06460F464C
:10A87000284609F0E5FD32463B4609F035FE06461E
:10A8800008200F46F6F78EFD80468946504609F0AF
:10A89000D7FD42464B4609F027FE32463B4609F0BB
:10A8A00071FC064610200F46F6F77CFD804689466F
:10A8B000584609F0C5FD42464B4609F015FE3246A2
:10A8C0003B4609F05FFC064618200F46F6F76AFD86
:10A8D00080468946204609F0B3FD42464B4609F0C2
:10A8E00003FE32463B4609F04DFCDDE9002309F04A
:10A8F000FBFD064628200F46F6F754FD0B460246A0
:10A900003946304609F03EFC059B012B06460F46B2
:10A9100037D12148FDF714FF204928460AF0EEFA06
:10A920000221FDF76BFF1E48FDF70AFF1B49504649
:10A930000AF0E4FA0221FDF761FF1948FDF700FF74
:10A94000164958460AF0DAFA0221FDF757FF144873
:10A95000FDF7F6FE114920460AF0D0FA0221FDF774
:10A960004DFF0F48FDF7ECFE394630460AF0B4F8CB
:10A970000A490AF0C3FA0221FDF740FF0948FDF732
:10A98000DFFE394630460AF0A7F804490AF0B6FA65
:10A9900009B0BDE8F08F00BF24AC010000002041E9
:10A9A00097A2010077A601002DE9F04F002485B0A1
:10A9B00083460E4691469A4627464FF00008B44219
:10A9C0003ADA5BF82450374928460AF09FFB002802
:10A9D00030D0354928460AF07BFB58B30021284681
:10A9E0000AF06CFB30BB0246034694420DDD5BF877
:10A9F00022100393284602920AF060FB029A039BFE
:10AA0000002818BF01230132EFE79BB91A46B34271
:10AA10000CDA5BF823100392284602930AF04EFBEF
:10AA2000029B039A00B101320133F0E79742BCBFA9
:10AA30001746A8460134C2E71C48FDF781FE484688
:10AA4000FDF7F4FEB74201D1194818E0022F15DDD9
:10AA50001848FDF775FE0025B54212DA404609F0A8
:10AA6000EFFC5AF8254002460B4609EB0400F6F7C6
:10AA7000CBFC0A2005F092FB0135EDE70E48FDF70F
:10AA80005FFE404609F0DCFC0523024600930B48BC
:10AA90000B4606F061FF0A48FDF752FE002005B0A4
:10AAA000BDE8F08F000020C10000204180A101001E
:10AAB0002DAC010031AC010035AC01005893FF1FF3
:10AAC0007CB701002DE9F0411C4C0FCC90B00AADD1
:10AAD0000FC594E80300083485E803000FCC6D46E9
:10AAE0000FC5236816482B60FDF72AFE00250DF1DF
:10AAF000280805AE00245DF8240058F82570384475
:10AB0000F6F750FC09F0E8FF46F824000134052C64
:10AB1000F1D16B463A4621463046FFF745FF052DF9
:10AB200002D00848FDF70CFE0135062DE2D106489B
:10AB3000FDF706FE10B0BDE8F08100BFA8AB010034
:10AB40003AAC010097A2010077A6010070B50C4C49
:10AB500005460E462046D02102F02DFD290A20464A
:10AB6000F6F784FAE9B22046F6F780FA3146204635
:10AB7000F6F77CFA002201212046FEF743FF70BD64
:10AB8000E09CFF1F38B50F4C0546D021204602F04F
:10AB900012FD290A2046F6F769FAE9B22046F6F7CF
:10ABA00065FA002201212046FEF72CFF0122D02168
:10ABB0002046FEF731FF2046FEF741FF20EAE07015
:10ABC000C0B238BDE09CFF1F08B58020FFF7DAFF58
:10ABD000012803D1BDE80840FFF7D8BC0248BDE812
:10ABE0000840FDF7ADBD00BF4DAC010070B50C4C89
:10ABF00005460E462046D12102F0DDFC290A2046FA
:10AC0000F6F734FAE9B22046F6F730FA3146204634
:10AC1000F6F72CFA002201212046FEF7F3FE70BD64
:10AC2000F49CFF1F38B5114C0546D121204602F097
:10AC3000C2FC290A2046F6F719FAE9B22046F6F7CF
:10AC400015FA002201212046FEF7DCFE0122D12167
:10AC50002046FEF7E1FE052005F0A0FA2046FEF7AB
:10AC6000EEFE20EAE070C0B238BD00BFF49CFF1FCA
:10AC7000062810B5044610D803F00AFD094B1B68DE
:10AC800003EB8403D3F834239042074A18BFC3F878
:10AC900034031378DB07FCD510BD0448BDE8104031
:10ACA000FDF74EBDBC8CFF1F0100024066AC0100E9
:10ACB00038B50D480D4DFDF743FD00242B6804F118
:10ACC000CC0203EB820301345868FDF7AFFD08485E
:10ACD000FDF736FD072CF1D10648FDF731FD06489A
:10ACE000BDE83840FDF72CBD6CAC0100BC8CFF1FEB
:10ACF00097A2010047AB010077A6010038B50D48C7
:10AD00000D4DFDF71DFD002455F824000121FDF730
:10AD100075FD01340948FDF713FD092CF4D1064BEC
:10AD20000121586AFDF76AFD0548BDE83840FDF786
:10AD300007BD00BF79AC01000498FF1F97A2010076
:10AD400077A6010038B50D480D4DFDF7F9FC00243C
:10AD500055F824000121FDF751FD01340948FDF7A4
:10AD6000EFFC052CF4D1064B01215869FDF746FD97
:10AD70000548BDE83840FDF7E3BC00BF8CAC0100DE
:10AD8000B497FF1F97A2010077A6010013B5012019
:10AD90000AF0C2FC04460AF0C7FC01A8001B02B07E
:10ADA00010BD70B5044608460E460AF0A7FF0546DA
:10ADB00020460AF0A3FF28442044002343706A423F
:10ADC000A04201D1002303E0835C00F80139F7E7DA
:10ADD000AB4203DAF25CE2540133F9E770BD70B5BF
:10ADE000054608460E460AF089FF044628460AF042
:10ADF00085FF33462A18991B8C4204DD13F8011B8A
:10AE000002F8011BF7E72C440023235470BDFFFF19
:10AE10002DE9F04F431E092B85B00646884615469E
:10AE200000F2EE80002140460AF052F90446002864
:10AE300040F0E6807548FDF783FC2846FDF7F6FCF8
:10AE40007348FDF77DFC3046FDF7F0FC7148FDF7D7
:10AE500077FC21464046FDF7D1FC6E48FDF770FCBB
:10AE600032250B24A946DFF8BCA1DFF8BCB1294686
:10AE70003046F5F709FBF5F729FB1AF806305BF8C1
:10AE80003330012283F88020052005F087F9002067
:10AE9000FFF77CFB052005F081F90020FFF776FB2A
:10AEA000052005F07BF90020FFF770FB01460746FF
:10AEB00040460AF00DF9CDF80CB0CDF808A020B14D
:10AEC00038460AF043F9824610E0284609F00AFFA6
:10AED0004FF07F5109F05EFF0AF05EF9013CA94690
:10AEE0000546C0D14FF47A6542F2107A14230193DB
:10AEF0004FF0000B43E040F6FF713046F5F7C4FA1F
:10AF0000F5F7E4FA029B9B5D40F6FF74039A52F852
:10AF10003330012283F88020052005F03FF900201E
:10AF2000FFF734FB052005F039F90020FFF72EFB71
:10AF3000052005F033F90020FFF728FB36490746C6
:10AF4000404609F027FF014638460AF0D5F868BBAD
:10AF5000394640460AF0DAF8002842D0584609F04F
:10AF6000C5FE014638460AF0D1F820B138460AF04D
:10AF7000EDF8A1468346019B013B019320D009EBEC
:10AF80000500401009F0B2FE0AF0E0F8B0F5805F6D
:10AF90000446B0DA0228B8BF022421463046F5F74D
:10AFA00073FAF5F793FA029B9B5DAFE71B494046A6
:10AFB00009F0F0FE014638460AF094F80028C7D0A0
:10AFC0000020FFF7E3FA0221FDF718FC1148FDF716
:10AFD000B7FB2046FDF72AFC1148FDF7B1FB2046E0
:10AFE00010E0504609F082FE014638460AF070F83B
:10AFF0000028C0D038460AF0A9F825468246BAE7AC
:10B000004FF0FF3005B0BDE8F08F00BFA4AC0100E9
:10B01000579C010097A201009A99593F3333933FFF
:10B0200077A60100D4AB010038B001002DE9F84F3C
:10B030001546002299460646FFF7EAFE01222946F8
:10B0400004463046FFF7E4FE002107463046F5F798
:10B050001BFAF5F73BFA2E4B2E4D13F8068055F8E8
:10B060003830012283F800214FF4C87005F096F8BB
:10B070002948FDF765FB3F1B97FBF9FA002709F10B
:10B0800001039F4233DC21463046F5F7FDF9F5F721
:10B090001DFA55F83830012283F880201E2005F073
:10B0A0007DF80020FFF772FA1E2005F077F80020E7
:10B0B000FFF76CFA142005F071F80020FFF766FA2C
:10B0C00083461648FDF73CFB2046FDF7AFFB1448CE
:10B0D000FDF736FB58460AF039F8FDF7A7FB4F4558
:10B0E00002DC1048FDF72CFB01375444C7E730461B
:10B0F0000021F5F7C9F9F5F7E9F955F838300A48AC
:10B10000012283F80021BDE8F84FFDF719BB00BF0D
:10B11000D4AB010038B00100B1AC010080A1010046
:10B1200097A2010077A601005B9C010070B5044660
:10B130000120F5F7C1FBA1B20646F5F759FB014620
:10B1400005462046F5F7A0F9F5F7C0F9114B1A5D51
:10B15000114B53F83230012283F88020322005F061
:10B160001DF80E48FDF7ECFA20460D4CFDF75EFB8E
:10B170002046FDF7E5FA02213046FDF73FFB204669
:10B18000FDF7DEFA2846FDF751FB0648BDE87040A2
:10B19000FDF7D6BAD4AB010038B00100C2AC010053
:10B1A00097A2010077A60100F8B507460E460025D4
:10B1B0000024B5420BDA384600F0F8F909F096FDA4
:10B1C0000146204609F0DEFC01350446F1E7304631
:10B1D00009F08CFD0146204609F090FEF8BDFFFF06
:10B1E0002DE9F0410646C820F6F7DCF809F074FCBA
:10B1F0008046D020F6F7D6F809F06EFC0025074609
:10B200000024B54211DA01210620FFF7CDFF0146E7
:10B21000404609F0BFFD394609F0B2FC0146204620
:10B2200009F0B0FC01350446EBE7304609F05EFD5D
:10B230000146204609F062FE04460648FDF780FA02
:10B2400020460221FDF7DAFA0348BDE8F041FDF798
:10B2500077BA00BFCDAC010097A2010010B5074C32
:10B26000072201212046522303F018FB2046044AFE
:10B270000449BDE810400AF099B900BF789CFF1F4F
:10B28000B08CFF1FC1E7000070B5602105460C4877
:10B2900002F091F92E120424EDB231460848FEF76F
:10B2A000CAFB013C2946064801F064FE14F0FF0485
:10B2B000F3D1224601210248FEF7A4FB70BD00BF76
:10B2C000E09CFF1F88B2FFF7DFBFFFFFF8B506461F
:10B2D0003248FDF735FA14273224204609F006FDDE
:10B2E0002F4909F057FD09F031FF044680B2FFF7FE
:10B2F000CBFF002004F052FF0020FFF747F9314652
:10B30000054609F003FF08B9013FE6D11427294695
:10B31000304609F0DDFE08B1224D01E04FF07E55C8
:10B32000204609F0E3FC294609F02CFC09F00EFF49
:10B33000044680B2FFF7A8FF642004F02FFF00202E
:10B34000FFF724F918490546304609F023FD014668
:10B35000284609F0DBFE40B11449304609F01AFDD9
:10B360000146284609F0B4FE08B9013FCFD10221B9
:10B370003046FDF743FA0E48FDF7E2F90221284670
:10B38000FDF73CFA0A48FDF7DBF92046FDF74EFAD7
:10B390000848BDE8F840FDF7D3B900BFD8AC0100BC
:10B3A0009A99993F000080BF3333733F6666863FAA
:10B3B00097A2010077A60100C37A10B5E3B172B677
:10B3C000C37ADC0705D5134AC36814682340836138
:10B3D0001360C37A9A0705D50F4A0369146823409E
:10B3E000C3611360C37A5B0705D50C4A43691468CF
:10B3F00023400362136062B60368DA688A4207D0AA
:10B40000074A1A60D960074A41F0804119611A6001
:10B4100010BD00BF80E100E084E100E088E100E0D1
:10B4200001403F0000003F8003684FF00042DA62B5
:10B430005963DA6A002AFCDA986BC0B27047036875
:10B440004FF0004241F08051DA625963DA6A002A13
:10B45000FCDA986B80B27047C37A83B1D90742BFD8
:10B46000074B82691A60C37A9A0742BF054BC269CB
:10B470001A60C37A5B0742BF034B026A1A607047C7
:10B4800000E100E004E100E008E100E0082888BFF6
:10B49000002038B50828234C13BFC0014FF43053A7
:10B4A000238040F47050204B18BF20801A682388F6
:10B4B00043EA82139B0001211620238004F0D0FC74
:10B4C0001A4B1B481968FFF777FF0021162004F07C
:10B4D00099FC25881648290AFFF7A6FFE9B2144807
:10B4E000FFF7A2FFC0250121162004F08BFC2B469C
:10B4F000013BFDD10021162004F084FC24880C4877
:10B50000210AFFF791FFE1B20948FFF78DFF012102
:10B51000162004F077FC013DFDD10548FFF79CFFA4
:10B5200038BD00BF8C9CFF1FCC97FF1F909CFF1F56
:10B530000C92FF1F024A0223136042F8043C70473A
:10B5400088F00F402DE9F041A0252B46013BFDD1AD
:10B55000114E124B30461968FFF72EFF104B022791
:10B560001F60104BB3F8008030464FEA1821FFF7F8
:10B570005BFF000284B25FFA88F13046FFF754FFA8
:10B58000094B204384B21F60013DFDD13046FFF7D7
:10B5900063FF2046BDE8F0810C92FF1F909CFF1FC7
:10B5A00088F00F408C9CFF1F84F00F4008B50021ED
:10B5B000FFF76CFFFFF7BEFF6023013BFDD1BDE845
:10B5C0000840FFF7BFBFFFFF144B2DE9F04780464F
:10B5D000894613481968134E134FDFF850A0FFF740
:10B5E000EBFE6FF001044C4513DA02253560BAF822
:10B5F00000103D600A483560FFF721FF002C3D60D8
:10B600004FF06003A8BF28F81400013BFDD10134BE
:10B61000E9E70348FFF720FFBDE8F087909CFF1F94
:10B620000C92FF1F88F00F4084F00F408C9CFF1F8E
:10B630002DE9F74F1E462E4B019119682D4DDFF86D
:10B64000C0B0890109B241F400539BB243F4E05306
:10B6500043EAC01000B2284B80B241EA80076FEA8B
:10B660004272196825486FEA1259FFF7A5FE3FB2EA
:10B67000BFB21FFA89F96FF00104AA460C9B9C42E5
:10B6800030DA4FF00208C5F800803946CBF8008068
:10B690001A48C5F80080FFF7D2FE002C4146A8BF2B
:10B6A000019BDFF85C80A8BF23F81400C8F80010E5
:10B6B00060200138FDD11148CAF80010C8F8001008
:10B6C000CAF800104946FFF7BAFE002C4FF00201FD
:10B6D000A8BF26F81400C8F8001060210139FDD178
:10B6E0000134CBE70548FFF7B7FE03B0BDE8F08FA4
:10B6F000CC97FF1F88F00F40909CFF1F0C92FF1FFC
:10B7000084F00F40014B024A1A607047909CFF1F63
:10B71000000001B837B50025447B8DE828001346AA
:10B7200000690A46214602F02BFAC0B203B030BDD0
:10B73000F0B5002A134E144F14BF4FF060544FF071
:10B740006454002236F8125097FBF5F5A94204D351
:10B75000190707D544F0806404E0551C172DF7D075
:10B760002A46EFE709495B0751F8222007D522F462
:10B770007043120902F4706244F000741A432243C9
:10B780000260F0BDB0AE0100006CDC02E0AE010072
:10B7900010B50446FFF7CCFF204610BDFF22027310
:10B7A00042738273C27370472DE9F04190F90F30F4
:10B7B000013305460F460CD1164B1B684FF0004273
:10B7C000DA625963DA6A002AFCDA986BC0B2BDE823
:10B7D000F081072600244FF001080021E87B04F0E7
:10B7E00011FB08FA06F13940687B04F00BFBE87B9B
:10B7F0000121640004F006FBA87BE4B204F022FB04
:10B8000008B144F0010416F1FF36E6D22046BDE847
:10B81000F08100BF0C92FF1F73B590F90C3001331B
:10B8200004460E46154611D101781C4801F0C3FEAE
:10B8300031461A4801F09EFB2946184801F09AFB50
:10B84000002201211548FEF7DDF825E090F90F30C0
:10B85000013309D112490023012201A8FFF798FF03
:10B8600001991048FFF7A8FD0021207B04F0CAFAD7
:10B8700006F07F012046FFF797FF29462046FFF795
:10B8800093FF0121207B04F0BDFA94F90F300133BE
:10B8900002D10448FFF7E0FD02B070BDF49CFF1F29
:10B8A00020A107000C92FF1F73B590F90C300133F3
:10B8B00004460E4618D1214D0178284601F07BFE42
:10B8C0003146284601F056FB002201212846FEF7AA
:10B8D00099F801231A4621782846FFF71BFF2869AB
:10B8E00002F066F9C5B226E090F90F30013309D1B4
:10B8F00013490023012201A8FFF74AFF01991148CB
:10B90000FFF75AFD0021207B04F07CFA46F080010D
:10B910002046FFF749FF00212046FFF745FF0121A0
:10B920000546207B04F06EFA94F90F30013302D102
:10B930000448FFF791FD284602B070BDF49CFF1F3C
:10B9400020A107000C92FF1F73B590F90C30013352
:10B9500005460C461ED1284E0178304601F02BFEDC
:10B960002146304601F006FB002201213046FEF759
:10B9700049F80123022229783046FFF7CBFE3069CF
:10B9800002F016F90446306902F012F940EA042088
:10B9900084B22DE090F90F30013309D1174900230B
:10B9A000012201A8FFF7F4FE01991548FFF704FDF5
:10B9B0000021287B04F026FA44F080012846FFF796
:10B9C000F3FE00212846FFF7EFFE0021044628463B
:10B9D000FFF7EAFE40EA042084B20121287B04F04C
:10B9E00011FA95F90F30013302D10548FFF734FD04
:10B9F000204602B070BD00BFF49CFF1F20A10700CD
:10BA00000C92FF1F08B5FFF79FFF40BA80B208BD38
:10BA100038B588210446FFF7F5FF8A2120822046A9
:10BA2000FFF7F0FF8C2160822046FFF7EBFF8E21AD
:10BA3000A0822046FFF7E6FF9021E0822046FFF734
:10BA4000E1FF922120832046FFF7DCFF94216083F1
:10BA50002046FFF7D7FF9621A0832046FFF7D2FFAD
:10BA60009821E0832046FFF7CDFF9A2120842046CD
:10BA7000FFF7C8FF9C2160842046FFF7C3FF9E218B
:10BA8000A0842046FFF7BEFFA121E0842046FFF7F7
:10BA90000BFFE12184F828002046FFF7B3FFE321E4
:10BAA00060852046FFF700FFE42184F82C00204643
:10BAB000FFF7FAFEE52105462046FFF7F5FE00F008
:10BAC0000F0040EA0510E085E6212046FFF7ECFE76
:10BAD000E52105462046FFF7E7FE001140EA051084
:10BAE0002086E7212046FFF7DFFE84F8320038BDCC
:10BAF00010B50446017090F90C00421C1BD00121C6
:10BB0000C0B204F07FF9207B012104F0A9F994F977
:10BB10000F00431C03D1134802F0DAFB0BE00121B4
:10BB2000C0B204F09DF90121607B04F099F9002175
:10BB3000A07B04F095F9D0212046FFF7B5FE6028E0
:10BB40000ED12046FFF764FF20460522F221FFF7C1
:10BB500063FE2046B722F421FFF75EFE012010BDF0
:10BB6000002010BD0C92FF1F73B590F90C3001330B
:10BB700005460C4621D12B4E0178304601F01BFDC5
:10BB80002146304601F0F6F9002201213046FDF74A
:10BB900039FF0123032229783046FFF7BBFD3069C6
:10BBA00002F006F80402306902F002F820430402B1
:10BBB000306901F0FDFF044331E090F90F300133AB
:10BBC00009D119490023012201A8FFF7E1FD0199DC
:10BBD0001648FFF7F1FB0021287B04F013F944F02D
:10BBE00080012846FFF7E0FD00212846FFF7DCFD35
:10BBF000002104022846FFF7D7FD2043040200215C
:10BC00002846FFF7D1FD01210443287B04F0FAF810
:10BC100095F90F30013302D10448FFF71DFC20468F
:10BC200002B070BDF49CFF1F20A107000C92FF1F03
:10BC300010B5FA210446FFF797FF228AC2EB2023B2
:10BC40005200C2EBE010B4F912205B435043B4F948
:10BC500014201B1353439B1303EBE020A06000EB65
:10BC600080008030001209F041F8024909F046F9DD
:10BC700010BD00BF0000C84210B50446FFF7D8FF52
:10BC8000FD212046FFF760FEB4F92E30A268B4F91A
:10BC900030101B05A2F59632C3EB803002FB110079
:10BCA00000F58043D81394F82C3094F932105343A4
:10BCB000DB124A43921203F5004353439B12B4F93B
:10BCC0002A2003F50013534303F500539B1343430A
:10BCD000D81394F828204043C0115043A3EB201000
:10BCE00020EAE070B0F1C85FA8BF4FF0C850001361
:10BCF00008F0FCFF4FF06A5109F04CF810BD2DE937
:10BD0000F84F0646FFF794FFF7213046FFF72CFF68
:10BD1000B468B6F91820E517B4F5FA3445F1FF35E3
:10BD2000A4FB048904FB05F309EB430902FB05F1BD
:10BD3000D31704FB0311A2FB04230B44190341EAAC
:10BD4000125107461003B6F91A20D31702FB09FE59
:10BD500008FB03EEA2FB082373444FEA122A4AEAC7
:10BD6000036A1AEB000AF28A4FEA232B4BEB010B12
:10BD70001AF100004BF50041A0FB02AB02FB01BB36
:10BD80004FEA6B024FEAEB7352EA03017FD0B6F938
:10BD900020A04FEAEA7B0AFB09F108FB0B11AAFB82
:10BDA0000889B6F91EA089444FEAEA7B0AFB05F12F
:10BDB00004FB0B11AAFB04450D444FEA454B4FEA27
:10BDC000444A38111AEB080AC0F580104BEAD43BFC
:10BDD0004BEB090B4FEAE0794FEAC97545EA50058C
:10BDE000C407B6F91C004FF0000818EB0A084FEA28
:10BDF000C00949EB0B0940F63547B4EB080465EB85
:10BE00000905A4FB070107FB051109F0E5F9B6F9DF
:10BE100026204C13450B45EAC14502FB04F7D31716
:10BE200005FB0377A2FB05233B44544305FB034476
:10BE3000A2FB05232344540E44EAC314B6F924207C
:10BE400024184FEA63654D41D317514300FB031398
:10BE5000A2FB00011944C20C42EA41321219B6F9A0
:10BE600022404FEAE1436B41100AE517220140EA04
:10BE7000036019122B0143EA14738018594108F02A
:10BE80004BFF4FF06E5108F085FFBDE8F88F0020A2
:10BE9000BDE8F88F80E8060012B11378022B02D0BB
:10BEA0000023036043607047036870B50E469BB182
:10BEB0004068A8B1002911DBC36899420EDA00F18D
:10BEC00010040025B54220460AD000F0ADF801303C
:10BED00004EB00140135F5E7184670BD002070BD75
:10BEE00070BD38B504460D6808461146FFF7DCFF03
:10BEF000294602462046FFF7CDFF204638BD10B543
:10BF00000446FFF7D1FF01462046BDE8104000F08F
:10BF100096B838B504460D6808461146FFF7C4FFC9
:10BF200029460246204600F016F8204638BD10B5D6
:10BF30000446FFF7B9FF01462046BDE8104000F077
:10BF40008AB810B50446FFF7AFFF01462046BDE8AA
:10BF5000104000F08BB880E8060012B11378012B76
:10BF600002D0002303604360704703682DE9F0416D
:10BF700005460F4613B3446804B3F9B110340026E4
:10BF80004FF002086B68DB6893FBF8F39E4215DA0A
:10BF90002146284600F06AF80146384609F09CFE22
:10BFA00004F1100310B91846BDE8F081184600F0FE
:10BFB0003BF8023004EB00140136E3E70020BDE853
:10BFC000F08108B5FFF7D1FF003018BF012008BD90
:10BFD00038B504460D6808461146FFF7C6FF2946E6
:10BFE00002462046FFF756FF204638BD10B50446EE
:10BFF000FFF7BBFF01462046BDE8104000F01FB828
:10C0000010B50446FFF7B1FF01462046BDE81040D9
:10C0100000F021B810B50446FFF7A7FF01462046FF
:10C02000BDE8104000F022B8826800F11003002043
:10C0300059688A4202DD10330130F9E770470B4638
:10C0400031B1097821B900685B6818440AF0C8BCAE
:10C0500000200021704739B10A782AB94B6800687E
:10C06000114618440AF068BD0020704710B561B150
:10C070000B78012B01D9032B09D102688B680024AE
:10C08000D45400684B68184410BD084610BD002009
:10C0900010BD03681B68184770B51F4C0646217811
:10C0A0001E48254601F087FA1C4C0EB1262100E0FF
:10C0B00027212046FFF7EDFF002211461748FDF724
:10C0C000A1FC296815480222FDF7A6FC206901F0B1
:10C0D0006FFD0546206901F06BFD04460022012139
:10C0E0000E482402FDF78EFC04F4FE44E8B220431F
:10C0F00008F0FCFD0A4908F04DFE08F0A1F904A380
:10C10000D3E9002308F03CF808F0E6FC70BD00BF5E
:10C110000000006066127140D48CFF1FF49CFF1F6A
:10C120000AD7A33C70B50C4C06460D4620461D218F
:10C1300001F041FA3146204600F01CFF2946204616
:10C1400000F018FF4FF47A7200212046FDF75AFCE8
:10C150004023013BFDD170BDF49CFF1F10B50E4C78
:10C160001D21204601F027FA0D21204600F002FF94
:10C170004FF47A7200212046FDF744FC4023013B36
:10C18000FDD101221D212046FDF746FC2046FDF78A
:10C1900056FCC0B210BD00BFF49CFF1F08B50021C3
:10C1A0002A20FFF7BFFF00210E20FFF7BBFF212150
:10C1B0002A20FFF7B7FFFFF7D1FF5A3818BF4FF01B
:10C1C000FF3008BD2DE9F843294C81460E46204634
:10C1D0001D21154601F0EFF90021204600F0CAFEAE
:10C1E0004FF47A7200212046FDF70CFC4023013BFE
:10C1F000FDD107221D212046FDF70EFC2046FDF74C
:10C200001EFC2046FDF71BFC07462046FDF717FCE9
:10C21000C0B240EA07231BB24FF47A774FF480484C
:10C2200013FB07F3204693FBF8F3C9F80030FDF742
:10C2300006FC81462046FDF702FCC0B240EA092315
:10C240001BB213FB07F3204693FBF8F33360FDF7B3
:10C25000F6FB06462046FDF7F2FBC0B240EA062098
:10C2600000B210FB07F797FBF8F72F60BDE8F883E3
:10C27000F49CFF1FC26000228160C270027170478F
:10C2800061F07F01017042708368024602210079EB
:10C290001847FFFF10B504460846E378A3B10B49E1
:10C2A00008F078FD08F078FF1822B0FBF2F0B0F546
:10C2B000807F024628BF4FF480722046D2B201210F
:10C2C000BDE81040FFF7DCBF10BD00BF00002041FB
:10C2D000C3780A4613B10F21FFF7D2BF704710B5DC
:10C2E00061F07F01044601708368024601210079F4
:10C2F00098472079E368224601219847207810BDAD
:10C3000038B5C5780446BDB9292303711221FFF75A
:10C31000E6FF142802D10123E3700CE01D28FAD0B7
:10C320003923237112212046FFF7D9FF1428F2D0B8
:10C330001D28F0D02571E578284638BD38B504466B
:10C34000FFF7DEFFE578C5B100212046FFF7C7FF04
:10C3500040F00102D2B200212046FFF791FF0320F6
:10C3600003F01CFF00212046FFF7B9FF40F0020256
:10C37000D2B200212046FFF783FF284638BDFFFFD9
:10C3800038B505460846EB78D3B31E4908F002FDE0
:10C3900008F0DCFE1728044606DC00212846FFF7DB
:10C3A0009EFF00F0F70225E0B0F5C05F0CDD022231
:10C3B0000D212846FFF764FFB4F5903FA8BF4FF466
:10C3C00090344FF4907205E000220D212846FFF7CB
:10C3D00057FF182294FBF2F4C4F58072D2B2032105
:10C3E0002846FFF74DFF00212846FFF778FF40F071
:10C3F0000802D2B228460021BDE83840FFF740BF0E
:10C4000038BD00BF0000204110B561F05F01044657
:10C410000170836802460121007998472079E3681A
:10C42000224602219847208810BDC37813B11421F9
:10C43000FFF7EABF18467047C37813B11621FFF71C
:10C44000E3BF18467047C37813B11821FFF7DCBF6C
:10C4500018467047C37813B11A21FFF7D5BF1846A5
:10C460007047FFFF0346114A1148190F515C0170D4
:10C47000C3F30361515C4170C3F30351515C81709C
:10C48000C3F30341515CC170C3F30331515C0171CB
:10C49000C3F30321515C4171C3F3031103F00F0394
:10C4A000515CD35C8171C371704700BF05AD010061
:10C4B000949CFF1F024B4FF0FF321A60704700BF81
:10C4C000D88CFF1F014B1868C0437047D88CFF1FE2
:10C4D0000D4A1368F0B50546002714462A1A914202
:10C4E0000FDD15F8012B08265A40084B42F30007D0
:10C4F0003B4083EA5203013E4FF001071A46F4D154
:10C50000ECE707B12360F0BDD88CFF1F2083B8EDA6
:10C510000C4A136830B501380025114610F8012F78
:10C520006AB15A400824084B42F300052B4083EAC5
:10C530005203013C4FF001051A46F4D1EEE705B174
:10C540000B6030BDD88CFF1F2083B8ED2DE9F04F74
:10C550004FF0030C00264FF0FF3E05684C5D002CA9
:10C5600000F0FF802C2C00F0F88011D80D2C00F08A
:10C57000F48004D8093C012C00F2BF80EDE0202CAF
:10C5800000F0EB80222C40F0B8806F1C076076E052
:10C590005D2C39D005D83A2C00F0DF805B2C08D018
:10C5A000ABE07B2C05D07D2C40F0A7804FF001093B
:10C5B0002CE0D0F804904B4540F2F08009F10107DF
:10C5C000476087684FEA091BB7F1FF3F02EB0B0A90
:10C5D00018BF02EB0718CAF80C6018BFD8F80C7027
:10C5E000CAF804E018BF0137CAF808E018BFC8F855
:10C5F0000C707B2C14BF0224012402F80B40CAF8F3
:10C600000450C0F80890A8E04FF002094468013CCB
:10C6100002EB0418002C18DBD8F80470013710D096
:10C62000D8F80870B7F1FF3F0BD198F800A0CA45C1
:10C6300040F0A88001358760C8F8085002EB041765
:10C640000CE0013CA8F11008E4E7013440F08580DB
:10C6500098E0013C651CA7F110077ED07D6801358C
:10C66000F7D0BD680135F4D1846076E0B8F1220FCF
:10C670000CD0B8F15C0F1BD004680134046004686E
:10C6800011F80480B8F1000FF0D12AE0D0F804804E
:10C69000434540F2828008F101054FEA08184560E1
:10C6A00002EB080502F808C06F60AC60EE604CE079
:10C6B000013404600C5D662CDED008D82F2CDBD052
:10C6C00001D8222C07E05C2CD6D0622C03E0722C1F
:10C6D000D2D002D86E2CCFD022E0743C012CCBD922
:10C6E0001EE0056055E0202C1CD00FD8092C09D283
:10C6F000203C5E2C14D8013707600768CC5D002C05
:10C70000F1D10FE00A2C0DD90D2C07E03A2C09D0FD
:10C7100001D82C2C02E05D2C04D07D2CE8D101E066
:10C7200005602FE04468A34237D904F101082401D1
:10C73000C0F8048002EB04081655C8F80870013FE1
:10C74000C8F80450C8F80C60076085686C1C1FBFEF
:10C7500002EB0515EC680134EC60046801340460F8
:10C76000FBE641684B1E02EB0112002B0EDB52F878
:10C770000C1C013103D052F8081C013109D0013BD7
:10C78000103AF2E76FF00100BDE8F08F0020BDE83D
:10C79000F08F6FF00200BDE8F08F05604FF0FF30C2
:10C7A000BDE8F08F0023036043604FF0FF338360E8
:10C7B00070470369D3F83801D3F83431C01A704791
:10C7C00038B5124B124C1B6893F82C50EDB2294629
:10C7D000204600F0F0FE07212046FDF72CF94FF42B
:10C7E0007A7201212046FDF70DF94023013BFDD16E
:10C7F000012229462046FDF70FF9022003F0CEFC66
:10C800002046FDF71CF9C0B238BD00BFBC8CFF1F2D
:10C81000F49CFF1F38B5144B144C1B6893F82C5034
:10C820000120EDB203F0BAFC2946204600F0C3FE19
:10C8300010212046FDF7FFF829212046FDF7FBF8DF
:10C84000A0212046FDF7F7F84FF47A720121204627
:10C85000FDF7D8F8012003F0A1FCFFF7B1FFC438C1
:10C8600018BF4FF0FF3038BDBC8CFF1FF49CFF1F7A
:10C870002DE9F0413A4B1B6893F82C40E4B2804616
:10C880000F4638482146164600F095FE11213548DE
:10C89000FDF7D1F808213348FDF7CDF80A2003F061
:10C8A0007DFC21462F4800F086FE01212D48FDF732
:10C8B000C2F84FF47A7201212A48FDF7A3F8402309
:10C8C000013BFDD1062221462648FDF7A5F80023AD
:10C8D000336024483B60C8F80030FFF76AFF20B19E
:10C8E0002048FDF7ACF8C5B200E005461D48FFF74B
:10C8F00060FF20B11B48FDF7A2F8C4B200E0044677
:10C9000044EA05231BB2C8F800301648FFF751FF70
:10C9100018B11448FDF793F8C5B21248FFF749FF64
:10C9200018B11048FDF78BF8C4B244EA05231BB2D6
:10C930003B600C48FFF73DFF18B10A48FDF77FF850
:10C94000C5B20848FFF735FF18B10648FDF777F87C
:10C95000C4B244EA052424B23460BDE8F08100BFCB
:10C96000BC8CFF1FF49CFF1F70B50C4B0C4C1B685C
:10C9700006460D46204693F82C1000F01CFE31466A
:10C98000204600F0F7FA2946204600F0F3FA4FF46B
:10C990007A7201212046FDF735F870BDBC8CFF1F6F
:10C9A000F49CFF1F044B01221A70044B1B68A0214A
:10C9B00093F82C00FFF7D8BFC49CFF1FBC8CFF1F4F
:10C9C00008B1FFF7EFBF034B802118701120FFF76C
:10C9D000CBBF00BFC49CFF1F2DE9F74F484B494A0E
:10C9E0001B68156801931846294608F0CBF84FF0EC
:10C9F0007C5108F0CFF9444A1060444AD2F800B0A4
:10CA0000434AD2F800A080465146584608F0BAF88A
:10CA10004FF07C5108F0BEF93E4A10603E4AD2F811
:10CA200000903E4A146807462146484608F0AAF896
:10CA30004FF07C5108F0AEF9394A019B106019465D
:10CA40000646284608F09CF8364B054618605946BD
:10CA5000504608F095F8344B494618608246204607
:10CA600008F08EF8314B1860314B1C688146A16884
:10CA7000284608F023FB00B9A5602E4A13782D4DF7
:10CA800013F0010FFAD06169504608F017FB08B99E
:10CA9000C4F814A02B78DB07FCD5216A484608F0BF
:10CAA0000DFB08B9C4F820902B78D807FCD5E168B5
:10CAB000404608F003FB08B9C4F80C802B78D9076E
:10CAC000FCD5A169384608F0F9FA00B9A7612B78BE
:10CAD000DA07FCD5616A304608F0F0FA00B9666200
:10CAE0002B78DB07FCD50020FFF76AFF124B0022F2
:10CAF0001A70124B01221A7003B0BDE8F08F00BF0C
:10CB0000BC9CFF1FC09CFF1FB89CFF1FCC9CFF1F3D
:10CB1000D09CFF1FC89CFF1FD89CFF1FDC9CFF1FE1
:10CB2000B49CFF1FA49CFF1FAC9CFF1FA09CFF1F79
:10CB3000BC8CFF1F01000240A99CFF1FB09CFF1F7F
:10CB400070B586B001A902AA6846FFF791FE009869
:10CB50002A4C08F0CBF82168054608F0B9FA10B164
:10CB60002560012400E00446254E2846316808F07F
:10CB7000CDFA08B1356001240198224E08F0B6F8CC
:10CB80003168054608F0A4FA08B1356001241E4E4C
:10CB90002846316808F0BAFA08B1356001240298D5
:10CBA0001A4E08F0A3F83168054608F091FA08B16A
:10CBB00035600124164E2846316808F0A7FA154B57
:10CBC00008B1356000E024B11A680392124A039953
:10CBD00011601B680493049BB3F57A7F0CD90D4B4D
:10CBE0000D4A1B6805931268059B9B1A41F2883217
:10CBF000934201D9FFF7F0FE06B070BDBC9CFF1F49
:10CC0000C09CFF1FCC9CFF1FD09CFF1FD89CFF1F08
:10CC1000DC9CFF1F889DFF1FD49CFF1F38B5144B61
:10CC20001B6893F82C40E4B205462146114800F0F9
:10CC3000C2FC29460F4800F09DF94FF47A72012199
:10CC40000C48FCF7DFFE4023013BFDD101222146C9
:10CC50000848FCF7E1FE00240648FFF7AAFD20B1D2
:10CC60000448FCF7ECFEC4B2F6E7204638BD00BF2E
:10CC7000BC8CFF1FF49CFF1F08B5084B012210203D
:10CC80001A70FFF7CBFF40F00101C9B21020FFF787
:10CC90006BFE03490348FBF7BBFF08BDA89CFF1FC1
:10CCA00016AD01005893FF1F08B5064B0022102057
:10CCB0001A70FFF7B3FFBDE8084000F0FC01102038
:10CCC000FFF752BEA89CFF1F38B50D4B1C780546D8
:10CCD0000CB1FFF7E9FF642003F060FA1020FFF7C2
:10CCE0009DFF00F0070129431020FFF73DFE64205F
:10CCF00003F054FA1CB1BDE83840FFF7BDBF38BDA2
:10CD0000A89CFF1F08B5104B104901221A70104B48
:10CD1000104A1A604FF047430B600F490A600F49F1
:10CD20000B600F490A600F4A1360FFF73BFE0E4B82
:10CD300000201870FFF7C8FF0C4B1B781BB9BDE82B
:10CD40000840FFF799BF08BDA99CFF1FC09CFF1FAB
:10CD5000BC9CFF1F00FEFF46CC9CFF1FD09CFF1F0A
:10CD6000D89CFF1FDC9CFF1FB09CFF1FA89CFF1FCF
:10CD70001FB51D491D481E4CFBF74AFFFFF7C2FFB8
:10CD800023784BB9FFF7DCFE1A491848FBF754FB30
:10CD9000642003F003FAF3E7FFF71EFE1649134879
:10CDA000FBF736FF03AA02A901A8FFF761FD1349AB
:10CDB0000E48FBF741FB01990C4804F0C2FD1049F5
:10CDC0000A48FBF739FB0299084804F0BAFD0D49FF
:10CDD0000648FBF731FB0399044804F0B2FD034811
:10CDE00004F064FD04B010BD2BAD01005893FF1F8B
:10CDF000B09CFF1FC2A0010045AD010051AD010074
:10CE000055AD01005BAD0100F7B50D4D0C46174661
:10CE1000002301228DE80C00697B23460246286925
:10CE200000F0AEFE013C7E1E3C44A64205D02869BF
:10CE300000F0BEFE06F8010FF7E703B0F0BD00BF3B
:10CE4000F49CFF1F417041F2883241F06001017093
:10CE50004286704738B50D4D01780446284600F0EB
:10CE6000AAFBE378A1789B0043EAC103217943EA56
:10CE70004103617941F0800119432846FCF7DBFD4D
:10CE8000002201212846FCF7BDFD38BDF49CFF1FA0
:10CE900030B49DF808508170C2700371457130BC88
:10CEA000FFF7D8BF38B50D4D01780446284600F08D
:10CEB00082FBE379A1799B0043EAC103217A43EA2B
:10CEC0004103617A41F0C00119432846FCF7B3FDE4
:10CED000002201212846FCF795FD38BDF49CFF1F78
:10CEE00030B49DF808508171C2710372457230BC34
:10CEF000FFF7D8BF70B50C4601460A48164600F049
:10CF00005AFB013C751E3444A54205D015F8011F9B
:10CF1000044800F02FF8F7E7002201210148FCF750
:10CF200071FD70BDF49CFF1F38B50446054614F82A
:10CF30000C1B0B4800F03FFB143534F8021F084867
:10CF4000090A00F017F82178054800F013F8AC4200
:10CF5000F3D1002201210248FCF754FD38BD00BF87
:10CF6000F49CFF1F00EB4101CA81FFF7DDBF0020E9
:10CF7000704770470269D2F84432B3F5817F09D80F
:10CF8000D2F84432581C1344C2F8440283F83C11CE
:10CF900001207047012303710020704738B50A4B08
:10CFA0000360036993F84822022A044609D1D3F8A2
:10CFB000745235B1284604F0C7FA0821284604F017
:10CFC000DDFE204638BD00BF6CAD010038B514460B
:10CFD0000269D2F84432B3F5817F05461AD8D2F8F7
:10CFE0004432D2F84402C3F581730133A34202F5FF
:10CFF0009E7238BF1C4610443CBF01222A71224653
:10D0000002F0F8F92A69D2F844322344C2F84432D3
:10D01000204638BD01230371002038BD10B50446F9
:10D0200003F09EF82368C01A10BDFFFF002210B560
:10D0300002710273064A02604FF47A74054A8460F2
:10D040004FF42674417304FB0121016110BD00BF40
:10D050006CAD0100DC8CFF1F30B5094C002322446D
:10D060001D5D854206D1D55C8D4203D1044A13442F
:10D07000D87830BD0433102BF2D1002030BD00BF72
:10D0800088AD0100F8B5C3681B789B0604460E46C0
:10D0900000F19780836880211970C368122119708C
:10D0A00090F84932012B03D01AB980F8482200E0E9
:10D0B0001A46531E012B00F2868016B94FF080717C
:10D0C00003E0012E03D14FF00071404B1960022A9A
:10D0D00073D1D4F8745245B9082004F04BFE2946A8
:10D0E000074604F0DDF9C4F87472D4F874526DB1D7
:10D0F0002B79102B0AD1284604F026FA082128465D
:10D1000004F03CFE0023C4F8743256E036BB2A68B3
:10D110002F48938B9BB243F0080393832A792D4BBE
:10D1200002F1100143F8210053119B0003F1604309
:10D1300003F5614302F01F02012101FA02F21A60B5
:10D140002A68938B9BB243F0020393832B7903F1FC
:10D15000804303F5043396221E7026E0012E25D16C
:10D160002A681D48938B9BB243F0080393832A7966
:10D17000184B02F1100143F8210053119B0003F1F9
:10D18000604303F5614302F01F0296402A681E6067
:10D19000938B9BB243F0020393832B7903F180437B
:10D1A00003F5043300221A7097221A70002384F8C2
:10D1B0005E32022384F8483205E0012084F84802F8
:10D1C000F8BD0020F8BD0120F8BD00BF00E100E07F
:10D1D000E1E100000084FF1FEDE10000F0B54FF435
:10D1E0007A74B1FBF4F3B2FBF4F21D4C1B02B3FBF7
:10D1F000F2F2002354F82350194EB2EB052F03DB53
:10D200000133372BF6D100E03BB35D1E56F8237097
:10D2100056F82540A2EB0424002CA2EB0722B8BF4D
:10D220006442002AB8BF5242944216DC0D4A436859
:10D23000525D1A7056F82530B1FBF3F3C0F8503246
:10D24000094B826999428FBF0423084BB1FBF3F16C
:10D25000C9B28CBF13701170F0BD1D46E6E700BF68
:10D260009CAD010078AE0100FF6BDC02001BB70033
:10D270002DE9F0479DF824809DF8207005468A46E8
:10D2800091461E46B8F1000F06D0C3681B789B0676
:10D2900002D50020BDE8F087012249465046FFF73D
:10D2A000DBFE95F84A329945044600D02CB9B8F116
:10D2B000000F0FD04FF0000920E0B8F1000F09D0A7
:10D2C00095F84C3295F84A02002B14BF0221002138
:10D2D00002F0C6FD240204F4E06417B944F06404CB
:10D2E00001E044F003041F4B03EBC9035B681C60BF
:10D2F00085F84A9285F84C724FF0010902223146B6
:10D300005046FFF7A9FE95F84B329E42044600D0E6
:10D3100028B9B8F1000F0FD04846BDE8F087B8F142
:10D32000000F09D095F84C3295F84B02002B14BF32
:10D330000221002102F094FD240204F4E06417B9F4
:10D3400044F0640401E044F00304064B03EBC6031D
:10D3500001205B681C6085F84B6285F84C72BDE863
:10D36000F08700BF38B00100F7B5044617469DF8B6
:10D3700020009DF824209DF828600D4631B9DFF883
:10D38000B4E0DEF8001041F0400107E0012907D1C8
:10D39000DFF8A0E0DEF8001041F08001CEF80010C8
:10D3A000002184F8551284F84972616917B9202365
:10D3B0000B7015E0002814BF282720270F7027685E
:10D3C00001D0984201D9590000E04100C9B239703A
:10D3D000E16920B198428CBF40005800C0B208708B
:10D3E00012B994F84A22D2B216B994F84B62F6B246
:10D3F000002301939DF82C300093294633462046A4
:10D40000FFF736FF0C9A0A492046FFF7E7FE9DF822
:10D41000342029462046FFF735FE94F84922A368B8
:10D420000AB9802200E0C0221A7003B0F0BD00BF2C
:10D43000006CDC0234800440F7B504460E46154605
:10D440001F4602F08DFE01900DB9D4F8785202F01B
:10D4500087FEA36801901A78920602D5B4221A704A
:10D460002AE025B101A8FFF7D9FD85420CD9E36870
:10D470001B7803F0200303F0FF02002BF1D1A36817
:10D4800084F84922B0221A70A3681B7803F02003A5
:10D4900003F0FF0583B9062384F85532D4F890329F
:10D4A00001331EBFD4F890320133C4F89032D4F85F
:10D4B00070321BB3984721E094F84832013B012BAE
:10D4C0001BD802F0B9FA1EB1012E01D10D4B00E0BC
:10D4D0000D4B1B78834210DB0F2802DC01253D70C9
:10D4E0000CE0103836B1012E04D1064BC0B21870D2
:10D4F000354603E0044BC0B218700125284603B03E
:10D50000F0BD00BF19E400E018E400E02DE9F743A6
:10D5100090F84C3290F84A5290F84B62002BF6B2D9
:10D520008946EDB214BF022100210446304602F0C4
:10D5300097FC0121284602F065FC0121284602F0F3
:10D540008FFC0A274FF0A008304602F07BFC014612
:10D5500088B9013F17F0FF070DD0284602F052FCB2
:10D560004346013BFDD10121284602F04BFC4346D6
:10D57000013BFDD1E8E794F84C3200930027334695
:10D5800001972A4649462046FFF772FEE3681B785A
:10D590005B060AD0A3681F70A0231A46013AFDD18A
:10D5A000A26880211170013BFDD1002384F855321F
:10D5B00003B0BDE8F0830369490083F83C110369B7
:10D5C0000122C3F844220022027183F855227047D9
:10D5D0002DE9F7431D4600238DF80330D0F844327F
:10D5E00004461646002B00F0ED800DB9D0F87852B5
:10D5F000E36812221A7020460DF103032A46FFF752
:10D600001BFF002800F0DE8094F8483213B19DF82B
:10D610000320D2B102F0A4FD02AF082347F8040DA5
:10D6200084F8546284F8553204F23B1800264FF017
:10D630000209D4F844329E4262D2002D48D03846C6
:10D64000FFF7ECFC854243D85AE0591E012900F24D
:10D65000B9800821022B84F8551284F85462C4F86A
:10D6600040222DD1D4F84432042B29D9D4F8741295
:10D6700001200D6884F85E02D4F84432EA7104F5A2
:10D680009F76A8802E600D68A8600868033B5D4205
:10D690009BB2C3830968C560CB82D4F87432206919
:10D6A0001968B0F1804F8A718A8208611A68C0F0E7
:10D6B00086809168002900F082801B6800229A61B0
:10D6C000A368F0221A70236994F83C211A7079E05B
:10D6D000236918F8012F1A70E3681B78980706D49D
:10D6E000002DF9D03846FFF799FC8542F4D8E3685D
:10D6F00083F8009055B33846FFF790FC854225D853
:10D7000094F85432012BA36801D1802200E0B022AA
:10D710001A70D4F844329E420FD2012384F8553255
:10D72000D4F88032013302D1D4F870320AE0D4F850
:10D7300080320133C4F88032F6E7002384F8553292
:10D74000D4F86032002B3DD098473BE0E268137874
:10D75000DBB2D90611D5042384F855321023137097
:10D76000A36880221A70D4F88C320133DCD0D4F84C
:10D770008C320133C4F88C32D6E7DB071DD566B98D
:10D78000022384F85532D4F88432013311D0D4F80E
:10D7900084320133C4F884320BE0032384F8553219
:10D7A000D4F8883201331EBFD4F888320133C4F86C
:10D7B0008832A36880221A70B6E7013639E7012162
:10D7C00091607AE703B0BDE8F0832DE9F341154697
:10D7D000002204469DF82080099E8DF80320002B2E
:10D7E00000F05D81B3F5827F03D3052380F85532C5
:10D7F00055E1C0F83421C0F85832C0F838210EB9CC
:10D80000D0F87862E36812221A7020460DF1030303
:10D810003246FFF711FE002800F0418194F84832AB
:10D8200013B19DF80310D9B102F09AFC6D000923E1
:10D8300084F8553202AF236947F8040D45F001051D
:10D84000EDB284F854821D70E3681B789D074AD4BA
:10D85000002EF9D03846FFF7E1FB8642F4D842E0CB
:10D860005A1E012A00F21B810922022B84F855223C
:10D8700084F854822DD1D4F85832042B29D90123AD
:10D8800084F85E32D4F8743220691A68B0F1804F9F
:10D89000D171106091801A6801D3916809B9012192
:10D8A0009160D4F874221B681168002604F13000DE
:10D8B000DE60D4F8583208618E71012088821168C8
:10D8C00088601168013B58429BB2CB831268886123
:10D8D000D382A368F0221A706D00236945F0010518
:10D8E000EDB21D70DBE0E36802221A7026B101A8D8
:10D8F000FFF794FB864254D9E2681378DBB2D9066D
:10D9000011D5042384F8553210231370A3688022A4
:10D910001A70D4F88C32013317D0D4F88C3201331A
:10D92000C4F88C3211E013F0010FA36814D0022266
:10D9300084F8552280221A70D4F8843201331EBF35
:10D94000D4F884320133C4F88432D4F87032002B16
:10D9500000F0A5809847A2E00A2284F85522D4F866
:10D960005822012A0CBFA822A0221A7023691B7812
:10D970000225D4F83821D4F858329A4280F08F80AA
:10D9800094F855320A2B40F08A80E3681B78980798
:10D9900017D4002EF9D001A8FFF740FB8642F4D837
:10D9A0000FE0A36880221A70012384F85532D4F85E
:10D9B00080320133C9D0D4F880320133C4F88032C8
:10D9C000C3E7E3681D70F6B101A8FFF727FB8642A5
:10D9D0008CBF00200120D4F83831D4F8582202330B
:10D9E000934212D010B194F85D3273B1D4F838314B
:10D9F000D4F85822013393420BD200283ED094F839
:10DA00005D3233B93AE03046E5E7A368A8221A70E0
:10DA1000ECE7002384F85D32A368B0221A70236912
:10DA20001A78D4F83831591C2344C4F8381183F8D3
:10DA3000302094F85432012B05D12023013BFDD135
:10DA4000A36880221A7080B1012384F85532D4F87B
:10DA5000803201331EBFD4F880320133C4F88032E3
:10DA6000D4F87032BBB1984715E0D4F8643284F82A
:10DA70005502002B3FF47DAF98477AE7D4F8383150
:10DA80005A1CC4F8382122692344127883F83020C4
:10DA900000283FF46EAF012384F85D3268E702B0DE
:10DAA000BDE8F081036993F85532013B052B0AD894
:10DAB000DFE803F0070305070E0702207047032085
:10DAC0007047042070470079003018BF012070476C
:10DAD0000120704773B50446154602F041FB0190E2
:10DAE0000DB9D4F8785202F03BFB02AE46F8040DB3
:10DAF00094F85532072B21D9002DF9D03046FFF785
:10DB00008DFA8542F4D801A8FFF788FA85420DD82E
:10DB100094F84832022B09D194F85E3233B194F86C
:10DB20005532072BFBD8012384F8553294F855322F
:10DB3000072B06D9012384F8553202E0002DF5D0D9
:10DB4000E1E78023013BFDD194F85502B0FA80F063
:10DB5000400902B070BDF8B5069E0C461546074652
:10DB60001A46294633462046FFF732FD32462946FB
:10DB70002046FFF7AFFF3846BDE8F840FFF792BFF9
:10DB8000F7B5099D04460E460BB900200EE09DF83E
:10DB9000207001950097FFF718FE2A46314620466F
:10DBA000FFF798FF0028F0D0D4F8380103B0F0BD9B
:10DBB000D0F83421D0F838319A423FBFD0F8343110
:10DBC0005A1CC0F83421C01834BF90F830004FF010
:10DBD000FF307047D0F83421D0F838319A423DBF39
:10DBE000D0F83431C01890F830004FF0FF30704753
:10DBF0000069FFF7EFBFFFFF2DE9F0410446C06861
:10DC0000A36805781A78D2B20E469106EDB216D501
:10DC100012F0100F94F85E2208D0022A00F0AC80B7
:10DC200094F85E22032A40F0D280A5E0022A00F098
:10DC3000BB8194F85E22032A40F01A82B4E115F009
:10DC4000100F05F0400303D010210170002B49D0C4
:10DC500003F0FF01002B4AD094F855320C2B04D16D
:10DC6000D4F86832002B40F0A98205F0040505F0D5
:10DC7000FF07F5B10B2384F855320023C4F8443272
:10DC8000A368D0221A7023691B785B0884F8563287
:10DC9000D4F86C3203B19847D4F844320BB984F805
:10DCA0003C31236994F83C211A700123C4F84032B6
:10DCB00018E0B74BB74984F85C720322002E18BFF6
:10DCC000194694F84B0202F0FDF80C2384F8553203
:10DCD000A368C4F83871C0221A7023691B785B08E6
:10DCE00084F85632E36802221A70BDE8F08102F02F
:10DCF000100202F0FF03F2B115F0010513D1D4F8C0
:10DD00004022D4F844329A4207D2D4F840325A1C06
:10DD10002344C4F8402293F83C5123691D70A36842
:10DD2000D0221A70DEE7A368C0221A7023691B781C
:10DD300084F85512D6E794F855220C2AD2D184F8EB
:10DD40005C329449924B94F84B02002E18BF19464E
:10DD5000032202F0B7F823691A78D4F83831B3F502
:10DD6000817FD2B2BED8D4F83831591C2344C4F8CC
:10DD7000381183F83020B5E7D4F874321A68928BE2
:10DD8000120600F1F58094F85E22032A0ED1027883
:10DD90001206FCD51A79804B1A70002384F85E3283
:10DDA000D4F84432013BC4F8403208E01A797B4B86
:10DDB0001968012393400B4200F007822CE1D4F84C
:10DDC00040322269234493F83C3113708AE794F877
:10DDD0005522082A64D105F0100202F0FF016AB151
:10DDE0000023042284F85E3284F855221022027047
:10DDF000A26880211170C4F840325FE015F001057F
:10DE000023D084F85E12D4F8402262B9022284F84A
:10DE10005522D4F88422013211D0D4F88422013260
:10DE2000C4F884220BE0032284F85522D4F8882217
:10DE300001321EBFD4F888220132C4F88822802221
:10DE40001A70E36802221A70DEE0D4F84022013230
:10DE5000C4F84022D4F844128A420ED394F85422D3
:10DE600084F85552012A0CBF8022B0221A70E36850
:10DE700002221A70D4F86032C8E094F85E22012AB7
:10DE80009DD1F121022284F85E221970D4F87432F7
:10DE90001979434B1970236994F83D11197075E095
:10DEA00094F85522092A49D1EE0615D5042384F8A1
:10DEB000553210230370A36880221A70E36802228F
:10DEC0001A70D4F88C32013300F09E80D4F88C3272
:10DED0000133C4F88C3297E0E90711D50222802182
:10DEE00084F855221970E3681A70D4F8843201332B
:10DEF00000F08A80D4F884320133C4F8843283E09D
:10DF000094F85E22012A0CD1E121022284F85E22DB
:10DF10001970D4F874321979214B197023691B7860
:10DF200034E00A2284F85522D4F85822012A0CBF82
:10DF3000E822E0221A7023691B78D3E694F8552270
:10DF4000012A13D194F85422012A0CBF8022B02256
:10DF50001A70E36802221A70D4F88032013353D069
:10DF6000D4F880320133C4F880324DE08022D8E604
:10DF700094F85E22022A7FF406AF1979094B1970D2
:10DF8000A368F0211970032384F85E32E368ABE6DE
:10DF90005DE2000051E200001C8000402C80004047
:10DFA0001B8000401F800040D4F874321A681B792F
:10DFB000928B12F0800F40F0A48094F85E22032A26
:10DFC00075D0834A116801229A400A4200F0FD8010
:10DFD000804A1370D4F874321A797F4B1A70002378
:10DFE00084F85E32072384F85532A36880221A70C1
:10DFF000E36802221A70D4F89432013304D0D4F8C2
:10E0000094320133C4F89432D4F87032002B00F00B
:10E01000DC80BDE8F04118476E4B1A70D4F87432BA
:10E020001A796D4B1A70002384F85E32072384F846
:10E030005532D4F89432013304D0D4F894320133F9
:10E04000C4F89432EF0611D5042384F85532D4F87D
:10E050008C3201331EBFD4F88C320133C4F88C32B9
:10E06000E36810221A700023C4F84032A368E6E681
:10E07000D4F83821D4F8581202328A424BD094F89E
:10E080005522012A03D194F85D22002A43D0D4F806
:10E090003831D4F85822013393423FD294F85532A4
:10E0A000012B79D194F85D32002B37D174E04B4AC3
:10E0B0001370002384F85E32A368B0221A70D4F87B
:10E0C0005832013BC4F83831D4F838315A1CC4F8FE
:10E0D000382122692344127883F8302094F854328E
:10E0E000012B05D12023013BFDD1A36880221A70AA
:10E0F000E36802221A70002384F85532D4F864329F
:10E1000084E794F85E22022A7FF457AF32490B70FD
:10E11000A368E82136E7E8221A70B8E7002384F8FC
:10E120005D32A368B0221A70D4F838315A1CC4F892
:10E13000382122692344127883F8302094F854322D
:10E14000012B05D12023013BFDD1A36880221A7049
:10E15000E36802221A7094F85532012B0BD1D4F8DF
:10E16000803201331EBFD4F880320133C4F88032CC
:10E17000D4F8703204E0002384F85532D4F86432C5
:10E1800003B1984794F85532DBB2012B1DD194F8B6
:10E190005D227AB1BDE8F081D4F838315A1CC4F858
:10E1A000382122692344127883F83020E368022260
:10E1B0001A70E7E784F85D32BDE8F0810022C4F808
:10E1C0003421D4F8380198474FE5BDE8F08100BF0D
:10E1D0002C8000401E8000401F8000401C800040BA
:10E1E00000210148FFF708BDDC8CFF1F0121014819
:10E1F000FFF702BD748FFF1F70B5C3681B7803F073
:10E200002003044603F0FF057BB980F8555290F8CF
:10E210004B0201F091FDD4F86832C3B1C4F8345117
:10E22000D4F83801BDE87040184790F85C320133EB
:10E23000DBB2012B80F85C3203D890F84932012B15
:10E2400005D094F84B02BDE8704001F075BD70BD7B
:10E2500000210148FFF7D0BFDC8CFF1F01210148DE
:10E26000FFF7CABF748FFF1F38B50C4B0C4D0D4C18
:10E2700018460021FEF7DAFE2A462146184607F026
:10E2800095F9094B01211846FEF7D0FE2A46214692
:10E290001846BDE8384007F089B900BFF49CFF1F5D
:10E2A000B08CFF1F9DCF0000E09CFF1FC38B1B04A1
:10E2B00041BFC38BC1F3080103F47E43194358BF28
:10E2C000C1F30E01C183C38B9BB2C3827047FFFFB2
:10E2D000436819685A6810B50C6822430A600268DE
:10E2E000154911601549D16001F18041116114494E
:10E2F0001160417A134A5C180A3194F8244053F8AB
:10E30000211002EBC40464682160017A5C1803EBFD
:10E310008101247EC96902EBC40464682160817AAA
:10E32000581803EB810390F830005B6B02EBC002DE
:10E330005268136010BD00BF01401F00011000387B
:10E3400000001F8038B0010070B5036B1A79304BA4
:10E350001A70C36A1A792F4B1A70026B12791A70ED
:10E36000826A0446002A3FD04368D9688A4203D9AA
:10E37000521A8262012110E0C36A511E1868FFF729
:10E3800095FF236BA16A1868FFF790FFA16A00232D
:10E3900011F1FF3118BF0121A362E36A1B681868FD
:10E3A00004F124029042226805D1D36894F8243005
:10E3B00043F000430EE0D06810F0804F186815BF9E
:10E3C0001D681D680088007814BF023501351D6086
:10E3D00040F000435363236B1A790F4B1A70A9B1B5
:10E3E000E26A12791A7070BD03680C491A63D96227
:10E3F000D96821F08041D960032380F82530406B33
:10E40000036811461B68BDE87040184770BD00BF27
:10E410001F8000401C8000401B80004000000FFF58
:10E4200008B50248FFF790FF08BD00BF0C92FF1F20
:10E430003C232DE9F041B0FBF3F403FB14020A7016
:10E44000B4FBF3F203FB124318244B704FF46163E7
:10E45000B0FBF3F3B3FBF4F204FB12338B7007222F
:10E460003C4BB0FBF3F0031DB3FBF2F2C2EBC20274
:10E470009B1A01330024CB70224640F26D184FF0F6
:10E48000640E4FF4C87CE6B206F2B27313F00307D1
:10E490000ED193FBFEF50EFB153565B993FBFCF52C
:10E4A0000CFB1535002D14BF45464FF4B77504E03D
:10E4B00040F26D1501E04FF4B7752A44904204F123
:10E4C0000104E0D28E7197B9642593FBF5F405FB46
:10E4D00014347CB94FF4C87593FBF5F405FB143480
:10E4E000002C40F26D1408BF4FF4B77404E040F202
:10E4F0006D1401E04FF4B774121B64264FF4C87416
:10E50000DFF854E0801A93FBF6F206FB123693FB19
:10E51000F4F204FB12330022012AD5B206D147B926
:10E520004EB9002B14BF1C241D2405E012F80E4028
:10E5300002E01C2400E01D24844205D801320C2A8C
:10E54000A0EB0400E8D11546013501304D7108718A
:10E55000BDE8F08180510100B4AF010038B5054C31
:10E5600023688342054603D00349FFF761FF256016
:10E5700038BD00BF089DFF1F0C9DFF1F08B5FFF7AA
:10E58000EDFF024B987900F2B27008BD0C9DFF1FA1
:10E59000F0B52C4B827940F2B271534364254FF4AD
:10E5A000C876A1F2B274A24211DD8C070DD191FBA5
:10E5B000F5F405FB141424B991FBF6F406FB1414CE
:10E5C0001CB903F5A83303F5C0730131E9E702F282
:10E5D000B27264244FF4C87546791B4FDFF86CE0C3
:10E5E00092FBF4F104FB112492FBF5F105FB1125DC
:10E5F000012102F003028E4211DD022907D132B956
:10E6000004B925B903F5181303F56E5305E007EBBC
:10E61000010C1CF801CC0EFB0C330131EBE7427806
:10E620008178C2EB02124FF46164920004FB012274
:10E6300001780A4401790548013900FB012018449A
:10E64000F0BD00BF8033E101B4AF01008051010093
:10E65000094B1860094B1B681844094B1860094B9B
:10E6600002221A70084B82B01B680193019A074B73
:10E670001A6002B0704700BF149DFF1F4492FF1F35
:10E68000249DFF1F189DFF1F889DFF1F209DFF1FBA
:10E69000F7B51B4B1B4C1A682168DFF87CE000259E
:10E6A000DEF8000001900198801AB0F57A7F02F53B
:10E6B0007A7701F1010603D331463A460125EFE7A7
:10E6C0000DB11A602160104D23682A689A4213D850
:10E6D0000E4B1B6883B1984710B1FFF7B9FF0BE0F1
:10E6E000084B1A680A4B1B6813440A4A2B601378BC
:10E6F000003318BF01231370206803B0F0BD00BFC2
:10E70000209DFF1F149DFF1F249DFF1F1C9DFF1FA9
:10E710004492FF1F189DFF1F889DFF1F08B5FFF73C
:10E72000B7FFFFF71BFF014B987808BD0C9DFF1F3B
:10E7300008B5FFF7ADFFFFF711FF014B587808BD93
:10E740000C9DFF1F08B5FFF7A3FFFFF707FF014B65
:10E75000187808BD0C9DFF1F08B5FFF799FFFFF75C
:10E76000FDFE014B187908BD0C9DFF1F08B5FFF792
:10E770008FFFFFF7F3FE014B587908BD0C9DFF1F7B
:10E7800008B5FFF785FFBDE80840FFF7F7BEFFFFBC
:10E7900070B5059C049E632C05460848CCBFA4F2C6
:10E7A000B2741E34847146718570037141700270B9
:10E7B000FFF7EEFEBDE87040FFF74ABF0C9DFF1F5C
:10E7C00010B50446806808B106F0AEFF94F9060063
:10E7D000002803DB0021C0B201F042FB204610BD3F
:10E7E00070B5054680680E4608B106F09DFFEB7BCC
:10E7F0002C7BA3420CBF0324042414FB06F4A4B214
:10E80000AC80204606F088FFA86028B1224600218F
:10E8100000F08AFE6E8070BDA880688070BD70B404
:10E82000C27B047B151B6C42C1F381066C41FF293E
:10E83000C1F38112C1F30115467301F003068CBFC9
:10E840000021012101708168C2730573867341B193
:10E85000511B4A424A41A24203D0418870BCFFF793
:10E86000BFBF70BC704738B5437804460D463BB116
:10E8700090F90600002803DB0021C0B201F0F0FA95
:10E880006378A5714BB12846012101F0E9FA2846C9
:10E890000021BDE8384001F0B5BA38BD70B50E466C
:10E8A000002104464170C17181600161194615461D
:10E8B000FFF7B5FF31462046FFF792FF2046294675
:10E8C000FFF7D1FF204670BD72B6BFF35F8FBFF375
:10E8D0004F8FBFF36F8F0120704780F31088BFF315
:10E8E0005F8FBFF34F8FBFF36F8FBFF35F8FBFF3A8
:10E8F0004F8FBFF36F8F70472DE9F74F894606465C
:10E9000001F09AF8A0F11103EE2B94BF103880208B
:10E910007F4B804C804A814DDFF82CB2DFF82C828F
:10E92000DFF82CA27E4FC0B21870236843F08063DA
:10E930002360136843F0804313602B68CBF80030EA
:10E9400000232B60336888F800901B683046984796
:10E95000744B754A197811705A788AF800207348F8
:10E960009A780270724AD978117019793970A9F1C0
:10E9700006018DE82008814645469046042945D881
:10E98000DFE801F0030F161D3C006A4A03211170F5
:10E990001278694A116821F0020111600420674968
:10E9A0001BE0644A042010701278654A03210CE0D1
:10E9B000604A042010701278614A022105E05D4A25
:10E9C0000420107012785E4A0121117012785A4AA0
:10E9D000116821F00201116058490860EFF3108BB3
:10E9E000FFF772FF00B130BF5846FFF776FF0020F7
:10E9F0000860116841F00201116007E04D4A0421EE
:10EA0000117012784E4A002111701278DA68454967
:10EA1000D00701D51A2202E0100702D521228A6010
:10EA200043E0D00601D50422F9E7900601D5102273
:10EA3000F5E7500601D51622F1E7100601D50922A7
:10EA4000EDE7D00501D50A22E9E7900501D50D22B1
:10EA5000E5E7500501D50B22E1E7100501D51E229F
:10EA600022E0D10401D502221EE0900401D5072244
:10EA70001AE0510401D5062216E0100401D5152232
:10EA800012E0D10301D524220EE0900301D5222209
:10EA90000AE0D10201D5252206E01003F7D4510384
:10EAA000F5D4920201D523229A601F4A4FF0000B41
:10EAB00082F800B08AF800B089F800B088F800B099
:10EAC0001A7983F800B083F801B083F802B083F8B4
:10EAD00003B03A701B4F83F804B0C3F80CB09B68C6
:10EAE0003B60336830465B68984723680A4A85F87C
:10EAF00000B043F0806323601368386823F08043DC
:10EB00001360019B009A1B68136003B0BDE8F08F8F
:10EB100015E400E004700440007004400C900440D0
:10EB200004C007402CA0FF1F00C0074002C00740E0
:10EB300003C0074001E0074010E000E010ED00E0F6
:10EB400002E007400082FF1F289DFF1F0482FF1F75
:10EB500001C007402DE9F8433D4B1D78012D0446C7
:10EB600073D0D0E90A67DFF8F4904FF00008304620
:10EB7000394606F081FB00B317B1B7FA87F202E01D
:10EB8000B6FA86F22032C2F13F02212A15D859F88E
:10EB9000323083F8808209EBC2030120596802F108
:10EBA000200304EB83035B680B60002105F0D8FAB7
:10EBB00026EA000627EA0107D9E7032D01D0052D33
:10EBC00043D1244B94F87C201A7094F87D205A701D
:10EBD00094F87E209A7094F87F20DA7094F8802060
:10EBE0001A7172B65720616D01F09EF8A16D582020
:10EBF00001F09AF8E16D592001F096F8216E5A2043
:10EC000001F092F8616E5B2001F08EF862B6A36E9F
:10EC10001BB9114B4FF400021A60E36E1BB90E4B87
:10EC20004FF080721A60236F1BB90B4B4FF00072CC
:10EC30001A60636F1BB9084B4FF080621A60A36FB4
:10EC40001BB9054B4FF000621A60BDE8F88300BFA6
:10EC50000482FF1F57E400E088E100E038B00100C3
:10EC60002129F8B505460C4617461E4614DC01233B
:10EC700080F825300A460120002105F071FAD5E917
:10EC80000A2310431943C5E90A01254446EA071639
:10EC900085F830602046F8BD4FF0FF30F8BDFFFF2B
:10ECA00021281ED804291CD8DFE801F00709050334
:10ECB0000B00092306E00A2304E0082302E00C23EA
:10ECC00000E00B2372B6074A02EBC00041680A68F5
:10ECD00022F4702242F0807040EA03430A600B6025
:10ECE00062B6704738B001002DE9F84FA94F397866
:10ECF0000129054600F04B81D0E90A23A6480329E3
:10ED0000C0E9002302D0052940F08B80A34C236882
:10ED100003F40003AB66236803F08073EB6623689B
:10ED200003F000732B67236803F080636B6723682D
:10ED300003F00063AB679A4B4FF4000E4FF0806115
:10ED40004FF000624FF080764FF00070C3F800E0A3
:10ED50001E60186019601A60C3F800E1C3F8006112
:10ED6000C3F80001C3F80011C3F8002100F064FEED
:10ED7000DFF84CE28B4E8C498C4AA0F11103EE2B4C
:10ED80009EF8003085F87C30337885F87D300B783C
:10ED900085F87E30137885F87F30854B94BF103826
:10EDA000802093F800C085F880C0C0B28EF80000C3
:10EDB000307008701070187072B67E4B7E49D3F8B0
:10EDC0009C216A65D3F8A021AA65D3F8A421EA653D
:10EDD000D3F8A8212A66D3F8AC316B66572000F02F
:10EDE000A3FF7549582000F09FFF7349592000F098
:10EDF0009BFF71495A2000F097FF6F495B2000F09C
:10EE000093FF62B64FF4000323604FF080732360DA
:10EE10004FF0007323604FF0806323604FF0006376
:10EE20002360DFF8A0A1654CD5E90A89D3464046A6
:10EE3000494606F021FA002800F0A980B9F1000F38
:10EE400002D0B9FA89F602E0B8FA88F62036C6F19F
:10EE50003F06222E00F29B80AB1906F1200293F8A8
:10EE600030100AEBC60305EB82025B68186850603D
:10EE7000081102D0821E012A7FD85BF836204FF09D
:10EE8000000E82F880E202284FF480721A6003D1EB
:10EE90001A6842F0030208E0032807D11A6842F01A
:10EEA00002021A601A6822F001021A603B78032BF2
:10EEB00001D0052B05D101F00F01F0B2FFF7F0FEF4
:10EEC0005BE0032804D002280CBF0223032300E0E8
:10EED0000123022E02D1E278134310E0042EF2B295
:10EEE00002D16278134334E0062A03D1E27842EA81
:10EEF000031304E0072A04D1E27842EA8303E370B3
:10EF00003BE0092A03D1627842EA831321E00A2A0E
:10EF100002D1A278134328E00B2A03D1A27842EA57
:10EF2000031322E00D2A03D1A27842EA83031CE0F6
:10EF3000102A03D1627842EA83030AE0152A03D13A
:10EF4000E27842EA8313DAE7162A04D1627842EAC9
:10EF50000313637011E01A2A02D1227813430BE0E5
:10EF60001E2A04D1A27842EA8313A37005E0212A65
:10EF700003D1227842EA8313237032460120002114
:10EF800005F0EEF828EA000829EA01094FE7BDE894
:10EF9000F88F00BF0482FF1F709DFF1F08E100E093
:10EFA00088E100E058E400E059E400E05AE400E0C1
:10EFB0005BE400E00084FF1FE18900002CA0FF1F3C
:10EFC00057E400E038B0010072B6074B03EBC00015
:10EFD0004268136823F0877323F4803343F080730F
:10EFE000136062B6704700BF38B001002DE9F843E6
:10EFF000604B614A1F681F6003F5804316681968FB
:10F000001660196002F58052A3F5805314681D68DC
:10F0100014601D60594B1B78063B032B40F2A78000
:10F02000574BD3E900894046494606F025F9D0B14F
:10F03000B9F1000F02D0B9FA89F102E0B8FA88F10B
:10F040002031C1F13F01212900F29180C8B2FFF7C0
:10F05000BBFF01200A46002105F082F828EA0008DB
:10F0600029EA0109DFE7F90401D503227DE0BA04AA
:10F0700001D5042279E0BB0601D5182275E017F00E
:10F08000100701D0212270E0F00303D53D4B1F6033
:10F09000BDE8F883B10301D5012266E0F20701D58E
:10F0A000102262E0B30701D511225EE0370701D5D7
:10F0B00012225AE0700701D5132256E0310301D520
:10F0C000192252E0720301D520224EE0230701D518
:10F0D00009224AE0E70601D50A2246E0660601D584
:10F0E0000B2242E0200601D50C223EE0A10601D50C
:10F0F0000D223AE0E20701D50F2236E0A30701D541
:10F10000162232E0670701D517222EE0A60501D5A9
:10F110001B222AE0E00501D51C2226E0610501D56D
:10F120001D2222E0220501D51E221EE0EB0701D59B
:10F1300002221AE02F0601D5052216E0EE0601D5BF
:10F14000062212E06C0701D507220EE0280701D540
:10F1500008220AE0A90701D50E2206E0AA0601D579
:10F16000142202E06B0602D51522064B1A60BDE898
:10F17000F88300BFA0900440A0A004400482FF1FB9
:10F18000709DFF1F0082FF1FFFF730BF70B52B4D32
:10F190002B78012B04464FD0032B01D0052B18D11F
:10F1A000274E337884F8273000F046FCA0F1110395
:10F1B000EE2B94BF10388020C0B2307072B6214B55
:10F1C0002149D3F89421214B55201A6000F0ACFD61
:10F1D00062B61F4B618D19801E4B1A68D2075EBF45
:10F1E0001A6842F001021A601B4A44BF012384F8E6
:10F1F00038301368E362194B1868206318480668B2
:10F200006663002606600520106019602B78032BCA
:10F2100001D0834208D1134B1A68002284F82820B9
:10F220004FF400121A6004E00F4A137943F001030F
:10F2300013710B4BC1221A6070BD00BF0482FF1F07
:10F2400055E400E00084FF1FE18900007C9DFF1F62
:10F25000789DFF1F388004400400044008000440EB
:10F260000000044008E100E02CA0FF1F1B4B00221F
:10F2700010B51A601A4B1B78012B04462DD0032BB6
:10F2800001D0052B11D194F828301BB9154B4FF440
:10F2900000121A60144B94F827201A7072B6134BA0
:10F2A0005520196800F040FD62B6114BE26A1A6001
:10F2B000226B5A60626B43F8042C94F8393023B9FE
:10F2C0000C4A137803F07F03137094F8383023B995
:10F2D000094A136823F00103136010BD00000440C5
:10F2E0000482FF1F88E100E055E400E07C9DFF1FE1
:10F2F000040004400050064038800440012380F898
:10F30000253041857047FFFF0B4B1B68DB0712D58B
:10F310000A4A0B4B1B88116811FA83F31360094BDF
:10F3200080221A60084B1B78032B01D0052B02D1D9
:10F33000064B24221A60704738800440889DFF1FC6
:10F34000789DFF1F000004400482FF1F0082FF1F02
:10F35000FFF7DABF7047FFFF104B1B78012B1CD063
:10F360000F4A002111700F4A11680F4A032B1160D8
:10F3700013D10E4A136843F48023136002F5283238
:10F38000CC32137803F07F031370094B1A7842F0E4
:10F3900001021A701A78D207FCD570470482FF1F49
:10F3A000109FFF1F889DFF1F4CA0FF1F348004404B
:10F3B000942007400B4B1B78032B11D10A4A13787A
:10F3C00043F080031370094B1A7802F0FE021A70A2
:10F3D0001A78D207FCD4064A136823F480231360FA
:10F3E000704700BF0482FF1F0021074094200740A0
:10F3F00034800440844641EA000313F003036DD1D6
:10F40000403A41D351F8043B40F8043B51F8043BE7
:10F4100040F8043B51F8043B40F8043B51F8043BEE
:10F4200040F8043B51F8043B40F8043B51F8043BDE
:10F4300040F8043B51F8043B40F8043B51F8043BCE
:10F4400040F8043B51F8043B40F8043B51F8043BBE
:10F4500040F8043B51F8043B40F8043B51F8043BAE
:10F4600040F8043B51F8043B40F8043B51F8043B9E
:10F4700040F8043B51F8043B40F8043B51F8043B8E
:10F4800040F8043B403ABDD2303211D351F8043B2E
:10F4900040F8043B51F8043B40F8043B51F8043B6E
:10F4A00040F8043B51F8043B40F8043B103AEDD2DD
:10F4B0000C3205D351F8043B40F8043B043AF9D22E
:10F4C000043208D0D2071CBF11F8013B00F8013B01
:10F4D00001D30B8803806046704700BF082A13D30E
:10F4E0008B078DD010F003038AD0C3F10403D21A26
:10F4F000DB071CBF11F8013B00F8013B80D331F85A
:10F50000023B20F8023B7BE7043AD9D3013A11F8D9
:10F51000013B00F8013BF9D20B7803704B78437044
:10F520008B7883706046704701B5EAB1102A17DB0B
:10F5300000F0070333B1C3F10803D21A013B00F80E
:10F54000011BFBDCC9B241EA012141EA01418C46C1
:10F55000D308013BE0E8021CFBDC12F0070203D0F9
:10F56000013A00F8011BFBDC01BD00BFF0B5374AD2
:10F57000374B11680906FCD4196811F08001F8D1E5
:10F5800072B634480378002B5DD0334B334A1F6882
:10F5900004330C321B6852F80C6C52F8085C52F8B9
:10F5A000044C12683B4433442B4423441344C3F3B8
:10F5B0004E032B4A43F4004313602A4B1F68043365
:10F5C00040321B6852F80C6C52F8085C52F8044C3C
:10F5D00012683B4433442B4423441344C3F34E0387
:10F5E000214A43F400431360204B02F500221F68B8
:10F5F000043310321B681668556894683B440C321B
:10F60000334412682B4423441344C3F34E03184A73
:10F6100043F400431360174B1F68043340321B68E8
:10F6200052F80C6C52F8085C52F8044C12683B44D7
:10F6300033442B4423441344C3F34E030E4A43F490
:10F6400000431360017062B6F0BD00BF24B00340F8
:10F6500024B00B40819DFF1F38B0034040B00340F1
:10F660002CB0034058B0034030B0034038B00B40DA
:10F670002CB00B4058B00B4030B00B4010B5204BB5
:10F680002048214960221A70E1225A701F4B204AFB
:10F690001C78204B082C01D1012402E00A2C03D154
:10F6A00039240460132005E00C2C0CBF35243D24C4
:10F6B00004601220086014601860174B17491B780B
:10F6C000174A03B101230B601360164B164A1978D1
:10F6D000164B012901D880210BE0042901D884218F
:10F6E00007E0082901D8852103E0102994BF86216D
:10F6F0008721116019600E4B01221A7010BD00BFE6
:10F700000040074008B003400CB003404892FF1F80
:10F7100008B00B400CB00B40849DFF1F20B003408D
:10F7200020B00B404992FF1F24B0034024B00B408F
:10F73000819DFF1F0E4B1A7860B1BAB90121197073
:10F740000C4B1B7823B10C4B1A6003F500231A6095
:10F75000FFF794BF52B11870064B1B78002BF7D0FF
:10F76000054B186003F500231860F1E7704700BFF0
:10F77000849DFF1F819DFF1F24B003400C2804D9E6
:10F78000102828BF1020102307E00A2804D80828D2
:10F790008CBF0A23082300E00C230A4AD9B2081AB6
:10F7A0001070094A107883420BD0084B11701B78F7
:10F7B0002BB1074A0023136002F500221360FFF704
:10F7C0005DBF7047809DFF1F4892FF1F819DFF1FF7
:10F7D00024B0034010B5144B1B7804460BB1FFF75F
:10F7E000C5FE012C114A02D80023136018E0042C36
:10F7F0000F4903D8042313600B6011E0082C04D8D0
:10F80000052313600B6008230AE0102C95BF062324
:10F8100007231360136095BF0B600B601023202338
:10F82000044A137010BD00BF819DFF1F24B0034028
:10F8300024B00B404992FF1F28282DE9F04150D8F1
:10F84000294B1C5CFF2C4CD0284B1B780BB1FFF7CD
:10F850008DFE210617D472B6254E264F3460012343
:10F860003B7062B6234D72B633681A0604D5224B3C
:10F8700000221B682A7026E02B78002BEED062B69F
:10F8800002F092FAEFE772B61C4EDFF8808004F0C7
:10F890004007FFB204F03F05336817B123F01003AF
:10F8A00001E043F01003164C33600123C8F8005008
:10F8B000237062B672B6D8F800301B060AD5114B19
:10F8C00000221B68227062B60F4A107843FA00F0DB
:10F8D000BDE8F0812378002BDED062B602F064FA36
:10F8E000E8E70020BDE8F081FCAF0100819DFF1F2B
:10F8F00000B00340839DFF1F10B003400CB00B40CD
:10F90000829DFF1F10B00B40809DFF1F00B00B4079
:10F91000094A136843F480531360084B1A78084B64
:10F920000AB1802200E0C0221A70064B80F30C005E
:10F9300000B21880704700BF2C800440849DFF1FD8
:10F9400021C00C4000C00C407FB51C4B6A4603F13F
:10F9500010066D4618685968144603C40833B3424C
:10F960002246F7D1164B1A7812F0020F1E4601D12B
:10F97000144B1EE0144A137813F0700318BF137071
:10F98000124B80221A70002203F8032C33221A71C2
:10F990000322DA7072B60C4C45F0010320469847FA
:10F9A00062B6237813F07003E2D0237004E0013BC9
:10F9B00002D03278D207FAD504B070BD26B001006B
:10F9C00001000240410D0300000002400700024018
:10F9D00008B50B4D2C462B68580301D501F078F87B
:10F9E0002368590501D500F029FF23681A0501D5C0
:10F9F00002F030FA2368DB04EDD502F0B9FAEAE749
:10FA00003480044008B5FFF7E3FF7047094908B5A3
:10FA10000B6868B16A461844A2F58052904206D33A
:10FA200005F0F6FD0C2303604FF0FF3008BD0860C1
:10FA3000184608BD4C92FF1FEFF31380A8B9EFF3EF
:10FA40001082A2B9EFF3058323B10F2B05D9084A21
:10FA5000985C03E04FF4807000E01046EFF31183F0
:10FA60002BB1984228BF184670474FF0FF307047BF
:10FA7000F0E300E030B503460020B3FBF2F402FBF4
:10FA80001433092B94BF30333733DBB20B54234686
:10FA90000CB10130F1E70A1823465470C41AA3428E
:10FAA00006DACC5C1578CD5402F801490133F5E74C
:10FAB000084630BD2DE9F04381EAE17985B00F4673
:10FAC000A9EBE1790146064615461C4605F028FBE0
:10FAD00078B30021304605F0FBFA002814BF04205B
:10FAE00003204845B4BFC0EB09050025002F07DA05
:10FAF00060192023844202D004F8013BFAE7002574
:10FB000030464FF07E5363F31E00002105F0E0FA0B
:10FB100010B12D232370013441234E226370E31C66
:10FB20002270A2705819202283423CD003F8012B86
:10FB3000FAE726F000487749404605F0F1FAA8BBFD
:10FB40004046744905F0CEFA804678BB0021304625
:10FB500005F0BEFA002814BF042003204845B4BFB6
:10FB6000C0EB09054546002F07DA601920238442BF
:10FB700002D004F8013BFAE700250021304605F0E9
:10FB8000A7FA10B12D2323700134492323704E238B
:10FB900046226370E31CA27058192022834202D0CF
:10FBA00003F8012BFAE700230370B0E002AB01AACF
:10FBB0002946304605F01FFD814665B9019B53B9C2
:10FBC00090F80090544B554AB9F1340F94BF9146C8
:10FBD000994601230193019B5B429D42BCBFDFF824
:10FBE0003C916B424846B8BF019306F087F8019BF1
:10FBF00098428046C8BF00F10108002B02D108F1ED
:10FC0000010825E024DA1DB32B44984205F10208CF
:10FC10001ED9A946B9F1000F07DD3046404905F06D
:10FC2000B9F809F1FF390646F4E7002DACBF691BAE
:10FC3000294602AB03AA304605F0DDFC019B039A7E
:10FC4000691CD21A8A4208BF0133814608BF01935A
:10FC5000029808B108F10108C8EB0703002B04EB78
:10FC6000080208DD1A44214623442026994203D085
:10FC700001F8016BFAE7234610B12D211970013309
:10FC80000199002909D135B11946302001F8020B3C
:10FC90002E2058700B462E2522E0FCDA002DFAD0DB
:10FCA0001D46302005F8020B2E265E702B46C91A21
:10FCB00000255E1803D503F8010B0125F9E7002D97
:10FCC000E9D00196E7E7581C19F8011B1970824228
:10FCD00009D001990139019109B9981C5D70034659
:10FCE0009A42F0D800E01346002F0DDA47447F42D5
:10FCF000194620207A1A1A44002A02DD01F8010B65
:10FD0000F8E7002FA8BFDB1900221A70204605B0C3
:10FD1000BDE8F083FFFF7F7FEE97010047AB010056
:10FD2000000020417047FFFF1030024B43F82010C5
:10FD3000704700BF0084FF1F194B03EBC0004268EF
:10FD400002F14043A3F592217C2910D9A3F5942117
:10FD50007C290ED9A3F596217C290CD9A3F59821ED
:10FD60007C290AD9A3F59A237C2B08D970470D4921
:10FD700006E00D4904E00D4902E00D4900E00D499F
:10FD800072B6136823F0877323F4803343F08073D3
:10FD90001360C2F38402084B41F8223062B6704708
:10FDA00038B001005092FF1F8892FF1FD892FF1FAA
:10FDB0000893FF1F2893FF1F25FD0000014B1868C3
:10FDC000704700BF00D00340044B054900221A6071
:10FDD0000A60044A106010221A60704714D0034071
:10FDE00004D0034000D0034020B11028034628BFB0
:10FDF000102300E00123024A10781370704700BFFF
:10FE00003093FF1F212810B518D80D4B53F8302020
:10FE100092F880423CB1012311B182F8803010BDCC
:10FE200082F8003110BD03EBC0035B681A6811B1A2
:10FE300042F0030201E022F002021A6010BD00BF8E
:10FE400038B0010021289FBF044B53F8303093F89D
:10FE50000002C0B288BF0020704700BF38B0010068
:10FE6000212810B52BD8164A02EBC00301295B6884
:10FE7000144601D004290FD154F83020012082F813
:10FE800080024FF4A2721A601A6804290CBF42F073
:10FE9000200222F0200211E052F83000002280F807
:10FEA000802211B94FF4807208E0022902D140F299
:10FEB000031203E0032908BF4FF481721A6010BDDA
:10FEC00038B00100212870B50E4659D8042A57D8F9
:10FED000DFE802F0070905030B00092306E00A2307
:10FEE00004E0082302E00C2300E00B231D04254B53
:10FEF00003EBC0035C68216811F4E06101D1FFF7F6
:10FF0000AFFF214B214AC3F89C21214AC3F8A0210D
:10FF1000204AC3F8A421204AC3F8A8211F4AC3F8E5
:10FF2000AC2104F14043A3F592227C2A10D9A3F519
:10FF300094227C2A0ED9A3F596227C2A0CD9A3F50B
:10FF400098227C2A0AD9A3F59A237C2B08D970BD64
:10FF5000134B06E0134B04E0134B02E0134B00E09D
:10FF6000134B72B6226822F47022226042F0807134
:10FF7000C4F3840243F8226045EA0103236062B6B9
:10FF800070BD00BF38B001000084FF1F758CFF1FDB
:10FF9000498CFF1F1D8CFF1FF18BFF1FC58BFF1F9F
:10FFA0005092FF1F8892FF1FD892FF1F0893FF1FD8
:10FFB0002893FF1F282838B504464D4B0FD11B78D6
:10FFC0000B2B03D8C3F10C03994003E00C2B1CBF8F
:10FFD0000C3B19410846BDE83840FFF799BC1A7838
:10FFE0000125002905FA02F301DC002102E08B4221
:10FFF00004D82946FFF706FF294674E00338C3B248
:020000021000EC
:10000000012B01D83B4B06E0202C01D0192C01D14B
:10001000394B00E0394B1B6803FB0113D3401D280B
:1000200059D8DFE800F03F45392758581B21585868
:10003000585858585858582D330F15585158585823
:100040005858584B2E4A136040F244422D4B40E022
:100050002D4A136040F244422C4B3AE02C4A136084
:1000600040F244422B4B34E02B4A136040F24442AE
:100070002A4B2EE02A4A136040F24442294B28E0E2
:10008000294A136040F24442284B22E0284A136078
:1000900040F24442274B1CE0274A136040F244429E
:1000A000264B16E0264A13604FF45172254B10E0A0
:1000B000254A13604FF45172244B0AE0244A13601E
:1000C0004FF45172234B04E0234A1360234B4FF447
:1000D00051721A6038BD7F29D4BF0021012120460A
:1000E000FFF790FE01212046BDE83840FFF7B8BE7B
:1000F0003093FF1F0890034008800B4008800340A6
:100100001080034004B004401880034008B004404D
:10011000208003400CB004402880034010B004400D
:100120003080034010C004403880034014C00440B5
:100130004080034018C00440488003401CC0044075
:1001400010900340309004401890034034900440D5
:1001500010800B4048A0044018800B404CA0044085
:1001600072B60B4B0B4A0C491B681268096862B6E1
:10017000490102D5322B88BF0132C3F5BB33602061
:10018000FF33B3FBF0F34FF47A7000FB023070479B
:1001900018E000E0889DFF1F04ED00E038B504463C
:1001A000FFF7DEFF054624B938BD013C0AD005F54E
:1001B0007A75FFF7D5FF401BB0F57A7FF5D201F0D5
:1001C000F3FDF6E738BDFFFF214B4FF4000210B5F9
:1001D0001A604FF080721A604FF000721A604FF090
:1001E00080621A604FF000621A601A4B1A4A1B4C68
:1001F00000204BF6FF71186059602823136093604C
:100200001361936113629362136393630922226003
:1002100004F58054043420606160A360236144F8D5
:10022000042C04F5FE2420600D4801600D490B608C
:100230008B600D4B1A60FFF721FA1920FFF7AEFF14
:1002400000F052FF40F21310BDE81040FFF7A6BFC8
:1002500008E100E0048003400C800340008003407C
:1002600008800B400C800B4000800B40254A13682F
:1002700043F480631360244A00231370234A1370ED
:10028000234A1370234A1370234A1370234B1B789D
:100290002BB1152B07D140F21332214B02E0214B39
:1002A00040F213321A60204B1B78012B05D0052B2E
:1002B00007D14FF451721D4B02E01D4B4FF45172A8
:1002C0001A601F281B4B98BF2020C0F344321A70BD
:1002D000C0F347125A700221042200F01F009872E6
:1002E0009A70D9745A7588221A743C22DA70124BAB
:1002F00040226FF44A711A700B444FF400521A6096
:10030000704700BF34800440139EFF1F919DFF1F64
:100310001C9EFF1F149EFF1F909DFF1FD29DFF1F5D
:1003200018C0044040A004403193FF1F1CC004408B
:1003300044A0044000A006402DE400E0134B9A784E
:1003400002F0EC0100F003020A43410748BF42F00B
:1003500010029A700D4900F00F02042A02BF8A7938
:1003600042F040028A715A79C30602F0EF02074B4D
:1003700048BF42F010025A719A79810602F0EF02EA
:1003800048BF42F010029A71704700BF00A00640BB
:100390001D4B1B685B0510B500D410BD1B4C2378AA
:1003A00003F0FF0213B101F0FFFCF8E7184B4FF424
:1003B00000511960174BDA70174B1B782BB1152BB6
:1003C00007D140F20312154B02E0154B40F2031225
:1003D0001A60144B1B7803F07F03012B05D0052B0B
:1003E00007D140F20312104B02E0104B40F203120F
:1003F0001A600F4A002313700E4A13700E4B1B68CD
:100400000BB101221A7010BD34800440909DFF1F73
:1004100084E100E000A00640D29DFF1F18C0044008
:1004200040A004403193FF1F1CC0044044A004407E
:10043000139EFF1F919DFF1F8C9DFF1F0A4A38B519
:100440000446137803F0FF05002BFAD10121204662
:10045000FFF706FD29462046FFF7D4FC034B53F86F
:100460003420034B1A6038BD909DFF1F38B0010047
:10047000189EFF1F10B509B140F08000144A137890
:100480009842144622D0134A126852051DD503F033
:100490007F03012B04D0052B05D100220E4B01E078
:1004A0000E4B00221A60002900F07F0214BF602367
:1004B0004423012A05D0052A07D143F44073064A94
:1004C00002E0064A43F440731360207010BD00BF81
:1004D0003193FF1F348004401CC0044044A00440FA
:1004E0000E4B1A78824218D00D490968490513D578
:1004F0002AB1152A05D10B4A0021116001E00A49F1
:100500000A6028B1152807D140F21331054A02E0EC
:10051000054A40F21331116018707047D29DFF1FD9
:100520003480044018C0044040A0044038B50D4B4E
:100530001B6813F480634FF0000410D021280A4D8B
:100540000AD80A4B012153F830302B60FFF788FCA2
:100550002B681C70012038BD2C60204638BD184621
:1005600038BD00BF348004408C9DFF1F38B00100AF
:100570000E4B1B6813F4806316D012280C4B03D16A
:1005800040F202310B4A04E0142809D10A4A40F231
:10059000023111605A7B42F001025A730120704708
:1005A0005A7B02F0FE025A730020704734800440E8
:1005B00000A006400CA0044014C004402DE9F843FC
:1005C0001F4B1B685A05064637D51E4B1B680BB1DF
:1005D00001221A701C4DDFF880902C781B4F0134DB
:1005E000402C28BF0024C84699F80030A34219D1F6
:1005F000FFF722FA402810DC3B791B06F4D599F866
:100600000030134A0133402B28BF0023D25CDBB2F9
:10061000D2B2FA7188F80030E6E7FF28E4DD01F095
:10062000C3FBE1E70A4BF6B21E550A4B01221A70D2
:10063000064BE4B2BC222C70DA70BDE8F88300BF30
:1006400034800440189EFF1F1C9EFF1F00A0064020
:10065000929DFF1F909DFF1F149EFF1F2DE9F84FD5
:10066000264B1B685A050646884645D5244B1B6811
:100670000BB101221A70234FB246B94606EB0803AC
:100680009A4536D23C78204BDFF87CB01B78013499
:10069000402C28BF00249C420AD01C4B1AF8011B96
:1006A00019551B4B0121E4B2197089F80040E5E7A8
:1006B000184DBC23EB70FFF7BFF9402810DC2B79F5
:1006C0001B0611D59BF80030104A0133402B28BF80
:1006D0000023D05CDBB2C0B2E8718BF8003003E0DD
:1006E000FF2801DD01F060FB9BF800309C42E2D066
:1006F000D3E7084BBC22DA70BDE8F88F34800440A1
:10070000189EFF1F1C9EFF1F149EFF1F929DFF1F20
:10071000909DFF1F00A0064010B5034C237813B135
:1007200001F042FBFAE710BD909DFF1F064B1878C1
:10073000064B1A78C0B2D3B298422CBF3F3303F1B4
:10074000FF33181A704700BF1C9EFF1F149EFF1F27
:10075000054B1878054B1A78C0B2D3B2984238BF0F
:100760004030C01A704700BF139EFF1F919DFF1FAE
:1007700010B5104B104C1B782278D9B2D2B29142EE
:1007800014D0531C402B28BF00230C4AD05CDAB293
:1007900022700B4A1268C0B252B18B4288BF4031FE
:1007A000CB1A1A2B04DC0023137010BD4FF0FF305E
:1007B00010BD00BF139EFF1F919DFF1FD39DFF1F04
:1007C0008C9DFF1F084B1A78084B1B78DBB29A42AE
:1007D00007D00133402B28BF0023054AD05CC0B2AC
:1007E00070474FF0FF307047139EFF1F919DFF1F12
:1007F000D39DFF1F0C4B1B685B0514D50B4BDA78A0
:1008000002F0CB02DA7040225A74DA7842F03402F5
:10081000DA70074B074A1B78DBB21370064B1B6874
:100820000BB100221A7070473480044000A00640CB
:10083000919DFF1F139EFF1F8C9DFF1FF0B5344934
:100840000B7913F0300F2FD072B68B7D03F0FF04BD
:1008500023B9CB7940234B7462B625E062B62D48AC
:100860002D4A037812782D4FDBB2D2B20546581CC0
:100870004028CE7928BF00209042F6B21CBF3E54DB
:100880000346601E10F0FF04F1D1D9B2297024494B
:10089000096849B1934236BFC2F140029B1A9B18C6
:1008A000272BC4BF01230B70194AD178C9B20D069A
:1008B0001ED513791C061BD51A4B1B481D780378CF
:1008C0001A4EEDB2DBB2AB420AD00133402B28BF47
:1008D00000231479F45CE4B2D471147D072CF2D9AE
:1008E000DBB203700A4B1A79100644BF7C22DA701F
:1008F00049060CD5064B1A79520608D50C4A002138
:1009000011700C4A126802B111703C22DA70F0BD0D
:1009100000A00640139EFF1F919DFF1FD39DFF1F48
:100920008C9DFF1F1C9EFF1F149EFF1F929DFF1F8B
:10093000909DFF1F189EFF1FF0B50C4C0C4E2378A6
:100940000C4D43F0020706EBC70283F00103506031
:100950002A782370002A14BFC820882082F0010260
:1009600040EA01412A7046F83710F0BD889EFF1F0B
:100970000080FF1F009FFF1F431E032B10B510D8E0
:1009800072B6094A52F8230048B1416842F8231070
:100990000649048831F81320121B21F8132062B68F
:1009A00010BD002010BD00BF789EFF1F3CA0FF1FA0
:1009B000013803280AD872B6054B53F820300020BE
:1009C00013B101305B68FBE762B6704700207047E7
:1009D000CC9EFF1F70B472B6174C184901231A1928
:1009E00012F8012C12071DD59A00144E51F83250FE
:1009F0002DB906EB431308305860114B09E042F063
:100A0000010251F832506DB906EBC203083058604C
:100A10000C4B46F832300C4A1378013B137062B627
:100A200070BC70470133052BD9D162B6064B00224A
:100A30001A7070BC00F0B8BBE0B101000080FF1F6D
:100A400088004000C8004000F69EFF1F431E032B95
:100A500010B532D8194A400140F01000104472B667
:100A6000174AD45C032C0BD8DFE804F01804020703
:100A7000052414E00830022411E0083004240EE0BC
:100A80001048114A50F8234014B940F8231002E0EE
:100A900052F82300416042F823100DE00324D4549F
:100AA00010F0080F01F108030A88436014BFC8233F
:100AB000882343EA0243036062B610BD0080FF1F33
:100AC000349EFF1FCC9EFF1FDC9EFF1F00BE7047A1
:100AD0002DE9F74FA94B1C78E4B214F0040F1D4622
:100AE0001AD0A74B1B78A3B1A64A117801F0FF03D7
:100AF00021B1013BDBB2137003B900BEA24A1178E9
:100B000001F0FF0329B1013BDBB213700BB900F018
:100B1000A3FC9A4A0423137004F0080303F0FF02B5
:100B2000002B00F07182994B994C1B78DBB21F09A6
:100B30004FEA930640F0EC8104EBC603596854F881
:100B40003630C3F38303013B0C2B00F2DD81DFE879
:100B500013F09A019A01DB01DB01DB01DB01DB0110
:100B6000DB01B901DB01DB01DB010D000A68894D06
:100B700089484B682A6001216B60DFF85082874BFF
:100B8000017092B240F2816044F8363082424FF0F8
:100B90000003C8F800302361A36117D8B2F5D06F05
:100BA00080F02781B2F5817F00F0D88006D8802AB6
:100BB00000F0C180822A00F0C28035E140F20233A9
:100BC0009A4200F00781B2F5A06F1AE042F22100CC
:100BD000824200F055810CD8B2F5086F00F0A58074
:100BE000B2F5106F40F02081654AA97811701E4659
:100BF0000AE042F221218A4200F00E8142F22133C2
:100C00009A4200F015810FE1A219136A1F0603D55D
:100C1000506A083800F0C8FA0836802EF4D1DFF8A0
:100C2000B0915F4F0026CA4659F826004FEA860B5E
:100C300030B14268009200F0B7FA009A1046F7E728
:100C4000584B594A4AF80B004BF803005BF8020076
:100C500040B141680192009100F0A6FA0099019A12
:100C60000846F5E7514B42F80B0023F816003B7895
:100C70004F4A023B4BF80200032B07D8DFE803F092
:100C800002040204002300E001233B700136042E1D
:100C900007F10107C8D1474B474E404F00221A7059
:100CA0004FF0010B9946454A0BEB06015A4411F8E7
:100CB000011C920011F0080F11704FEA8B0A24D02A
:100CC00000F054FA38B104EB4B1208303C4B506042
:100CD00044F83A3006E099F8002044F83A0001322E
:100CE00089F8002000F042FA4AF0010230B104EB2A
:100CF000C2010830486044F8327006E044F832001F
:100D000099F80020013289F800204AF002010BF125
:100D1000010B4AF0030A0022BBF1050F44F8312011
:100D200044F83A20BFD1134683E0154B254E1B787B
:100D300033700B4680E0234E337073707BE0AA88DB
:100D400002F07F02042A6FD81E4E92003370737037
:100D50001D4B9B5C9C076ED531706CE0AA8802F03D
:100D60007F02042A60D86B88002B5DD1164992005F
:100D700011440A7822F0020239E000BF80200740C7
:100D8000FF9EFF1F899EFF1F019FFF1F90200740AE
:100D90000080FF1FEC9EFF1F009FFF1FC800400048
:100DA000349EFF1F249EFF1FCC9EFF1F3CA0FF1FF1
:100DB000DC9EFF1FF69EFF1FE0B1010030C801104E
:100DC00088004000F79EFF1FC0200740209EFF1FA5
:100DD000789EFF1FAA8802F07F02042A24D86B881D
:100DE00013BBA549920011440A7842F002020A702E
:100DF0001FE06A88A988A14B5E68AEB1188890424E
:100E000008D15888884205D1120A032A0CBF3378CA
:100E10001B8911E00C33EFE7994A1168994A116078
:100E2000994AA978117004E0934B0F221A7027E0B9
:100E300000231E4600E00223EC889C4228BF1C468B
:100E4000402C254628BF402530462946FFF774FD33
:100E5000641B2E4403D1402D12D1254603E0402CC3
:100E6000254628BF402530462946FFF765FD641B0F
:100E70002E4401D1402D03D1844BC8F800601C8062
:100E80000122834B3FE0834B1A8842F221039A42AE
:100E900014D1814A0023C85C98540133072BFAD13E
:100EA0007D4B1B68862B08BF7C4B4FF0000108BFB1
:100EB0000F22084608BF1A70FFF73EFD784B44F832
:100EC000363021E0774F3E68A6B1DFF8C081B8F830
:100ED0000040402C254628BF402530462946FFF7D4
:100EE0002BFD601B80B2A8F8000008B9402D00D18E
:100EF00070193860674B1A88B2F5A06F04D10022D0
:100F00005A709A78684B1A70614B01221A7077E018
:100F100004EBC605013F6A6803F00803A2F108006C
:100F2000FFB203F0FF0E002B36D000F03DF95F4812
:100F30005F4A50F82710E9B14B6840F8273001F1BB
:100F400008036B60D35D032B0BD8DFE803F00204CA
:100F50000608032304E0022302E0052300E0042343
:100F6000D35515F0080F0A8814BFC823882343EA15
:100F7000024343E0D35D032B07D8DFE803F0414190
:100F80000204002306E0012304E015F0080F14BF5B
:100F900003230223D35533E054F836301B0C99B2A7
:100FA00022F8081C23B3434B22F806EC42F804EC69
:100FB00053F82720DFF82CE112B943F8270002E0AC
:100FC0005EF8273058603C4A4EF8270032F8173058
:100FD0000B4422F8173000F0C9F810B108306860EF
:100FE00006E0364A44F8360013780133137007E000
:100FF000334A2B4B15F0080F08BF134644F8363020
:10100000304A0823137065E5E0071ED520492C48B7
:101010002D4C02230B702D4B1A702D4B18609860CD
:101020002C48D8601A619A615C60134B0D201870CF
:101030002948FF2303702B700274284A1370284B31
:101040009F221A7001230B7012E0210604D50A4B6F
:101050000D221A7080232B70A20705D51E4A137823
:10106000DBB2137002232B70E30644BF10232B70F6
:1010700003B0BDE8F08F00BFC0200740E4B101001D
:10108000889DFF1F4CA0FF1F109FFF1FF49EFF1F96
:1010900094200740EC9EFF1F44A0FF1F899EFF1F66
:1010A000C8004000209EFF1F98200740CC9EFF1FD5
:1010B000349EFF1F789EFF1F3CA0FF1FF69EFF1F60
:1010C0008800400080200740389EFF1F889EFF1F39
:1010D0000080FF1F8C9EFF1F882007408C20074048
:1010E00084200740249EFF1F10B500F0A7FF0023B7
:1010F000194819461950C4180833882B164A6160DC
:10110000F8D116490B6843F480230B60144BC2F3EB
:1011100007211970C2F30741120E19751A76114A88
:10112000FF2313700021137202F8703C0123137522
:1011300082F8801013710C4B70226FF450711A708A
:101140000B444FF400721A6003F1C04303F5C82347
:1011500010221A7010BD00BF0080FF1F34800440B1
:101160009C2007408020074049E400E010B572B69B
:101170000B480268B2FA82F10B2902DD62B6002048
:1011800010BD4FF00043CB4022EA0302026062B67A
:10119000044C48234B43E0180022E250426010BD4B
:1011A0003493FF1FBC85FF1F0C4B4822C31AB3FBAF
:1011B000F2F30B2B11D80A4A127822B1094A12789D
:1011C0000AB1FFF707BC72B607494FF0004222FA96
:1011D00003F30A681A430A6062B67047BC85FF1FB2
:1011E000F69EFF1FFF9EFF1F3493FF1F10B5104C8C
:1011F00023686BB1206843885A1C03441C7A038817
:101200009A4212D3FFF7D0FF094B00221A600DE07B
:10121000084B1B7813B94FF0FF3010BD0320FFF7C8
:10122000ABFB20600028E5D1F5E74280204610BDE9
:101230000C9FFF1FFF9EFF1F10B50B4C236813B1BF
:1012400022686AB902E0094B1B7813B94FF0FF30EE
:1012500010BD0320FFF790FB20600028F0D1F5E7D8
:1012600053881344187A10BD0C9FFF1FFF9EFF1F69
:10127000044B9888044B1A681AB1138852889B1A39
:10128000184470473CA0FF1F0C9FFF1F10B5094B6F
:101290001B786BB1084C206818B1FFF785FF00235D
:1012A00023600320FFF768FB10B1FFF77DFFF8E72D
:1012B00010BD00BFFF9EFF1F0C9FFF1F2DE9F84FC1
:1012C000314DDFF8D490012382460C462B700E4638
:1012D0004F46002E53D0D9F800303BBBDFF8B0B0FA
:1012E0004AF2F928294B1B7803F0FF010BB929704A
:1012F00015E00420FFF75CFB072807D801232B70BB
:10130000FFF734FF386088B91F4B1870B8F1010837
:1013100002D09BF8003033B11D4B01221A704FF000
:10132000FF30BDE8F88F00F03FFDDBE7184B0021F0
:10133000197039684B88C3F14000B04228BF30466D
:1013400003EB000E0B44A1F802E0361A07330AEB58
:101350000008C24504D01AF8010B03F8010FF8E7A2
:101360004B883F2B06D940230B800420FFF76EFBF0
:1013700000233B60074B05221A70C246A9E72E7076
:101380002046BDE8F88F00BF029FFF1FFF9EFF1F92
:10139000089FFF1F019FFF1F049FFF1F07B502ABA0
:1013A000012103F8010D1846FFF788FF03B05DF82F
:1013B00004FBFFFF38B50E4C0E4D012323702B6844
:1013C0007BB90D4B1B7813B90020207038BD042069
:1013D000FFF7EEFA0728F7D8FFF7C8FE28600028C5
:1013E000F2D02B68588800232370C0F1400038BD2C
:1013F000029FFF1F049FFF1FFF9EFF1F2DE9F0416B
:10140000114B1B78F3B1114F114B3C68114D012664
:101410001E7098464CB1002663882E7021462380AA
:101420000420FFF713FB3E6009E0FFF79FFE014633
:1014300020B104202C70FFF709FB00E02E70002380
:1014400088F80030BDE8F081FF9EFF1F049FFF1F5A
:10145000029FFF1F019FFF1F38B50E4B1B7803F043
:10146000FF05ABB90C4C216831B14B880B800420CF
:10147000FFF7ECFA256038BDFFF778FE014620B192
:101480000420BDE83840FFF7E1BA044B01221A708E
:1014900038BD00BF029FFF1F049FFF1F019FFF1F5A
:1014A00030B572B6254C89B9016879B103790F2B33
:1014B0000CD822881A41D20708D503F1007303F52E
:1014C0009063B1EB431F01D162B630BD2188002388
:1014D00041FA03F212F0010227D101259D40294370
:1014E000218062B6164DD9B201712C6844F0020415
:1014F0002C6055F8044C03F1007344F0020445F8E5
:10150000044C03F590630F4C5B0182252560A176A6
:10151000A1772176E17703601A605A609A60DA60F9
:101520001A615A619A61DA6130BD0133102BCFD153
:1015300062B600220260037130BD00BF129FFF1F20
:10154000408004400080004003790F2B10D8094AE6
:10155000137072B608490279012303FA02F20B886C
:1015600023EA02030B8062B6102303710023036099
:10157000704700BF1A800040129FFF1FEFF31080DA
:1015800072B6B0FA80F04009704700B162B6704799
:10159000F8B50C4E0C4F0025FFF7F0FF34680246FB
:1015A0006CB1636933600BB19D6100E03B60104634
:1015B000FFF7EBFF6577A36820469847ECE7FFF756
:1015C000E4FFF8BD149FFF1F189FFF1FFFF7E0BF48
:1015D00015490B6830B513B98360C36009E004682E
:1015E0001A68944207D20025121B8360C560D86038
:1015F0001A60086015E002681C689968121B026096
:1016000061B10C68A2420B46F5D28160C968C16025
:10161000D860C168A21A88601A6002E08160C36065
:1016200098600223037530BD1C9FFF1F70B5164DD7
:101630002C680026BCB1236813B1013B236012E083
:10164000A26802B1D36020692A60036826751B680E
:1016500022460021984763681BB123602046FFF7AC
:10166000B7FF2C68E6E7FFF789FF084B00221C68EC
:101670001A60FFF78AFF2CB1A5682046FFF7A8FF84
:101680002C46F8E770BD00BF1C9FFF1F2C9FFF1F5B
:10169000024A136801331360FFF7C8BF889DFF1F1C
:1016A0000368C9B21B6818470368C9B21B681847AA
:1016B0000368C9B21B6818470368C9B21B6818479A
:1016C00008B50846FEF77AFF012008BD08B50846B0
:1016D000FEF774FF012008BD38B508460D4604F03A
:1016E0000DFB044601462846FEF7B8FF204638BDEC
:1016F00010B5084614461146FEF7B0FF204610BD4F
:10170000FFF778B808B50846FEF732FF003018BF7B
:10171000012008BD08B50846FEF708FF003018BFD5
:10172000012008BD08461146FEF7A4BE0846FEF794
:10173000D7BE0846FEF782BEFEF72ABE4B0803F16D
:10174000376000F5D830B0FBF1F0FEF78FBD10B573
:101750004B0803F13760144600F5D830B0FBF1F0C8
:10176000FEF784FD2046BDE81040FEF7E7BDFFF719
:1017700029B8FEF7FDBFFEF7EBBFFEF7CDBFFEF7C2
:10178000D5BF70477047FFFF036830B523B1002411
:101790009C600124DC6017E0194C236843F40003CB
:1017A000236000BF174B01241C6003F58073164CA7
:1017B000036003689D683DB11033A3420360F8D90C
:1017C00000230360184630BD0468104B2260234498
:1017D0001B110F4D0322A2600E4A45F82310017918
:1017E000995444335A11920002F1604202F5614269
:1017F000012003F01F0300FA03F3136030BD00BFA4
:101800003C800440007003403F710340008FFCBFE8
:101810004893FF1F44E400E0016830B5A1B10B4BD1
:101820000B441B1103F144025511012402F01F0265
:1018300004FA02F2064C44F82520064A064C42F807
:10184000234000238B60036030BD00BF008FFCBFCE
:1018500080E100E04893FF1F85170100024B012241
:101860001A60024B1B6818470C7103404893FF1F16
:10187000024B01221A60024B5B6818471C7103403F
:101880004893FF1F024B01221A60024B9B681847C6
:101890002C7103404893FF1F024B01221A60024B38
:1018A000DB6818473C7103404893FF1F07B5064BA0
:1018B0001B88ADF80430036802225B6801A99847D1
:1018C00003B05DF804FB00BFA8B1010070B5054688
:1018D0008AB022B90368C9B21B6898472FE0012A71
:1018E00008BF0A2209B1212004E030228DF825200A
:1018F000212014E0B1FBF2F602FB1611CCB209294B
:1019000094BF04F1300104F137010AAC0444C9B2B8
:1019100004F8241C314616B10138C0B2EAE733B1ED
:101920000138C0B20AAB03442D2203F8242C2B68E3
:1019300001A9C0F1220201445B68284698470AB019
:1019400070BD0029BABF49422D2300230A22FFF7A8
:10195000BDBFFFFFFFFFFFFF2DE9F04F85B007463A
:101960001946104615461C469DF8386003F056F897
:1019700008B14D4912E024F000484FF0FF324B4BC4
:101980002846414603F04AF868B94FF0FF32474B0A
:101990002846414603F024F828B945493846F6F769
:1019A0004BFD804676E04FF06042424B2846214690
:1019B00003F02AF808B14049F0E74FF060423F4B8E
:1019C0002846214603F002F80028F4D10022002323
:1019D0002846214602F0FAFF20B104F100444FF0FE
:1019E000010800E0804636494FF0000900205FFA08
:1019F00089F39E4207D92AA3D3E9002302F074FD9C
:101A000009F10109F3E702460B462846214602F098
:101A1000B9FB0D46044603F03FF8434601468146B4
:101A20000A223846FFF752FF80469EB3484602F02E
:101A3000E5FC0B4602462946204602F0A1FB0F2E8C
:101A40004FF02E0328BF0F268DF800300DF1010551
:101A50003446013CE4B2FF2C15D00022194B02F0B1
:101A600043FD8B46824603F017F8C0B200F1300305
:101A700005F8013B02F0D2FC02460B46504659469F
:101A800002F07EFBE5E73B68721C5B68D2B26946F8
:101A900038469847404605B0BDE8F08FAFF3008068
:101AA000000000A09999B93FAAB10100FFFFEF7FA4
:101AB000B2B10100FFFFEF41AEB10100FFFFEFC186
:101AC0000000E03F00002440002310B503730360D2
:101AD00043600C68836004604C6844608C68846078
:101AE0000B604B608B6010BD10B50446006803F0BE
:101AF0001BFE204610BD38B504460D460068013176
:101B000004F066F810B184E82100012038BD436874
:101B10008B4210B5044606D2FFF7EDFF20B1A36853
:101B20000BB922681370012010BDF8B504460F46AA
:101B3000154622B9036803B11A7000230BE0114661
:101B4000FFF7E5FF064640B9206810B103F0ECFD51
:101B5000266000236360A36004E0A5603946206826
:101B600004F0C4F82046F8BD38B5002304460360ED
:101B70004360836003730D4639B1084604F0BEF834
:101B8000294602462046FFF7D0FF204638BD38B52B
:101B9000054608460C4604F0B1F8214602462846A0
:101BA000BDE83840FFF7C1BF10B50023044603600D
:101BB000436083600373FFF7EAFF204610BD38B52A
:101BC000054608460C4604F099F821460246284688
:101BD000BDE83840FFF7A9BF10B50446002386B022
:101BE00023606360A3602373084601A903F077FDB7
:101BF00001A92046FFF7E3FF204606B010BD10B54F
:101C0000044600238AB023606360A3602373084600
